:020000040000FA
:040000006FD00400B9
:101000006F00107D00000000000000009020002014
:10101000AA220020A9BDF9F56C23002000000000E1
:10102000000000006C230020902000200000000041
:101030000000000090200020000000009020002010
:101040000000000090200020902000209020002030
:101050009020002090200020402F00207A240020A3
:101060000000000090200020902000200424002098
:1010700090200020D22300209020002090200020EB
:101080009020002090200020902000209020002020
:101090009020002001A04111B7170040985F3AC688
:1010A000945F3247E39CE6FE3245410182800111A4
:1010B00013078008F337078093F787083EC20100C3
:1010C0000100B7170040930570052380B70413068D
:1010D00080FA2380C7040100010083C6B70493F699
:1010E000F60DA385D704238007049246F3A6068055
:1010F0000100010093760502D5CEF336078093F602
:10110000860836C4010001002380B7042380C70489
:1011100001000100B70614007D89558D88C70100C4
:1011200001000100010023800704A246F3A6068007
:101130000100010073370780137787083AC6010062
:1011400001002380B7042380C704010001000100CF
:1011500001003727004093061005A303D7802380A2
:101160000704B247F3A70780010001009307800836
:10117000F3B7078093F787083ECE01000100B71749
:101180000040130770052380E704130780FA2380CB
:10119000E7040100010003C7B70413670708A3852C
:1011A000E70423800704F247F3A70780010001004A
:1011B0000561828093760504BDC6F336078093F6F9
:1011C000860836C8010001002380B7042380C704C5
:1011D00001000100B7061400938606047D89558D31
:1011E00088C7010001000100010023800704C246F6
:1011F000F3A6068001000100733707801377870884
:101200003ACA010001002380B7042380C70401000B
:1012100001003727004093062005A303D7802380D1
:101220000704D24781B773370780137787083ACC12
:10123000010001002380B7042380C70401000100DE
:1012400098471367070C98C723800704E24719BF24
:101250000111814601468145114506CE97000000E7
:10126000E780C05693078008F3B7078093F7870895
:101270003EC601000100B717004013077005238028
:10128000E704130780FA2380E7040100010003C785
:101290006704136717002383E70423800704B2471A
:1012A000F3A7078001000100F2400561828041112F
:1012B000814601468145114597000000E7800051B5
:1012C00013078008F337078093F787083EC40100AF
:1012D0000100B7170040130670052380C70493066A
:1012E00080FA2380D70401000100FD552396B70240
:1012F00023800704A245F3A5058001000100733790
:101300000780137787083AC6010001002380C704CD
:101310002380D7040100010003C767041367170087
:101320002383E70423800704B247F3A70780010063
:10133000010001A0B1473305F50201007D1575FDDF
:101340008280411122C426C206C6AA8401446317C2
:101350009400B24022449244410182800504130566
:10136000803E420497000000E78000FD4180C5B741
:101370009305000273A04580824573901534924016
:101380002242B2424243D2436244F2440255925551
:101390002256B2564257D2576258F25806499649D9
:1013A000264AB64A464BD64B664CF64C065D965DD1
:1013B000265EB65E465FD65F09617300203041113C
:1013C000B7170040985F3AC6945F3247E39CE6FE49
:1013D000324541018280B71700401307000323887C
:1013E000E702854717170000232EF74473002030CB
:1013F000411122C406C637040020976000E0E78050
:10140000E0241C408297D5BF373700408347470010
:101410009146BD8B639ED702B73600401306F00F8E
:10142000973500009385051F9737000083D7872ED7
:1014300003C7A6001377F70F1DE3B7E70400BC4FFF
:101440000946894517150000034585F7829731A0A5
:1014500099466394D700834757007300203003C731
:1014600086001377F70FE365F6FC13851700AE9738
:10147000173800002310A82A2380E70075B7B78724
:10148000004003C76700098B6309071003C7770093
:101490009306000313770703630DD708173800007E
:1014A0000348D87417360000130686730547B30641
:1014B00006012380E60083C5770017370000130775
:1014C000A772429793F5F50F2300B70003C5870075
:1014D0009735000093850571C2951375F50F23802C
:1014E000A5000347070089451377F703630CB70C82
:1014F00063E7E50A6306071A8545630CB712973759
:10150000000083C7B76E3307F60003470700137761
:10151000F70F19CB850793F7F70F0D476363F71A9A
:1015200017370000A304F76CB787004009472383EF
:10153000E700B787004083C77700E207E18763DEF3
:1015400007049737000083C7776A1737000013072F
:1015500027693E9785462300D700173700001307F9
:10156000A7683E97930600032300D70017370000B3
:10157000130747673E97A14685072300D70093F7D7
:10158000F70F0D476364F71417370000A300F766E1
:10159000B787004009472383E70073002030930694
:1015A00010026300D70E930620026305D706930648
:1015B0000002E316D7F403C727021377C70F136798
:1015C0002700D5A803C767001377070465CB03C7B7
:1015D000A70217380000130828421735000013052A
:1015E0006539134707082385E70203C7A702137766
:1015F000370F136787002385E7028147130700042D
:10160000B305F5008C41B306F80091078CC2E3994D
:10161000E7FEF5B503C7A702134707042385E702D2
:1016200003C7A7021377C70F136727002385E702B5
:10163000F9B503C767001377070449C303C76702F7
:10164000173800001308082F17350000130545262A
:10165000134707082383E70203C767021377370F8F
:10166000136787002383E702814713070004B3054C
:10167000F5008C41B306F80091078CC2E399E7FEB0
:10168000BDBD03C76702134707042383E70203C7EF
:1016900067021377C70F136727002383E70285B517
:1016A00003C767001377070411CB03C7270213771B
:1016B000370F136787002381E70291B52380060067
:1016C0003DBD97370000A3830752B9BD973700008F
:1016D000A38E075075BD2303048015472303E480C0
:1016E00001002302A480828083076480E3CE07FE8A
:1016F00023030480828083076480E3CE07FE0345D2
:101700004480828083076480E3CE07FE2302A480A6
:101710008280411126C44AC24EC006C61377F50B1B
:10172000AD47AA892E899544630CF70019459700A7
:101730000000E78080FA97000000E78020FB8D44DE
:101740004E8597000000E78040F9FD59FD1463982D
:101750003401B240A24412498249410182801355AA
:1017600009011375F50F97000000E780E0F92209E1
:10177000F1BF011126CC06CEB70408009700000087
:10178000E780C0F6154597000000E78000F5970058
:101790000000E78080F697000000E78000F62AC688
:1017A00097000000E78080F432459377150089EBBD
:1017B000136515001375F50FF240E2440561828050
:1017C000FD14E9F00145CDBF397126DC4ADA4ED867
:1017D00052D656D45AD25ED006DE62CE66CCB7E779
:1017E00000E07D5783AA070022C603AA470023A072
:1017F000E71823A2E718B7170040130770052380E6
:10180000E704130780FA2380E70483C74704930B98
:1018100075FFB684E20793FBFB0F8546AA892E8BE2
:10182000328937240040E187015763FA7601630863
:10183000D5008946130700026313D5000157D98FDD
:1018400093F7F70FB71C00402382FC0411472303D2
:10185000E4801305F00F97000000E78000E8094CD2
:1018600097000000E78080E863657C15B7050700F6
:10187000DA9537870700795563FEE504B38795004D
:10188000636AF704370B0800A94733EB65016395DA
:10189000F90881E8814497000000E78020E526856B
:1018A00015A8DA85094597000000E780C0E605091C
:1018B0000345F9FFFD14050B97000000E780C0E425
:1018C00081C49377FB0FE5F797000000E780A0EA5B
:1018D00069F17D55B7170040130770052380E704B1
:1018E000130780FA2380E70403C74704418B238250
:1018F000E704F250B7E700E023A0571123A24711F5
:10190000E25432445259C259325AA25A125B825B93
:10191000724CE24C21618280A547639BF906856980
:101920001309F00FB3069900B3742B01B694134951
:10193000F9FFB3749900856B33796901416B938723
:10194000F9FFB3F7270199E363FC340193D9490008
:10195000C147E3E637FF3DBF0569C1697D19D9B7C6
:101960001305800D63886901130500026384790102
:1019700013051008CA8597000000E780C0D99700BA
:101980000000E78040DF31D54E99B38434416DBF0C
:10199000DA852D4597000000E780E0D7CA94E30B75
:1019A00099EE050997000000E78020D5A30FA9FE56
:1019B000FDB79387F9FF93F7F70F636DFC0C83C7AF
:1019C0001C04130730086315F70637070800636126
:1019D000EB06B3079B00B706100063FBD704334B3D
:1019E000EB0089476399F9068980D549E38404EAC5
:1019F000DA85094597000000E780E0D11109032747
:101A0000C9FF91472320E48003076480E34E07FE6B
:101A100023033481FD17EDFBFD14110B81C4937773
:101A2000FB0FE9FF97000000E780E0D461F155B5B6
:101A3000B717004003C75704B7070800137707021A
:101A400019E3B78707007955E376FBE833079B0076
:101A5000E3F9E7F841B58547E380F9F0DA852D45EC
:101A600097000000E78020CB9389F4FFE38404E231
:101A700097000000E78060C893F7390091EB832658
:101A800004800327090093074900E396E6E03E89B6
:101A9000CE84D9BFB5476399F9001305900B970021
:101AA0000000E78080C3FDB3B1471305B00AE388A7
:101AB000F9FE99476397F904B7050800B365BB00C1
:101AC0002D4597000000E78000C581448D4BA1495A
:101AD00097000000E78060C263967401832704804A
:101AE0002320F9008504E39534FF8327048013172E
:101AF0002B01635507002312F90069BB2322F9006B
:101B000051BB9D47639FF90281451305B0049700BF
:101B10000000E78040C0BD442320090023220900C3
:101B2000FD5997000000E78040BD93F77400CA9705
:101B300003C70700FD14398D2380A700E39334FF0A
:101B400091BBA1476397F90697000000E780A0C208
:101B50008144630D0B008D479304C0036308FB00B1
:101B60009304000563048B01930440041375C507B7
:101B7000E30295D2194597000000E78000B6970070
:101B80000000E780A0B6054597000000E780E0B4BC
:101B9000268597000000E78020B7094597000000E0
:101BA000E78080B697000000E780E0BCE31405CE34
:101BB0000DB39147639FF90013056006970000007D
:101BC000E780A0B197000000E78040B213059009BC
:101BD000F9B5E38109CCF1547DB9BD6601471736EB
:101BE00000001306E61D938606A68545834706007A
:101BF00093F7F70F91C382800507E3F9E6FE973765
:101C00000000238FB71ADDB77D1662066186931731
:101C10008601E18763D4070001458280931726007F
:101C20003307F500AE9718439C4363E7E7007D1642
:101C3000E37FF7FC7D55828005458280FD15E20536
:101C4000E18513978501618793F7F50F63480700D6
:101C5000FD15139725002A97584365D7138517005C
:101C60006205618582803308B5021C4283A80600A4
:101C7000B335B502C29733B50701AE98469585488E
:101C80006367B5006394A50063E3070181480C43D3
:101C9000C6950CC388C21CC28280814713978701F6
:101CA00061876343B7008280139727002A97232018
:101CB00007008507E5B78147014793968701E186CD
:101CC00063C5B60013351700828093962700AA9645
:101CD00094428507558FD5B793D755408A07AA9761
:101CE0009C4305453315B5007D8D828017F3FFDFDA
:101CF000E702A33D2A8497000000E78060F405C551
:101D0000931725003E940327C4FF814711EB7D15EF
:101D100016053E954205418517F3FFDF6700233D19
:101D200005838507E5B70145C5BF8147139787013F
:101D300061876343C700828013972700B386E5005D
:101D400094422A97850714C3D5B77D16620661862B
:101D5000014793178601E18763D507001335170004
:101D6000828093172600B306F500AE9794429C43F9
:101D70007D16B58F5D8FF1BF8A05AA950147636314
:101D8000B500828083A6C5FFF11593D71600D98FC1
:101D90009CC11397F601E5B72A8301480147014525
:101DA0006343D7008280B387050183A80700B30788
:101DB00006019C43C697AA976384F80033B51701C0
:101DC0000507B3080301620723A0F8006187110823
:101DD000C1BF2A8301478147014563C3D700828081
:101DE0003388E50083280800330EE600032E0E003A
:101DF0003388A8403308C8416384080133B508011B
:101E00008507B308E300E20723A00801E187110773
:101E1000E9B717F3FFDFE702432B0111B286B28463
:101E20002E86AA850A8597000000E780C0FA2A84DA
:101E3000A6850A8597000000E78020E833348000FB
:101E4000060413351500018D056117F3FFDF6700E8
:101E5000032A17F3FFDFE702C3244111AA89AE8AE0
:101E6000328BB68402C202C402C60144131C840130
:101E7000135C8C4163499C02939B1400FD1B054934
:101E8000138CF4FFF15C33048901620461846340C4
:101E9000740792478E04CE9423AEF4FE410117F3EB
:101EA000FFDF6700832313192400B30B2B01014AC2
:101EB00093172A00D69783A50B0088437800340037
:101EC000500097000000E78040DA050A93178A0166
:101ED000E187F11BE35EFCFC92474E990504232049
:101EE000F900A2473EC2B24702C63EC441B7131A28
:101EF0008901135A8A41131D240093178A01E1872F
:101F000063CF970092470A044E941CC0A24705096C
:101F10001379F90F3EC2B24702C63EC4ADB7B3074C
:101F20009A0313152A005695084178003400500092
:101F3000050AEA97DA978C4397000000E780E0D221
:101F40006DBF0000197106C212C416C61AC81ECA97
:101F500022CC26CE2AD02ED232D436D63AD83EDA69
:101F600042DC46DECAC0CEC2D2C4D6C6DAC8DECA99
:101F7000E2CCE6CEEAD0EED2F2D4F6D6FAD8FEDA49
:101F8000971500009385858B8841E70005009240F6
:101F90002242B2424243D2436244F2440255925535
:101FA0002256B2564257D2576258F25806499649BD
:101FB000264AB64A464BD64B664CF64C065D965DB5
:101FC000265EB65E465FD65F096173002030000072
:101FD0009721002093810103175100201301818272
:101FE00017F5FFFF1305450297050020938585012E
:101FF000171600201306C6FD63FAC50083220500EC
:1020000023A0550011059105E3EAC5FE170502005E
:1020100013058520971500209385C5FB1716002012
:102020001306466563FAC5008322050023A0550008
:1020300011059105E3EAC5FE171500201305856318
:1020400097450020938585236377B50023200500FD
:102050001105E36DB5FEFD42739002BC8D42739095
:102060004280B722000093828288739002309702E8
:102070000020938222F993E23200739052309752FB
:1020800000009382A29D739012346FB07477730036
:102090002030397101436EC619A0397141536AC8A5
:1020A00066CA62CC5ECE19A0397101535AD056D29D
:1020B00052D44ED64AD826DA22DC06DE33016140FD
:1020C000828241114AC026C222C406C68282B24D13
:1020D0004101024D924C224CB24B4101024B924ABB
:1020E000224AB2494101024992442244B24041018C
:1020F00082803D432A876373C3029377F700BDEF65
:10210000ADE5937606FF3D8ABA960CC34CC30CC767
:102110004CC74107E36BD7FE11E28280B306C34090
:102120008A069702000096966780A6002307B700EC
:10213000A306B7002306B700A305B7002305B70021
:10214000A304B7002304B700A303B7002303B70019
:10215000A302B7002302B700A301B7002301B70011
:10216000A300B7002300B700828093F5F50F939684
:102170008500D58D93960501D58D61B7939627007F
:102180009702000096968682E78086FA9680C117AD
:102190001D8F3E96E374C3F8A5B73367B500FD53B2
:1021A0000D8B79E7B7877F7F9387F7F710419441CD
:1021B000B372F6003363F600BE92B3E26200639737
:1021C000720C6318D6065041D441B372F6003363E3
:1021D000F600BE92B3E262006398720A631BD604F3
:1021E00010459445B372F6003363F600BE92B3E235
:1021F00062006391720A631ED6025045D445B372E1
:10220000F6003363F600BE92B3E26200639A72088E
:102210006311D60210499449B372F6003363F60095
:10222000BE92B3E26200639372085105D105E30FD9
:10223000D6F61317060193970601631CF700135790
:10224000060193D706013305F7409375F50F91E921
:1022500082804183C1833305F7409375F50F91E187
:1022600082801377F70F93F7F70F3305F7408280DB
:102270000346050083C60500050585056313D600E2
:1022800065FA3305D640828011059105E312D6FE2A
:10229000014582802105A105E31CD6FC0145828011
:1022A0003105B105E316D6FC014582804105C10523
:1022B000E310D6FC01458280B717004003C77705BD
:1022C0001377E70FA38BE704130700F8A38DE70448
:1022D0003D47238CE70413075003A38CE70403C78F
:1022E000A7051377D70F238DE7048280B717004027
:1022F00003C7E7020D8941111377C70F498F930672
:102300008008F3B6068093F6860836C60100010001
:10231000930670052380D704930680FA2380D704A0
:10232000010001002387E70223800704B247F3A7D7
:102330000780010001004101828041112A83014E82
:10234000930E407E130F0019930F400663E56E1243
:102350009308001913034006B3781503854E0D4FFB
:10236000A14F337365020D891335150063EFBE125B
:102370001308F6FF7946729842081358080133078C
:10238000C70213D61700BE0732976146B3F6C602DE
:1023900013068070B386C6023697A166F58F420792
:1023A0005D8FB716004083C7F60293F70708A303B3
:1023B000F1000346710083C7F60293F70708E39420
:1023C000C7FE83477100B716004093F7F70F638885
:1023D000071293078008F3B7078093F787083EC476
:1023E00001000100B7170040930670052380D70451
:1023F000930680FA2380D7040100010023AA070373
:1024000083C6170393E60608A388D7022380070430
:10241000A247F3A70780010001001166B71700402B
:102420007D16D45BC85F93854703A98EF18EF5FABC
:1024300093068008F3B6068093F6860836C6010038
:102440000100930670052380D704930680FA238049
:10245000D7040100010098C103C7170313670704DD
:10246000A388E70223800704B247F3A7078001008F
:102470000100410182807D133368E3039308E01675
:10248000630E08003368F3039308D016630808004E
:102490009378330093B818009388D81633081E0138
:1024A000131E0801135E0E0155B56393E50305483D
:1024B000638608000148630303002A887108729844
:1024C000FD15131E0801C205135E0E01C18179BD01
:1024D00013F8150063F4BF007908D5B71338180056
:1024E000E5BF83C7F60293F70708A303F10003468D
:1024F000710083C7F60293F70708E394C7FE83478A
:10250000710093F7F70FF1DFE9B531714AD966CB66
:1025100006DF22DD26DB4ED752D556D35AD15ECF09
:1025200062CD6AC96EC7AA8C02D897100000E780F6
:1025300020B12A8993078008F3B7078093F78708AB
:102540003EDA01000100B717004013077005238031
:10255000E704130780FA2380E7040100010003C7A2
:10256000F7021377770FA387E70203C7F702136712
:102570008700A387E70223800704D257F3A70780C9
:1025800001000100054597000000E78060D61307B1
:1025900080C13347E902116A93070AE893065002A3
:1025A000BD69930BA004814A014B13048008930476
:1025B00070057D1AB347F9023307D7023EC0FD8785
:1025C0003ECC938709A69309803E3347F7023AC26F
:1025D0007D873AC4334739038549B399990193D923
:1025E0003940B306D702B30B7703B3C6F602B3CBB9
:1025F000FB0236C6FD8636C893D6FB4136CEB746BB
:102600000F00938606243349D9028566938606FA1D
:10261000B3969601B389E902130760553309D902CD
:1026200093060010B389E9023349D902B3C9F9020C
:102630009316390036CA37190040FD8636D0930DFF
:10264000090493D7F9413ED2F336048093F6860805
:1026500036DC01000100930770052380FD0093061E
:1026600080FA2380DD00010001008346390593F6DE
:10267000860FA309D9048346390593E61600A309FA
:10268000D90423800D00E256F3A606800100010064
:10269000130C80FA116DF336048093F6860836DE4B
:1026A00001000100930770052380FD0023808D0148
:1026B0000100010083463905216693E60602A3095D
:1026C000D90483560905B3E6A6012318D904835615
:1026D0000905D18E2318D90423800D00F256F3A6E4
:1026E0000680010001008346390593F606026381E6
:1026F000061A03463905218A6DDE08189710000076
:10270000E78000987336048013768608B2C2010011
:10271000010023809D0023808D0101000100B71777
:10272000004003C637051376F60DA389C70403C618
:10273000370513660602A389C70483560905216677
:10274000B3E6A6012318D90483560905D18E2318B0
:10275000D90423800D009646F3A6068001000100EF
:102760008346390593F60602638B061483463905C2
:10277000A18AEDFE97000020E780E091AA8636D47A
:1027800097000020E7802091A256E30AD5FE8356E9
:1027900009054255B3E6A6012318D9049710000095
:1027A000E780C08F83463905A18AEDDE035609050F
:1027B0008346290582473376CA00B306DA0293D5E9
:1027C000F641B296B388F640E24733B8C6002E9879
:1027D0003308F840A247B3B616013308D84063C7A0
:1027E0000701631DF800924763FA1701C247634F60
:1027F000F80E63950701B24763EAF80E894663E96C
:10280000660FF2469315180013D3F8015E861395F0
:102810001800B365B30042D646D497C00100E780E4
:10282000E0BC3258050B137BFB0F63470001631AB2
:102830000838A2586387083813081500B336A80073
:10284000B69513D6F5013298B336C800AE96135834
:102850001800FE06B3E60601733604801376860878
:10286000B2C60100010023809D0023808D0101007C
:1028700001000356C902B296C206C1822316D902CC
:1028800023800D00B646F3A606800100010021B5A5
:10289000F336048093F68608B6C001000100238059
:1028A0009D0023808D01010001008346390593E6D8
:1028B0000602A309D90423800D0086460DB5F33620
:1028C000048093F68608B6C40100010023809D00B1
:1028D00023808D01010001008346390593E606023D
:1028E000A309D90423800D00A646BDB5E30B0BF068
:1028F000F336048093F68608B6C8010001009306FB
:1029000080FA23809D002380DD00010001008346C2
:10291000390593F5FC0F93F6860FA309D904834676
:102920003905CD8EA309D90423800D00C646F3A630
:10293000068001000100130580FA0346390593065D
:1029400039051D8A631C9629733604801376860820
:10295000B2CC01000100130680FA23809D00238081
:10296000CD000100010003C606001376F60D23809A
:10297000C60003C60600136606022380C6008356FF
:1029800009051166D18E2318D904835609052166DD
:10299000D18E2318D90423800D00E646F3A60680C5
:1029A00001000100130680FA8346390593F60602FA
:1029B0006380062683463905130C3905A18AFDDAA2
:1029C000081897000000E780A06BF336048093F6A8
:1029D0008608B6D001000100930680FA23809D008E
:1029E0002380DD000100010083460C00116693F690
:1029F000F60D2300DC0083460C0093E6060223005C
:102A0000DC0083560905D18E2318D90483560905A5
:102A10002166D18E2318D90423800D008656F3A693
:102A2000068001000100130680FA8346390593F6FB
:102A30000602638A062083463905A18AEDFE97F0D7
:102A4000FF1FE78040652A8C97F0FF1FE780A06496
:102A5000E30C85FF8356090511664255D18E231874
:102A6000D90497000000E7806063834639051306A8
:102A70003905A18AFDDAF336048093F68608B6D4C8
:102A800001000100930680FA23809D002380DD0071
:102A9000010001008346060093F6F60D2300D600E0
:102AA00023800D00A656F3A6068001000100835680
:102AB000090503462905D247B376DA003306CA0270
:102AC0001305800C9355F6413696330DF640825728
:102AD000333CD6002E9C3336A601330CFC40330C1D
:102AE000CC403308850392564E86B335A503330593
:102AF000A503C29597C00100E780408F634680011F
:102B0000631E0C16630C0D16130615003335A60054
:102B10002E959356F5013696B335D600AA95939621
:102B2000F50105828585D18E6346B000639D051A47
:102B3000638B061A0356C90215823305D600333655
:102B4000C500B2956348B000639105241306F00FE9
:102B5000637DA622894663F3561593078008F3B771
:102B6000078093F78708BED60100010037170040A1
:102B7000930770052300F704930780FA2300F704F6
:102B8000010001008356C70289678117D58FC207EC
:102B9000C1832316F70223000704B657F3A7078063
:102BA00001000100FA506A54DA544A59BA592A5AB3
:102BB0009A5A0A5BFA4B6A4CDA4C4A4DBA4D296173
:102BC00082801308F5FF3335A800FD152E951356A6
:102BD000F5013298B336C800AA9695B9F336048049
:102BE00093F68608B6CA0100010023809D00238069
:102BF000AD000100010083463905CD8EA309D9043B
:102C000023800D00D646F3A606800100010035B3EF
:102C1000F336048093F68608B6CE010001002380C7
:102C20009D002380CD00010001008346390593E615
:102C30000602A309D90423800D00F646F3A60680F8
:102C40000100010095B3F336048093F68608B6D2EE
:102C50000100010023809D002380CD0001000100C0
:102C60008346390593E60602A309D90423800D00A3
:102C70009656F3A606800100010045BB9306F5FFBA
:102C800033B5A600FD152E959355F501AE96B3B557
:102C9000B600AA951396F501858269B5F3360480CE
:102CA00093F68608B6D801000100930680FA2380C7
:102CB0009D002380DD00010001008356C9020566E6
:102CC000011693F6F60FD18EC206C1822316D902E1
:102CD00023800D00C656F3A6068001000100850A78
:102CE00093FAFA0F95B233E6B60045C20356C9020D
:102CF0003305D0403338A000B305B040B38505415B
:102D000015826345B000D1E16371A608894663F07E
:102D1000560593078008F3B7078093F78708BEDA54
:102D200001000100B7170040130770052380E70476
:102D3000130780FA2380E7040100010003D7C702CC
:102D40007D8B2396E70223800704D65781BDF33697
:102D5000048093F68608B6DC01000100930680FA31
:102D600023809D002380DD00010001008356C902FD
:102D70000566011693F6F60FD18EC206C1822316A0
:102D8000D90223800D00E656B9B793078008F3B740
:102D9000078093F78708BEDE010001003717004067
:102DA000930770052300F704930780FA2300F704C4
:102DB000010001000356C70293975600B297C2075D
:102DC000C1832316F70223000704F657C1BB9147BE
:102DD00063EEB70217D701001307C74C8A05BA95EF
:102DE0009C41BA978287B717004003A7470B13454A
:102DF000F5FF698F23AAE70A03A7070B698F23A8AA
:102E0000E70A03A7070A798D23A0A70A8280B717CC
:102E1000004083A6470B1347F5FFF98E23AAD70A74
:102E200083A6070B558D23A8A70A83A6070A758FCB
:102E300023A0E70A8280B717004003A7470B498FFA
:102E400023AAE70A03A7070B1345F5FF45BFB717EA
:102E5000004083A6470B1347F5FF758F23AAE70AA7
:102E600003A7070A598D4DB7B717004003A7470BB3
:102E7000498FEDB7914763EEB70217D701001307EB
:102E8000A7438A05BA959C41BA978287B717004035
:102E900003A7470D1345F5FF698F23AAE70C03A786
:102EA000070D698F23A8E70C03A7070C798D23A0D2
:102EB000A70C8280B717004083A6470D1347F5FF84
:102EC000F98E23AAD70C83A6070D558D23A8A70C2E
:102ED00083A6070C758F23A0E70C8280B7170040EC
:102EE00003A7470D498F23AAE70C03A7070D134536
:102EF000F5FF45BFB717004083A6470D1347F5FF01
:102F0000758F23AAE70C03A7070C598D4DB7B71788
:102F1000004003A7470D498FEDB7797122D43714CC
:102F2000004026D24AD0035924028354040206D614
:102F30004209C2044ECE52CC56CA13590901C1806F
:102F40002DE11379F9F793F4F49F4209C204135960
:102F50000901C18093078008F3B7078093F78708BA
:102F60003EC401000100930770052300F404930799
:102F700080FA2300F404010001002311240323102C
:102F8000940223000404A247F3A707800100010074
:102F9000B250225492540259F249624AD24A4561CF
:102FA0008280B7F5070081463000B10519459700CA
:102FB0000020E7806081A24713972701E34A07FCBE
:102FC0001369090893E4044093098008F3B7098062
:102FD00093F787083EC001000100930A70052300A3
:102FE0005405130A80FA230044050100010023114F
:102FF000240323109402230004048247F3A70780CC
:1030000001000100294597F0FF1FE780A032F3B9C6
:10301000098093F989084EC201000100230054057C
:1030200023004405010001008357040293E70720B1
:103030002310F402230004049247B9B7B7170040E5
:103040008847420541819377050491EB9377F50119
:103050003755E801130505803345F50282809377E3
:10306000050C130700046397E7009377F5013745D4
:103070009C1CCDB72165130505D0828037E700E0A1
:103080001C435443A183E206D58F1CC1FD57232066
:10309000F7182322F718828013178500B7E700E09E
:1030A00023A0E710618123A2A7108280B7F700E078
:1030B0008847CC478280814737370040A14663C4A8
:1030C000C700328582800345B740E38EA6FE338574
:1030D000F5000345050085072304A740CDB79707F2
:1030E0000020938727EF9C43173700201307071909
:1030F0003E95636EE500173700201307A7506368FD
:10310000A700170700202327A7EC3E858280FD57E4
:10311000EDBF8280411122C406C62A8497000000B8
:10312000E78000F22947B307E502B2408D83B3D7A9
:10313000870222449507B3D7E70237370040C2071A
:10314000C1832316F70041018280411137150E001B
:1031500006C697000000E78020FCB7370040130741
:1031600070F82381E7000D47A381E70013070004EF
:10317000A380E70005472387E700B2404101828032
:1031800037370040834727001A0593F7F703C98FA5
:1031900093F7F70F2301F7008280B737004003C78A
:1031A000170019C9D98DA380B70003C7070013679B
:1031B00087002380E700828093C5F5FFF98DA38007
:1031C000B7008280AE872A87B7360040214637385D
:1031D000004089E7170300006700E3F383C8B600E7
:1031E000E30916FF05078348F7FFFD17C20723040D
:1031F0001801C183F9BF411122C406C62A84970071
:103200000000E780E0E32947B307E502B2408D8381
:10321000B3D7870222449507B3D7E7023737004078
:10322000C207C1832316F7404101828071654111B5
:103230001305052006C697000000E78000FCB7379D
:103240000040130770F82381E7400D47A381E74052
:1032500013070004A380E74005472387E740B240F7
:1032600041018280CC41411106C6328503C615005A
:1032700083C5050022064D8E42068D654186138862
:1032800075A2630C0611634BC804138845A2630042
:10329000060D634AC800938535A26301B6082390E2
:1032A000060029464DA0138855A26305060D938597
:1032B00065A2E316B6FE8D451D4663E6E508114698
:1032C000198E63F3C7003E86B7E704002390C6005B
:1032D000FC4797D50100938565009DA0138895A2B2
:1032E00063030611634E060D1388A5A2630006133F
:1032F000938505A5E315B6FA99451D4663E5E504F2
:10330000198E63F3C7003E86B7E704002390C6001A
:10331000FC4797050020938525D61DA09D451D4699
:1033200063E3E5022146198E63F3C7003E86B7E7E3
:103330000400FC472390C6009705002093850534C0
:10334000BA9582970146B240328541018280AD45EF
:103350001D46E3EAE5FE3146198E63F3C7003E865B
:10336000B7E704002390C600FC4797D5010093857A
:1033700065F9F9B7B1451D46E3E7E5FC3546198E19
:1033800063F3C7003E86B7E704002390C600FC47FE
:1033900097D50100938505F865B78D451D46E3E493
:1033A000E5FA1146198E63F3C7003E86B7E70400BD
:1033B0002390C600FC4797D501009385E5F249B7F5
:1033C0008D451D46E3E1E5F81146198E63F3C7000C
:1033D0003E86B7E704002390C600FC4797D501005E
:1033E000938505F5B1BFA5451D46E3EEE5F42946F5
:1033F000198E63F3C7003E86B7E704002390C6002A
:10340000FC4797D501009385E5EE1DBFB5451D46E8
:10341000E3EBE5F23946198E63F3C7003E86B7E762
:1034200004002390C600FC4797D50100938505EA68
:1034300001BFB7E7040003A3071397060020938694
:10344000A6C24146A545170500201305E5B802832D
:103450002D455DE703C505000947631FE50803A87F
:103460004500411106C6034718003285034608008F
:1034700022074168518F930828FE6307170563E907
:10348000E80005186303070323900600294591A867
:10349000130648FE630AC7041518E31707FF15460D
:1034A0003E87637BF600154701A8130600023E879E
:1034B0006374F60013070002B7E704002390E600E8
:1034C000FC471316070111A83E8691C30546B7E7CE
:1034D0000400FC472390C6004206CC4541828297F7
:1034E0000145B24041018280130600083E87E37522
:1034F000F6FC13070008C9B7239006000545828033
:103500008280416779176304E504411122C406C62D
:1035100085472A84639FF500B7E70400228522448B
:10352000B24003A38713970500209385652F4101BF
:10353000028389476399F500B7E7040083A7070B67
:103540008545829771D9B2402244410182808280B0
:10355000797122D452CC2E842A8A97D50100938582
:1035600025DF17D50100130525E106D63AC626D278
:103570004AD0B68432894ECE97B00100E7804032FF
:10358000A68517D50100130525E097B00100E78057
:103590002031294597B00100E780603583478400DA
:1035A00093F70702E1E7834904008947054532475D
:1035B0006396F908544083C7160083C60600A20725
:1035C000D58FC166138616FE638CC7028D16638F76
:1035D000D7068D669386269029456391D706B7E76F
:1035E0000400A285225403A34714B250F249A686D0
:1035F0004A86925402595285624A85474561028340
:103600002D450DEF93070002354563E99702B7E7B3
:103610000400FC47484413060002CA85829781498A
:1036200097070020938787209C43014581CB9C43CB
:1036300091C74E852686CA8582970145B25022548D
:1036400092540259F249624A456182802D457DF7C4
:103650009307700F3545E3E397FEB7E70400FC4797
:1036600048441306700FCA8582975DBF2145F9B79C
:10367000411122C437E404008327841326C2AA849C
:10368000416506C697050020938585197D158297AB
:103690008327C40A170500001305E5E6858882978D
:1036A00095C0032304132244B2409244970600209D
:1036B000938606AE4146C545170500201305459C77
:1036C00041010283B240224492440145410182807B
:1036D00019C59707002023ABA714014582804545F3
:1036E00082801147636AA70A97D60100938606C5B0
:1036F0000A0536951841411106C63697AE87B28540
:103700000287130700026145639DE700B7E70400E5
:10371000FC4713060002170500201305A5F6829743
:103720000145B2404101828005476145E39BE7FEC8
:10373000B7E70400FC47054617050020130585F68A
:10374000F9BF1307700F6145E39DE7FCB7E704007D
:10375000FC471306700F170500201305E5F4C1B7E9
:10376000130700086145E39EE7FAB7E70400FC474A
:103770001306000817050020130585024DB71547ED
:103780006145E390E7FAB7E70400FC4715461705E3
:1037900000201305250961B709458280411126C221
:1037A000B7E4040083A7C41322C44AC006C62E840B
:1037B000970500209385C5062A898297058905C546
:1037C000970700209387C78B83D7A70BA28503A3F6
:1037D000440D2310F4002244B24092444A85024929
:1037E000014641010283B2402244924402494945C4
:1037F0004101828097070020238C07029707002051
:1038000023AA0702B717004003A7070CB706C0FF9B
:10381000FD16758F23A0E70C03A7070DB706400020
:10382000558F23A8E70C03A7070C3D9B23A0E70CAB
:1038300003A7070D1367070123A8E70C8280B717BA
:10384000004003A5470C83A7470C59811345150079
:10385000C18B058999E3136525009707002083C76D
:1038600027FD6380A702970700202383A7FC11C9C7
:1038700097070020938707FC03A307006303030057
:1038800002838280114517F3FFFF670043C841118F
:1038900093962500AA852D4506C697F0FF1FE78061
:1038A000A0F2B240014541018280011122CC06CE36
:1038B0003714004026CA4AC84EC652C48344740511
:1038C000034AB405834984050349940597F0FFFF33
:1038D000E780C09E8347A40593F4F40F137AFA0F90
:1038E00093E71700230DF40493F9F90F1379F90FF7
:1038F000B717004003C7A705058B6DFF03D5C705A4
:10390000A38D4705238C3705A38C2705A38B97042C
:10391000F2406244D2444249B249224A056182805F
:1039200041119397050122C406C626C2C1872E8481
:1039300063DC0700B7E40400FC54829719C1BC544F
:1039400082972165218D15A893F7150013C51500E1
:103950008DE793F725009DC797000000E78060EE94
:10396000B7E70400BC4F1306000A8945170500207D
:103970000345C5EC829713452400B240224492448B
:10398000410182809397250163D80702B7E40400C0
:1039900083A7C41E829797000000E780E0EEBC4C2E
:1039A00037560700130606308965170500200345C2
:1039B000E5E88297096579B7939715010145E3DE3C
:1039C00007FA17D50100130525A497B00100E78079
:1039D0000005B7E70400BC4F1306006491651705A6
:1039E00000200345A5E582971165A9BF2D71232A03
:1039F0009110FD74E98C232C81102328211123269A
:103A000031112A84AE893289930600100A86A68570
:103A10002D45232E111097F0FF1FE780E0DA1315D4
:103A20004401B7E70400FC4751810A0513962900B9
:103A3000CA850A958297A68585660146254597F031
:103A4000FF1FE78060D80A86A685930600102945E7
:103A500097F0FF1FE78040D78320C1110324811115
:103A600083244111032901118329C110156182802A
:103A7000B7F7070003C70701411106C622C426C2D3
:103A80004AC0A547631DF70097000000E78040F695
:103A9000B24022449244024901454101828013947C
:103AA0002500AA843289A286AA850146254597F079
:103AB000FF1FE78060D1A2864A86A685294597F038
:103AC000FF1FE78060D0E9B71D71A2CC37E4040086
:103AD0005C5C485886CE494697D501009385458E53
:103AE000829711E917D501001305C58E97B0010023
:103AF000E780E0F201A0B7F600E0795798CAFD57D9
:103B0000DCCA0567B7E700E023A0E7101306F00260
:103B100090C223A0E71801000100370700201847D2
:103B20001306000481459706002023A7E6D04157DD
:103B3000A38AE7403C4408088297970700209387B0
:103B4000E76C3EC8856713870740231AE1001D67AD
:103B50003ACC37070105130707103ACE938757D1A0
:103B60001307B00F2310E1022312F102054797F764
:103B7000FFFF9387E7532301E1023ED817070000B8
:103B8000130727D197070000938767D2B7F507007F
:103B9000BAC23EDC170700001307C7ED9707000005
:103BA000938787CE81463000E1051945BAC43EDED1
:103BB00097F0FF1FE78040C1180881479946300001
:103BC0003E960346060085070507A30BC700E3984A
:103BD000D7FEC24791C70357410185676373F7005A
:103BE00001A0B7E7040083A7470A08088297AA85BF
:103BF00011C917C501001305257F97B00100E780A3
:103C000020CA01A0F640664425618280411126C287
:103C1000B7E4040083A7040806C622C41705000001
:103C2000130545D0829717040020130424C12300F4
:103C3000A40097000000E780800297000000E78062
:103C4000A0BB03450400224403A38405B240924470
:103C500013060032896541010283797106D622D4A8
:103C600013078008F337078093F787083EC20100E7
:103C70000100B7170040930570052380B7041306B1
:103C800080FA2380C7040100010083C6F70293F67F
:103C9000A60FA387D702238007049246F3A60680C7
:103CA0000100010073370780137787083AC40100C9
:103CB00001002380B7042380C7040100010003C76B
:103CC000F70213672700A387E70223800704A247B0
:103CD000F3A7078001000100054597E0FFFFE7809B
:103CE000206197000000E78020BA014781468147A4
:103CF000054685451305407E97E0FFFFE780206479
:103D000037E404003C446800514681458297B70778
:103D1000C0A83EC8B787E803938707D03ECA97E795
:103D2000FF1F9387C7693EC67C5868008297B250D0
:103D3000225445618280411197D50100938505D3B6
:103D400017C501001305456306C697B00100E7805B
:103D500020B517D50100130525EA97B00100E780CB
:103D600020B4B2402945410117B30100670023B8D0
:103D7000411197D501009385A5D017C50100130502
:103D8000A55F06C697B00100E78080B117D5010096
:103D9000130545E597B00100E78080B0B2402945A2
:103DA000410117B30100670083B4411122C406C664
:103DB000834705002A849DC797D50100938505D2C6
:103DC00017C501001305455B97B00100E78040ADC2
:103DD0004C4017D50100130565F097B00100E7804E
:103DE00020AC3DA058410DEF97D50100938505CF3C
:103DF00017C501001305455897B00100E78040AA98
:103E000017D50100130505EF97B00100E78040A921
:103E10002244B2402945410117B30100670023AD98
:103E2000A1679386D7036313D70297D501009385C3
:103E3000E5CA17C501001305255497B00100E780B6
:103E400020A617D501001305E5EB7DBFED0797D53B
:103E500001009385A5C817C501001305E551631B33
:103E6000F70097B00100E780A0A317D50100130564
:103E7000A5EA59BF97B00100E78080A24C4017D552
:103E80000100130565EB91BF411197D501009385A2
:103E900065C017C501001305254E06C697B0010081
:103EA000E78000A0B2402945410117B30100670037
:103EB00003A4797122D426D24AD02E842A8981453E
:103EC000B2844800714606D697E0FFFFE780A02243
:103ED00097F7FF1F9387874CDC4783D7070023148E
:103EE00021012313F10097500000E780E0C39547BC
:103EF000A305F1009307401F3EC6FD572305A1000F
:103F0000230AF10097500000E78040D62686A2855C
:103F1000480097500000E78000C4B25022549254E9
:103F2000025945618280971700202394077E9717D6
:103F30000020238D076CB7E70400BC47411106C67B
:103F400041468145170500201305851A8297972061
:103F50000000E780C05F97200000E780C040014577
:103F600097500000E780C068170700200347471AF2
:103F70009307F00A6315F7029307F0F889451705D0
:103F800000201305E518170700202303F7189707EB
:103F90000020A38F071697600000E780E08F9760EE
:103FA0000000E780A09C81453705040097070020AA
:103FB00023AE0712970700202398071297070020C7
:103FC00023850712970700202396070A97070020EA
:103FD00023940708970700202397071097070020CE
:103FE0002390071297300000E780800C014597600E
:103FF0000000E780609397D50100938525AC17C535
:1040000001001305653797B00100E780608917D577
:1040100001001305A5D897B00100E7806088B24081
:104020002945410117B301006700638C411122C487
:1040300006C626C293F715002E84638F07108146AB
:1040400017F6FF1F1306C6328545170500200355D6
:10405000650097C00000E78060F615C997D501009C
:10406000938585A617C501001305053197B001009A
:10407000E780008317C501001305C54797B001000D
:10408000E7800082294597B00100E780408697D5F8
:104090000100938565A317C501001305E52D97A0C1
:1040A0000100E780E07F17C501001305E54597A0F3
:1040B0000100E780E07E294597B00100E78020837A
:1040C00017F5FF1F1305852D5C4505472390E70075
:1040D00097400100E780E0A697D501009385C59E33
:1040E00017C501001305452997A00100E780407B13
:1040F00017C501001305854297A00100E780407AAB
:10410000294597A00100E780807E930710F81707E4
:104110000020230FF7FE9707002083D767F31707C8
:104120000020A307F7FE17050020130565FEA183F5
:10413000914517070020230EF7FC97070020A38A5C
:1041400007FC97500000E780207513451400B2402B
:10415000224492444101828093F72500E1C317076E
:104160000020035767F845CB97060020938606F892
:10417000944297D70100938767C41706002003462F
:10418000C6F6814517050020130585F697700000D7
:10419000E7802002AA8441C197D5010093858599C3
:1041A00017C501001305451D97A00100E780406F6A
:1041B000A68517C501001305E53797A00100E78024
:1041C000206E294597A00100E780607297070020C4
:1041D000239C07F0930710F817070020230AF7F233
:1041E0009707002083D7C7E617070020A302F7F23E
:1041F000A18317070020230EF7F091458D4717057F
:1042000000201305E5F017070020A304F7F09750EE
:104210000000E78060681345240015BF93F7450050
:10422000D1C397D501009385E59017C5010013050B
:10423000A51497A00100E780A06617C5010013052B
:10424000253197A00100E780A065294597A00100CE
:10425000E780E069930720F817070020230AF7EAB0
:104260009707002083D707E117070020A302F7EA8A
:10427000A18317070020230EF7E8854717070020C2
:10428000A309F7E897500000E780409E170500203B
:10429000130505E8914597500000E780E05F13455E
:1042A000440075B593F78500A9C797D5010093859C
:1042B000658817C501001305250C97A00100E7804C
:1042C000205E17C501001305E52997A00100E780CE
:1042D000205D294597A00100E780606197070020D5
:1042E000239407E097700000E78080FC134584006A
:1042F000B9BD93F70501D1C38545170500200355C6
:1043000065D797600100E780A0AE97D5010093853F
:10431000658217C501001305250697A00100E780F7
:10432000205817C501001305252597A00100E78037
:104330002057294597A00100E780605B930730F87C
:10434000170700202306F7DC9707002083D787D2C2
:1043500017070020A30EF7DA17050020130545DB29
:10436000A1838D45170700202305F7DA9750000039
:10437000E780805213450401D9BB93F70502D1C7EA
:1043800097C501009385057B17C501001305C5FE80
:1043900097A00100E780C05017C501001305052054
:1043A00097A00100E780C04F294597A00100E78052
:1043B0000054930740F817070020230BF7D4970702
:1043C000002083D767C917070020A303F7D4A18370
:1043D00017070020230FF7D2854717070020A30AED
:1043E000F7D297070020239907C697500000E7806F
:1043F000E087170500201305A5D1914597500000CF
:10440000E78080491345040299B393F70504FDC37F
:1044100097C501009385057217C501001305C5F501
:1044200097A00100E780C04717C501001305851854
:1044300097A00100E780C046294597A00100E780CA
:10444000004B9707002083C7A7CC1307700A638629
:10445000E7061307800A638CE7081307600A639373
:10446000E704930760F8170700202303F7CA9707AC
:10447000002083D747C717070020A30BF7C8A183E5
:10448000170700202307F7C8854717070020A30652
:10449000F7C8B14517050020130585C797500000E0
:1044A000E780803F97400000E780407C134504048C
:1044B00097070020239907C259B9930770F8170787
:1044C00000202307F7C49707002083D7C7C1170729
:1044D0000020A30FF7C2A18317070020230BF7C208
:1044E000854717070020A307F7C2994565B79307CB
:1044F00080F8F1B793F705080145E38A07C497C52B
:1045000001009385256317C501001305E5E697A013
:104510000100E780E03817C501001305250B97A0BF
:104520000100E780E037294597A00100E780203CA3
:104530009307A0F817070020230CF7BC970700206B
:1045400083D707BC17070020A304F7BCA183170774
:1045500000202300F7BC854717070020A30BF7BAFC
:1045600097070020239E07B897400000E78000705F
:10457000170500201305C5B9914597500000E78045
:10458000A03113450408E1B6411122C497C50100CA
:10459000938505562A8417C501001305E5DD06C677
:1045A00097A00100E780C02F4C4017C501001305FC
:1045B000657097A00100E780A02E294597A0010013
:1045C000E780E032034704009307F00F631FF70210
:1045D00097C501009385C55117C501001305C5D9BD
:1045E00097A00100E780C02B4C4017C501001305C0
:1045F000656D97A00100E780A02A2244B2402945BA
:10460000410117A301006700832EB24022444101FB
:104610008280B1C1411122C417C501001305C5D55F
:104620002E8497C501009385A54706C697A0010073
:10463000E7800027A28517C501001305E57397A041
:104640000100E780E0252244B2402945410117A33B
:1046500001006700C3298280411122C426C22E8432
:10466000AA8497C501009385654417C50100130509
:10467000A5D006C697A00100E780802217C50100DB
:104680001305457097A00100E7808021294597A078
:104690000100E780C02597C5010093852541970754
:1046A00000202399979A17C501001305E5CC85448E
:1046B00097070020239E879897070020239B9798B1
:1046C000971700202397870497A00100E780401DDB
:1046D0009715002083D5E50317C501001305056B69
:1046E00097A00100E780C01B294597A00100E78043
:1046F000002097170020238B97F097200000E78079
:1047000080C6228597500000E78080EE05459750CF
:104710000000E780602197F7FF1F938727C8DC47D9
:1047200003D70700C167FD176312F7022244B7E7FA
:104730000400B240924403A3870517F5FF1F034509
:1047400065101306000A854541010283B2402244E8
:10475000924441018280011122CC37E404005C5C68
:1047600006CE354697C501009385454A17D5010009
:1047700013054510829711E917C50100130585C57A
:1047800097A00100E780A02901A097F7FF1F93875A
:10479000270C3EC4B7F507008567938707808146DD
:1047A00017F6FF1F1306460AE10519453EC697E0B6
:1047B000FF1FE78060017C44194697F5FF1F938532
:1047C000A508170500201305258B8297340017F6DE
:1047D000FF1F1306660797D501009385659417D5CB
:1047E00001001305659597600000E78080712A84B9
:1047F0001DCD97C501009385E53217C5010013054E
:10480000A5B797A00100E780A009A28517C5010000
:104810001305C54097A00100E7808008294597A0AF
:104820000100E780C00CF24062440561828097E09D
:104830000000E780E0D317C5010013052535975028
:104840000000E780C06597A00000E78020289760FF
:104850000100E780A08C17F5FF1F1305A5B0975046
:104860000100E780407517C50100130525339760E7
:104870000100E780208D2A8497600000E78000CC4B
:1048800097000100E780806497800100E780A0FD29
:1048900097700000E780402497600000E7800042A6
:1048A00097300100E780E02597C5010093858527B3
:1048B00017C50100130545AC19C897A00100E78092
:1048C00020FEA28517C5010013058537A1B797A063
:1048D0000100E780E0FC17C501001305A53897A08B
:1048E0000100E780E0FB294597A00100E780200058
:1048F00097300100E780C00197F00000E78080203A
:1049000055C985453705040097200000E780407AA7
:1049100097C501009385052117C501001305C5A59D
:1049200097A00100E780C0F717C501001305053502
:1049300097A00100E780C0F6294597A00100E78015
:1049400000FB97F7FF1F9387279583D7070017175B
:1049500000202310F7DC8547171700202308F7CA2B
:1049600097200000E78020B997200000E780A09FF3
:10497000171500200355E5D997500000E78040C780
:10498000054597500000E78020FA97C50100938500
:10499000651917C501001305259E97A00100E78042
:1049A00020F017C501001305A52F97A00100E7808F
:1049B00020EFADB597C501009385C51617C5010059
:1049C0001305859B97A00100E78080ED17C50100C6
:1049D0001305C53C97A00100E78080EC294597A00E
:1049E0000100E780C0F0014569BF411122C437E4EE
:1049F00004008327041A06C6829797500000E780B8
:104A0000E0C28327040817F5FFFF1305656282974C
:104A100097F7FF1F2388A7E217F5FF1F13050598D7
:104A200097400000E78020572244B240410117031D
:104A30000000670083D2B7E70400FC471171A2DDD4
:104A4000CAD986DFA6DBCED72E8432892E86AA85E8
:104A500017F5FF1F1305C56B829717F7FF1F130785
:104A6000276B83470700930680029387E70793F736
:104A7000F70FE3ECF610BA898A0717C7010013078E
:104A8000E798BA979C43BA9782878D4797C50100EC
:104A90009385850B17C501001305058E630FF40080
:104AA00097A00100E780C0DF17C50100130585C886
:104AB00097A00100E780C0DEBDA497A00100E780B9
:104AC00020DE17C50100130565C897A00100E78027
:104AD00020DD294597A00100E78060E1930720F8D9
:104AE000114697F5FF1F9385A5624A8517F7FF1FAB
:104AF0002300F76297F7FF1FA38D076097F0FFFF72
:104B0000E780603B2A841DC997C501009385C503D2
:104B100017C501001305458697A00100E78040D81E
:104B2000A28517C50100130525C697A00100E780DF
:104B300020D7294597A00100E78060DB97C50100D9
:104B40009385850017C501001305058397A0010013
:104B5000E78000D517C50100130545C497A00100E3
:104B6000E78000D4294597A00100E78040D841653F
:104B7000930730FA054697F5FF1F938565597D1514
:104B800017F7FF1F2306F75897F0FFFFE780A032C3
:104B90002A841DC997C50100938505FB17B501003F
:104BA0001305857D97A00100E78080CFA28517C5FA
:104BB0000100130565BD97A00100E78060CE29457F
:104BC00097A00100E780A0D2B7E70400BC4F0566BC
:104BD000130606C8A14517F5FF1F0345A5C6829712
:104BE000FE506E54DE544E59BE5911618280914779
:104BF0006303F40297C50100938505F517B501001D
:104C00001305857797A00100E78080C917C50100CB
:104C1000130505BC71BDB7E70400FC4F914517F5BE
:104C2000FF1F034525C2829797C501009385C5F1F3
:104C300017B501001305457497A00100E78040C631
:104C400017C50100130585BA97A00100E78040C58C
:104C5000294597A00100E78080C997400000E780C0
:104C6000E000914535A485476303F40297C5010030
:104C7000938585ED17B501001305057097A0010018
:104C8000E78000C217C501001305C5B715B597F732
:104C9000FF1F2391273FB7E704000566BC4F1306AB
:104CA00006C8C1450DBF8D476303F40297C50100D7
:104CB000938585E917B501001305056C97A00100E0
:104CC000E78000BE17C50100130585B5D5B393076E
:104CD00040F8114697F5FF1F938585434A8517F7DE
:104CE000FF1F2307F74297F7FF1FA384074297F0A0
:104CF000FFFFE780401C2A84E30405EE97C501000E
:104D0000938585E417B501001305056797A0010099
:104D1000E78000B9A28517C501001305E5A697A095
:104D20000100E780E0B7294597A00100E78020BC9B
:104D300045BD9147E31CF4F6B7E70400FC4F93052B
:104D4000000217F5FF1F0345E5AF829797C50100E5
:104D5000938585DF17B501001305056297A0010053
:104D6000E78000B417C50100130505ADF1BD894703
:104D700063E3870297C50100938505DD17B5010040
:104D80001305855F97A00100E78080B117C501007A
:104D90001305C5AB31BB97F4FF1F83C4843797F766
:104DA000FF1F83C7F73697C501009385E5D9A20495
:104DB00017B501001305455CDD8C97A00100E78065
:104DC00020AEA28517C50100130585A997A0010093
:104DD000E78000ADC204294597A00100E78020B11B
:104DE000C1849305D4FF93960401C1824A8693F54A
:104DF000F50F17F5FF1F1305D53197200000E78049
:104E0000E02EE35F90DC930750F817F7FF1F2301B4
:104E1000F73083C73900228697F5FF1F9385452F0A
:104E200085074A8517F7FF1FA305F72E97F0FFFFA9
:104E3000E78060082A84E30505DA97C501009385B9
:104E4000A5D017B501001305255397A00100E780F1
:104E500020A5A28517C50100130505F1C9B589472D
:104E600063E3870297C50100938505CE17B501005E
:104E70001305855097A00100E78080A217C50100A7
:104E80001305C59F35B197400000E78020DEA2855D
:104E900017F5FF1F1305C52797500000E780C09F37
:104EA00081B38D476303F40297C501009385C5C99B
:104EB00017B501001305454C97A00100E780409EFF
:104EC00017C501001305459DE5B6B766020001460A
:104ED000B7750200054597E0FF1FE780E08E930756
:104EE00060F817F7FF1F2305F72297F7FF1FA3822C
:104EF00007229307000617F7FF1F230DF7208947A6
:104F000017F7FF1FA308F72097F7FF1F2385072038
:104F100097F7FF1FA3810720C14717F7FF1F230D36
:104F2000F71E930720F917F7FF1FA307F71E314657
:104F300097F7FF1FA383A71E97F5FF1F9385451DB6
:104F40004A8597F7FF1F238A071C97F0FFFFE7802A
:104F500080F62A84E30605C897C501009385C5BE7F
:104F600017B501001305454197A00100E780409364
:104F7000A28517C501001305A59355B3B147630377
:104F8000F40297C50100938525BC17B501001305F0
:104F9000A53E97A00100E780A09017C5010013056A
:104FA000E59239B6B7E70400FC4F9305000417F506
:104FB000FF1F03452589829797400000E78000CBBB
:104FC000B145F9B5914763E3870297C50100938521
:104FD000A5B717B501001305253A97A00100E78092
:104FE000208C17C5010013052590D9B497F4FF1F35
:104FF00083C4441297F7FF1F83C7B711A204DD8C47
:105000008E04B77702006D14BE942286A68517C55C
:1050100001001305A58E97A00100E7806088B7E71F
:105020000400FC47228697F5FF1F9385B50E2800E4
:10503000829793160401C1823000A685094597D056
:10504000FF1FE78060782A8409C917C5010013058E
:10505000A58C97A00100E780809C930770F8194603
:1050600097F5FF1F9385C50A4A8517F7FF1F230190
:10507000F70A97F7FF1FA38F870897F0FFFFE780D6
:1050800080E32A84E30E05B497C501009385C5AB80
:1050900017B501001305452E97A00100E780408059
:1050A000A28517C501001305258895B99947630B9B
:1050B000F41297C50100938525A917B501001305C2
:1050C000A52B97900100E780A07D17C5010013056F
:1050D0002587F9BA914763E3870297C50100938555
:1050E000A5A617B501001305252997900100E780B3
:1050F000207B17C50100130525865DBA97F4FF1FB5
:1051000083C4440197F7FF1F83C7B700A204DD8C57
:105110008E04B77702006D14BE942286A68517C54B
:1051200001001305A58497900100E7806077B7E739
:105130000400FC47228697F5FF1F9385B5FD2800E4
:10514000829793160401C1823000A6850D4597D041
:10515000FF1FE78060672A8409C917C5010013058E
:10516000A58297A00100E780808B930780F81946FD
:1051700097F5FF1F9385C5F94A8517F7FF1F230988
:10518000F7F897F7FF1FA38787F897F0FFFFE780EF
:1051900080D22A84E30605A497C501009385C59AA9
:1051A00017B501001305451D97900100E780406F7A
:1051B000A28517B501001305657E95B6994763036F
:1051C000F40297C501009385259817B501001305D2
:1051D000A51A97900100E780A06C17B50100130590
:1051E000657DF9B0B7E70400FC4F9305000417E5AF
:1051F000FF1F03452565829797400000E78000A7C1
:10520000994579B18D476303F40297C501009385F1
:10521000A59317B501001305251697900100E780A7
:10522000206817B501001305657A59B017B501005C
:105230001305C57A97900100E780607E1305C012C0
:1052400097D0FF1FE780E00F014597E0FFFFE78061
:1052500020E30D4597100000E780009F294597D077
:10526000FF1FE780000E97D0FF1FE78060FE8DBA1A
:1052700099476303F40297C501009385E58C17B540
:1052800001001305650F97900100E780606117B575
:1052900001001305657529B817F7FF1F034797E746
:1052A00097F7FF1F83C707E722075D8F9166BA96BE
:1052B000C2061166C1821306F6EF8D476365D602FA
:1052C00097E7FF1F9387870D9C4B17F6FF1F034639
:1052D00056E49386C7002DC203D6070069CA890722
:1052E000E39CD7FE89471307A0F8114697F5FF1FE7
:1052F000938505E24A8597F6FF1F238BE6E017F7B3
:10530000FF1FA308F7E097F0FFFFE780C0BA2A84E9
:10531000E308058C97C501009385058317B5010047
:105320001305850597900100E7808057A28517B582
:1053300001001305A56CE5B203D60700630EE60A6B
:105340008907E39BF6FE8D4779BF91476304F4021A
:1053500097B501009385457F17B501001305C50179
:1053600097900100E780C05317B501001305856AC7
:105370006FF00FF4B7E70400FC4F9305000817E542
:10538000FF1F0345254C8297C9B897B50100938547
:10539000A57B17B50100130525FE97900100E78056
:1053A000205017B50100130565686FF06FF023906A
:1053B000E70017E5FF1F130565FE97200100E78052
:1053C000A07A97B501009385257817B501001305DC
:1053D000A5FA97900100E780A04C17B501001305CE
:1053E000E56597900100E780A04B29459790010063
:1053F000E780E04F8147C5BD2390070017E5FF1FF9
:105400001305C5F997200100E780007697B50100E4
:105410009385857317B50100130505F69790010074
:10542000E780004817B501001305C5625DBF411153
:1054300022C406C6834705002A849DC797B501008C
:105440009385456C17B50100130505F3979001008E
:10545000E78000454C4017C501001305259797903C
:105460000100E780E043E1A05841B707CF009387F0
:10547000777D631DF70697B501009385A56817B57D
:105480000100130565EF97900100E78060411C441F
:105490008356E4008355C40003C6070017C5010006
:1054A0001305459497900100E780803F2945979028
:1054B0000100E780C0430357E4009707002083D72B
:1054C00047256309F7008355C400084497E0FFFFB0
:1054D000E78080CF0356E4008355C400084422448B
:1054E000B240410117F3FFFF67002355B707CC0017
:1054F0009387777D6315F70497B5010093858560E1
:1055000017B50100130545E797900100E780403982
:105510001C448356E4008355C40003C6070017C526
:1055200001001305258C97900100E7806037224425
:10553000B24029454101179301006700433BB7077B
:10554000CE009387777D6304F70297B501009385BA
:10555000655B17B50100130525E297900100E78010
:1055600020344C4017B501001305057DCDBDB24078
:10557000224441018280B7E70400FC4741112E8696
:1055800006C622C426C24AC02E842A89AA8517F5D7
:10559000FF1F1305E5B7829797B501009385855CDA
:1055A00017B50100130545DD97900100E780402FF6
:1055B00097F5FF1F83C5C5B517B501001305850213
:1055C00097900100E780C02D294597900100E78062
:1055D000003297F4FF1F9384A4B383C704004147AC
:1055E0009387070693F7F70F636AF75C17B7010015
:1055F000130707EC8A07BA979C43BA9782879D479F
:105600006307F40297B501009385C55517B50100EE
:10561000130585D697900100E780802817B5010013
:105620001305C5FC97900100E7808027ADAC97F784
:10563000FF1F83C7F7ADDDCB17F7FF1F034777AD1C
:1056400097F7FF1F83C7E7AC22075D8F97F7FF1F10
:1056500083C747ACC2075D8F97F7FF1F83C797AB20
:10566000E207D98F17F7FF1F2322F7A883C764002B
:1056700097B501009385054F17B501001305C5CFF8
:1056800017F7FF1F2303F7A697900100E78040213B
:1056900097F7FF1F938787A58C4317F6FF1F0346D5
:1056A000C6A417B50100130525F697900100E78001
:1056B000201F294597900100E780602397F7FF1F7F
:1056C000A38807A42244B24092440249930700F8F9
:1056D00017F7FF1F230EF7A29D4517F5FF1F1305B0
:1056E00025A34101174300006700031B97600000DA
:1056F000E78080CB97F7FF1F238DA7A093578500E6
:1057000017F7FF1FA307F7A0935705012A8417F780
:10571000FF1F2301F7A093578501014517F7FF1FCE
:10572000A30AF79E97600000E780C0C897F7FF1FA5
:105730002383A79E97B501009385C54217B5010045
:10574000130585C397900100E780801517F6FF1FAA
:105750000346669CA28517B50100130565ECB1B739
:10576000CD476303F40297B501009385A53F17B5B4
:105770000100130565C097900100E780601217B51E
:105780000100130565EB79BD37E404007C44414614
:1057900097F5FF1F9385D59717F5FF1F13054595BF
:1057A000829717F5FF1F1305A59497100000E78057
:1057B000A0CD97100000E78000BB97F7FF1F83C7BD
:1057C000479617F7FF1F0347B795A20703238405E2
:1057D000D98F17F7FF1F2319F7901306000A894581
:1057E0002244B2409244024917E5FF1F0345850554
:1057F000410102838D476303F40297B5010093854D
:10580000653617B50100130525B797900100E780AD
:10581000200917B501001305E5F129B517F4FF1F9D
:105820000344248F97F7FF1F83C7978E97B5010016
:1058300093854533220417B501001305E5B35D8C4C
:1058400097900100E780C005A28517B501001305F8
:1058500025E097900100E780A0042945979001007A
:10586000E780E0080D4697F5FF1F9385658A22853E
:1058700097E0FFFFE7802064AA8421C197B501006B
:105880009385452E17B50100130505AF97900100CC
:10589000E7800001A68517B501001305A5DC9790E8
:1058A0000100E780E0FF2244B240924402492945CA
:1058B0004101179301006700830397E7FF1F239BB4
:1058C000877AB7E70400116603A38705130606E885
:1058D000914539B78D476303F40297B5010093856D
:1058E000652817B50100130525A997900100E780E9
:1058F00020FB17B501001305A5F22DB317F4FF1F08
:105900000344248197F7FF1F83C7978097B5010051
:1059100093854525220417B501001305E5A55D8C87
:1059200097900100E780C0F7A28517B50100130525
:10593000A5D497900100E780A0F629459790010033
:10594000E780E0FA0D4697E5FF1F9385657C228589
:1059500097E0FFFFE7802056AA841DC197B501009C
:105960009385452017B50100130505A19790010007
:10597000E78000F3A68517B50100130525D105B70B
:1059800097E7FF1F239A876CB7E70400116603A30C
:105990008705130606E89305000299B5894763E376
:1059A000870297B501009385E51B17B50100130524
:1059B000A59C97900100E780A0EE17B501001305A4
:1059C000E5E88DB197E4FF1F83C4A47497E7FF1F38
:1059D00083C7177497B501009385C518A20417B53E
:1059E000010013056599DD8C97900100E78040EB7D
:1059F000A68517B501001305E5CA97900100E78059
:105A000020EA294597900100E78060EE228697E51D
:105A1000FF1F9385E56F268597E0FFFFE780A0498C
:105A20002A84630E051A97B501009385A51317B54F
:105A300001001305659497900100E78060E6A28558
:105A400017B50100130545C799BD854763F9871848
:105A5000834519002244B24092440249B335B00054
:105A600097E7FF1F2382B76217B50100130505C62C
:105A70004101179301006700A3E2A2852244B240CE
:105A800092444A850249410117030000670003223E
:105A900099476303F40297B501009385A50C17B5E8
:105AA00001001305658D97900100E78060DF17B551
:105AB0000100130565F3BDB617E4FF1F03446465D9
:105AC00097E7FF1F83C7D76497B5010093858509C2
:105AD000220417B501001305258A5D8C97900100FB
:105AE000E78000DCA28517B501001305A5BF9790DC
:105AF0000100E780E0DA294597900100E78020DF88
:105B0000194697E5FF1F9385A560228597E0FFFF63
:105B1000E780603AAA841DC197B50100938585048A
:105B200017B501001305458597900100E78040D720
:105B3000A68517B501001305E5BB95B397E7FF1FD1
:105B40002390875CB7E70400116603A3870513065B
:105B500006E89305000869B1854797B5010093856C
:105B6000650017B5010013052581630BF4009790BC
:105B70000100E780E0D217B501001305E5B85DB478
:105B800097900100E780C0D117B50100130545B912
:105B900097900100E780C0D0294597900100E780E9
:105BA00000D52244B2409244024997E7FF1F239D4B
:105BB00007524101175300006700836F97B501003A
:105BC000938545FA17A501001305057B9790010001
:105BD000E78000CD17B50100130545E5A1B4B2403B
:105BE00022449244024941018280411106C622C4E6
:105BF00097E0FFFFE780202C9377F50FA1C32A845D
:105C000097B50100938585F717A501001305C576A3
:105C100097900100E780C0C89375F40F17B5010095
:105C20001305851497900100E78080C72244B24095
:105C30002945410117930100670063CBB24022441C
:105C400041018280411122C491462A8417E6FF1F38
:105C50001306465A9D652D4506C697D0FF1FE7805F
:105C6000A0B6B7F7070003C70701A5476313F700FE
:105C700001A09306001001469D65254597D0FF1FA2
:105C8000E78080B497E7FF1F238687562244B240FF
:105C9000914617E6FF1F1306E6559D65294541010C
:105CA00017D3FF1F670043B21171CED7B7E90400C5
:105CB00083A7C904CAD917E9FF1F13096945A2DDE3
:105CC0002E8686DFA6DB2E84AA854A85829797E7F3
:105CD000FF1F83C7E7431307700A6385E710636DEF
:105CE000F7001307600A6385E704FE506E54DE5424
:105CF0004E59BE59116182801307800A6385E716E9
:105D00001307900AE393E7FE8D476306F41C97B5EB
:105D100001009385A51817A501001305E565979067
:105D20000100E780E0B717B501001305651425A051
:105D30008D47630CF40297B501009385251617A5CE
:105D400001001305656397900100E78060B517B502
:105D500001001305250B97900100E78060B42945E9
:105D600097900100E780A0B849B7854717B50100B3
:105D70001305050B17E7FF1F2308F7309790010065
:105D8000E780E0C9B7750200B76602000146054525
:105D900097D0FF1FE78040A3930760F817E7FF1F26
:105DA0002308F73697E7FF1FA385073693070026DA
:105DB00017E7FF1F2320F736E5779387072117E7BB
:105DC000FF1F231BF734B14597E7FF1F23870734D5
:105DD00097E7FF1FA383A7344A8597000000E78059
:105DE000E01621B7914763E3870297B501009385D9
:105DF000E50A17A501001305255897900100E780D3
:105E000020AA17B501001305A503B1B797E4FF1F3A
:105E100083C4443097E7FF1F83C7B72FA204DD8CEC
:105E200083A7C9046D14228697E5FF1F9385952EDD
:105E3000280082978E0493160401B7750200C18270
:105E40003000A695094597D0FF1FE780E09793079C
:105E500070F817E7FF1F230DF72A994597E7FF1FF3
:105E6000A38AA72A95BF914763E3870297B50100EC
:105E70009385C50217A501001305055097900100F1
:105E8000E78000A217B50100130505FDE9B597E409
:105E9000FF1F83C4242897E7FF1F83C79727A20407
:105EA000DD8C83A7C9046D14228697E5FF1F9385B7
:105EB0007526280082978E0493160401B775020098
:105EC000C1823000A6950D4597D0FF1FE780C08F97
:105ED000930780F8BDBF17B501001305A5FA979089
:105EE0000100E780C0B3930790F82304F1008347D3
:105EF00019008D452800A304F100834729002305DC
:105F0000F10097000000E78060041305C01297C0FD
:105F1000FF1FE7800043014597D0FFFFE780401651
:105F20000D4597000000E78020D2294597C0FF1F4C
:105F3000E780204197C0FF1FE78080317DB397E75E
:105F4000FF1F23A1A72C828097E7FF1F9387872B32
:105F500003A30700630303000283174300006700E5
:105F6000A39341114AC097F6FF1F83D6867A3289E0
:105F700017D6FF1F0356A64422C426C206C62A848B
:105F8000AE8497000000E780606435C12DC099475A
:105F900063FF97048347140003470400A207D98FC7
:105FA00013978700A183D98FC2073167C183130775
:105FB000C755639EE70297D7FF1F83D74740A301CA
:105FC000F400A1832302F40097F7FF1F83D76774BF
:105FD00091C7A302F400A1832303F400A68517B59B
:105FE00001001305A5EF97900100E780608B97F7FC
:105FF000FF1F83C7A761B9CF97D5FF1F83D5253C66
:1060000017B50100130545EF97900100E78040891F
:106010002686A28517D5FF1F0355653A9700000015
:10602000E780E0BC6301090497E7FF1F83C7C71D32
:106030009DCB95C897E7FF1F83C707058DE722858E
:106040002244B2400249A685924441011743000010
:106050006700838417B50100130505EB97900100D5
:10606000E780E09BC1B7B24022449244024941011B
:106070008280834755008345450017B5010013050D
:10608000A5E4A207DD8D179301006700638117B5B2
:106090000100130565E217930100670043988D47DF
:1060A00063FBB70A011126CA06CE22CC0344350091
:1060B00097E4FF1F83C4541597B50100938585E5C8
:1060C000B337800017E7FF1FA300F71409C497B583
:1060D00001009385E5E417B501001305E5E4978019
:1060E0000100E780E07B97E7FF1F83C7F711638616
:1060F000970097000000E780202B97E7FF1F83C7DA
:10610000B7108DC785472306F100B7E7040083A7C2
:1061100047177000854513055030829717B5010069
:10612000130585E197900100E780608F9967938759
:1061300057EE2316F100680085479145A3078100BB
:106140002307F10097000000E78040E0F24062443E
:10615000D244056182808280894763F7B7080111C4
:1061600022CC06CE26CA8344250085472A84639D17
:10617000F404914763F5B7040345450083473400B1
:1061800022055D8D97D7FF1F239BA7229700000054
:10619000E780A04C9967938767EE2314F10083474B
:1061A000340023059100A305F10083474400954581
:1061B00028002306F10097000000E78020D9F24074
:1061C0006244D24405618280FDF89967938767EE47
:1061D0002314F10097D7FF1F83D7671EA305F10093
:1061E00023050100A183E1B782800111996722CCC8
:1061F000D51717F4FF1F130464412314F1008347DC
:10620000040026CA97F4FF1F9384A4502305F100CD
:1062100083D7040028009545A305F100A18306CE8D
:106220002306F10097000000E78040D203D6040067
:106230008345040017B50100130585D1978001003F
:10624000E7800066F2406244D244056182809D6727
:106250007971D9172316F10097F7FF1F83C7073B02
:1062600006D62307F100A9C3B7E70400FC4741465F
:1062700097E5FF1F9385C5E71305F1008297680036
:10628000CD4597000000E78060CC97F5FF1F83C5E0
:10629000E53717B501001305A5CE97800100E7800B
:1062A0002060B25045618280B7E70400BC47414698
:1062B00081451305F1008297D9B75DC1411106C62A
:1062C00022C4930750FA2300F5009307A005A3000A
:1062D000F50089472301F5009147A301F500ED473B
:1062E000A302F50097F7FF1F9387473283C7070084
:1062F000230205002A842303F50097E7FF1F9387F5
:10630000B7F083C70700414697E5FF1F938545DE39
:10631000A303F50097F7FF1F83D7A73F2304F500DA
:10632000A183A304F50097D7FF1F83D7470923054F
:10633000F500A183A305F500B7E70400FC4731058C
:1063400082972285F14597000000E7802024230EE4
:10635000A4002181A30EA400B24022444101828006
:1063600082805D710A8586C6A2C497000000E7801E
:1063700000F537E404007C448A850810794682974A
:106380003C441305E10309468145829710109305AB
:106390000002014597D0FFFFE780E034B640264475
:1063A00061618280B7C7A55A01119387C7333EC484
:1063B00097E7FF1F83C757E53EC6B7F7070003C738
:1063C000070106CE22CCA5476313F70001A0116494
:1063D000930504F0930600100146254597C0FF1F62
:1063E000E780803E3000930504F0A146294597C020
:1063F000FF1FE780603D97E5FF1F83C5F5E017B5F8
:1064000001001305A5C897800100E7806049F240AC
:1064100062440561828001119165A1463000938537
:1064200005F02D4506CE97C0FF1FE780E0392247D3
:10643000B7C7A55A9387C7336314F702B24517B598
:1064400001001305E5B7B335B00097E7FF1FA38D33
:10645000B7DA97800100E780A044F24005618280AE
:10646000814517B501001305E5B797E7FF1FA38D19
:1064700007D897800100E780A04297000000E780DE
:10648000A0F2E1BFB7C7A55A79719387F7353EC629
:10649000B7E70400FC47AA8506D622D4414608087F
:1064A0008297B7F7070003C70701A5476313F700F3
:1064B00001A01164930504E89306001001462545E8
:1064C00097C0FF1FE78040307000930504E8D14675
:1064D000294597C0FF1FE780202F17B5010013053E
:1064E000A5BE97800100E7808053B25022544561D9
:1064F000828079719165D1467000938505E82D45BC
:1065000006D697C0FF1FE780202C3247B7C7A55A91
:106510009387F73517B501001305C5B46310F7026B
:10652000B7E70400FC4717E5FF1F130565BC4146AC
:106530000C08829717B501001305C5B097800100BC
:10654000E780E04DB25045618280B7F7070003C78E
:106550000701A5476313F70001A091654111930658
:1065600000100146938505E8254506C697C0FF1F24
:10657000E7808025B24017B501001305A5A24101AF
:10658000178301006700A349C16769768146FD173B
:1065900005061397060141836364B7003E85828038
:1065A0003307D50003470700B98F214713F81700B9
:1065B000858363050800B18FC207C1837D171377F8
:1065C000F70F6DF78506F1B741C5A547054763F29B
:1065D000B70883471500034705003168A207D98F24
:1065E00013978700A183D98FC207C1831308C855A9
:1065F000054763900707411106C622C426C203441B
:106600002500914763F087049307540063ECF5027B
:10661000A301C50021822302C5009304340091C662
:10662000A302D500A1822303D5002A84A685970062
:106630000000E780A0F526942300A4002181A30098
:10664000A4000147B240224492443A85410182802D
:1066500005473A858280B7C7A55A01119387E73469
:106660003EC42AC6B7F7070003C7070106CE22CCEF
:1066700026CAA5476313F70001A091642A84938575
:1066800004EE930600100146254597C0FF1FE780E2
:10669000A0133000A146938504EE294597C0FF1F43
:1066A000E7808012A28517B50100130525A0978009
:1066B0000100E780E01E97000000E780C0CAF240BA
:1066C0006244D2440561828001119165A146300087
:1066D000938505EE2D4506CE97C0FF1FE780C00EBF
:1066E0002247B7C7A55A9387E7346318F702B24524
:1066F00017B501001305059197D7FF1F2391B7CC5C
:10670000C205C18197800100E780801997000000D1
:10671000E78060C5F24005618280D147D14517B559
:1067200001001305259017D7FF1F231AF7C897807C
:106730000100E780E01617D5FF1F035545C89700F5
:106740000000E78080F1F9B721C1411126C206C6D9
:1067500022C4AE848DC52A8497000000E780A05D26
:1067600097E7FF1F83C747AA99CB22852244B240EF
:10677000A68592444101173300006700E311B2403F
:106780002244924441018280828001114AC806CE8F
:1067900022CC26CA4EC693F715002E899DCBAD6735
:1067A000371700409387A7AA1CC3B7E70400BC4F64
:1067B00013060019854517D5FF1F034525C082978D
:1067C00013451900F2406244D2444249B24905617E
:1067D000828093F725006382071C17F7FF1F03577A
:1067E00027F3954763F9E70C014417F6FF1F1306DB
:1067F00026E293063005130550041308100493088D
:10680000B00413039005930764006374F7043A849B
:10681000FD5997F4FF1F83C4A4DF97F7FF1F83C7B9
:1068200037DFA204DD8CAD679387B7556383F4141B
:1068300063E3970AA9679387A7556386F414A28533
:1068400017F5FF1F1305C5DC97000000E78000F077
:10685000F5A8B307860083C50700639AD50483C5EE
:1068600017006396A50483C527006392050583C5B9
:106870003700639ED50283C54700639A150383C71B
:10688000570063966702A2890DE897F5FF1F83D52D
:1068900025E8B3853541C20517F5FF1F130545D718
:1068A000C1814E9597000000E78040EA65A8050485
:1068B0004204418089BF3A84FD598547E3EB87F460
:1068C00059CC854517F5FF1F130585D497000000A7
:1068D000E780C0E769A0B1679387C7556380F40478
:1068E000B5679387D755E39CF4F4A28517F5FF1F8E
:1068F000130505D297300000E78000FA8947630747
:10690000F4049305E4FFC205C18117F5FF1F1305C9
:1069100045D097000000E78000420DA897000000D6
:10692000E780C04011C9A28517F5FF1F130545CEAA
:1069300097000000E78020400546A28517F5FF1F5D
:10694000130505CD97F0FFFFE780E061A68517A549
:1069500001001305657997800100E78060F4FD5719
:10696000E395F9F297F7FF1F239407DA13452900FF
:1069700091BDA28517F5FF1F130585C997F0FFFF8D
:10698000E780606FE1B7A28517F5FF1F130545C8C3
:1069900097F0FFFFE780E06F55BF93F74500014593
:1069A000E38207E217A501001305457597800100F2
:1069B000E780E00697300000E78000FD13454900BE
:1069C00011B5411122C437E404005C5C06C63546AB
:1069D00097A501009385852317B50100130585E967
:1069E000829711E917A50100130505729780010030
:1069F000E780E00201A08327041C82972A840545D2
:106A000097C00000E78020B697600100E780403B18
:106A100097600100E780401097B00000E780A0C7B2
:106A20002285B2402244410182801567B717004099
:106A30001307575598C3D8439D66558FD8C3D8437D
:106A4000FD76758FD8C3D8431367F70FD8C3356762
:106A50001307C7CC98C382804111054506C622C4DE
:106A600026C297C0FFFFE780804B1305A00497B0B4
:106A7000FF1FE780C063757585457D1597C0FFFFD3
:106A8000E78020357D7585451305F53697C0FFFFF6
:106A9000E780803E371400408327840A8D45130524
:106AA000002093E707202324F40A97C0FFFFE78024
:106AB0004032B7E4040097C0FFFFE7806077C85812
:106AC00097800100E780A0F517B50100130585DA6E
:106AD00097800100E780A0F48327840C8545414519
:106AE00093E707082324F40C97C0FFFFE780C03822
:106AF0008D451305000897C0FFFFE780E03797C07A
:106B0000FFFFE780C06437A507001305051297C093
:106B1000FFFFE7806060014597C0FFFFE780806668
:106B200095450545894717F7FF1F2305F7BE97C011
:106B3000FFFFE780C066B7E700E013070006238D7C
:106B4000E7403707000423A0E71097D0FFFFE78056
:106B5000E0F797D0FFFFE780A00B97000000E780E9
:106B600080E697000000E780408B97000000E780F8
:106B7000E0B597E0FFFFE78080E797000000E7803F
:106B8000C01C97000000E780600B83A7040817056E
:106B900000001305C5BF829797D7FF1F2380A782E8
:106BA000BC4C130600648545829797000000E7807F
:106BB00000E897C0FF1FE780A08301458280B7F7F8
:106BC000070003C70701A547AE866316F700939732
:106BD000450191C301A0AA850146254517C3FF1FA2
:106BE000670083BE4111B2862E86AA852D4506C652
:106BF00097C0FF1FE78040BDB24001454101828040
:106C00009307000463E8C7021D71A2CC2A84080818
:106C100086CE32C697800100E78020BDB2461008BC
:106C2000A285294597C0FF1FE78000BAF640664459
:106C3000256182803955828041110D658D4506C6DA
:106C400097C0FFFFE780E018B71700408D6623A6C6
:106C5000D70A17F5FF1F130525AC1387C70A9387BB
:106C6000870A1CC15CC5856689675CC958C114C5A3
:106C700018C9B7E70400B24003A3871E410102838D
:106C80008145B307B5008387070089E71723000014
:106C9000670023A28505C205C181E5B7411126C25F
:106CA000E97797F4FF1F9384A4B722C49387A7556D
:106CB0002E842381B4002E86AA8517F5FF1F1305A5
:106CC00065B606C62390F400A381040097800100F6
:106CD000E780A0B193052400C205C18117F5FF1F0D
:106CE000130525B497000000E780408AB38784002D
:106CF0002382A7002181A382A70093056400224478
:106D0000B24026859244C205C1814101172300008B
:106D10006700239A09C99307800263E6B700170347
:106D200000006700E3F7828017F5FF1F034545A0C9
:106D3000828097F7FF1F83C767AE89E7172300009C
:106D400067002397828097F7FF1F83C747B099EFAB
:106D5000411106C697200000E780808DB24085472C
:106D600017F7FF1F2305F7AE410182808280630E73
:106D70000532638C05325D71CAC04EDE86C6A2C480
:106D8000A6C252DC56DA5AD85ED662D466D26AD02F
:106D9000B9472A89AE8963F9B706394697A5010034
:106DA0009385453D97800100E780C0A131ED834781
:106DB000E900130710036394E702854717F7FF1FE5
:106DC000230EF7A417A501001305C53B97F7FF1F76
:106DD000239507A497000000E780C0EA71A013077D
:106DE000000317A501001305E53CE395E7FE97F7BF
:106DF000FF1F238507A297F7FF1F239007A217A560
:106E000001001305A539F9B797F7FF1F83C707A13D
:106E100063870722BD6AB96B938CFA55014A17FB49
:106E2000FF1F130B2B91138CEB65938AFA6605A851
:106E3000B307490183C6070097F7FF1F83D7E79D74
:106E4000B1E39307A005639BF600854717F7FF1F83
:106E50002315F79C97F7FF1F238ED78C050A9317EE
:106E60000A01C183E3E637FDB6402644964406494D
:106E7000F259625AD25A425BB25B225C925C025D6A
:106E800061618280054D639BA7039307500A639E4F
:106E9000F600894717F7FF1F2311F798930750FA59
:106EA00017F7FF1FA308F78855BF9307A005E387CF
:106EB000F6FA97F7FF1F239207964DB7138717002F
:106EC0004207DA9741832380D70017F6FF1F231666
:106ED000E6948D47E3F4E7F817F4FF1F0344B48505
:106EE00097F7FF1F83C7278522045D8C9307F4FF64
:106EF000C207C1839306F00DE3EDF6FA9307640031
:106F0000C207C183E31CF7F493052400C205C181C5
:106F100017F5FF1F1305258297F0FFFFE780006735
:106F200033078B008347570003474700A207D98FD9
:106F300017F7FF1F2313078E6318F50E8144630CA8
:106F4000A40197E4FF1F83C4247FA20497E7FF1FD7
:106F500083C7977EDD8C170500001305E5DB97F0EE
:106F6000FFFFE78000FE63878407636D9C029387C1
:106F7000EB556382F40497E7FF1F83C7E77B054760
:106F80006389E70681CB1387A7051377F70F8D4633
:106F900063F2E6081307F0072300E100A300F10005
:106FA00089459DA063829405E39754FD97F0FFFF08
:106FB000E780202A11A8A28517E5FF1F1305C577D2
:106FC00097F0FFFFE780E00D014597F0FFFFE780B6
:106FD00040F769B5A28517E5FF1F1305E57597F022
:106FE000FFFFE780A017CDB797F0FFFFE7802020D5
:106FF000E1BF930710F8130511002300F10097F08B
:10700000FFFFE780C02BFD450A8597000000E78061
:1070100020C95DBFA28517E5FF1F1305E57197F035
:10702000FFFFE780A0C84DB79307F00789450A85A1
:107030002310F10097000000E78080C605B5C14726
:1070400063FE3705414697A501009385E5184A85FB
:1070500097700100E780007731E18347090113074A
:107060001003639CE700854717E7FF1F2302F76CB7
:1070700017A5010013058517B1BB1307000317A55A
:1070800001001305A519E397E7D497E7FF1F2381B4
:10709000076A17A501001305E5162DBBCE854A85A5
:1070A00097C0FFFFE7804012C1B38280411126C222
:1070B000AE848D4522C406C62A8497C0FFFFE780B0
:1070C000A0DBB717004099C803A5C70C418D23A6C4
:1070D000A70CB240224492444101828003A5870C50
:1070E000418D23A4A70CF5B783470500034715007E
:1070F000A207D98FC2076177C18713072720639A38
:10710000E7008345250037050400170300006700EA
:1071100023FA828017E6FF1F1306C6738147B286E3
:107120001303F00FA9483308F6000348080013F7CB
:10713000F70F6307A80C630668008507E39517FF40
:107140002947B387E6002380A70097E7FF1F9387AF
:1071500027715DA8411113D765001347170006C6B4
:1071600093F63500058B954791CA05469947638785
:10717000C60009469D476383C600A14713F6450034
:107180003336C00093F68503050685C2A145638B9F
:10719000B604E145638AB604930580026388B604A9
:1071A000930580036393B600914697F5FF1F238EE6
:1071B000F59097F5FF1F2389C59097F5FF1FA385CD
:1071C000D590BE8517A501001305450A97700100EB
:1071D000E780006DB240854717F7FF1FA307F78EC2
:1071E000410182808546D1B78946C1B78D4675BFBA
:1071F00017A501001305050A177301006700436A0C
:1072000017E7FF1F1307C765BA972380B700E14749
:10721000E302F5F493077002E30CF5FC82802A8701
:1072200023800500814717E5FF1F1305A56213089A
:10723000F00F2946B306F50083C606006396E60202
:1072400097E6FF1F9386C661B69783C7070005457B
:107250002380F5009947636EF7029D4763FDE700C1
:10726000E147630DF7008280638506018507E3939C
:10727000C7FC0145C5B7238005008280B7370040B1
:1072800003C7370083C7050093F70704D98F23800E
:10729000F5008280797126D24AD097F4FF1F83C40B
:1072A000A49417F9FF1F1309699306D622D44ECE72
:1072B00052CC56CA5AC8B307990083C7070093F740
:1072C000F70FA5C79387140093F7F70F0D47636176
:1072D000F70C17F7FF1F2309F79097F7FF1F938706
:1072E0006790A69783C707001307100293F7F70369
:1072F0006389E7226363F70A054463808720E3829A
:10730000076809476389E71413070002E387E75218
:10731000B7E700E03707400023A0E71801000100AD
:10732000CA942380040023A0E710B787004003C756
:107330006700058BE308077297F6FF1F83C6E68A8E
:107340000547E393E67029472381E7020947238332
:10735000E7022385E70297E7FF1FA389077697F7E0
:10736000FF1FA3840788B7870040A381070017E7A2
:10737000FF1FA30F077405472383E700B250225471
:1073800092540259F249624AD24A424B4561828084
:1073900097F7FF1F238A078489B713073002638694
:1073A000E70A63E6E71413074002638AE708130756
:1073B0000003E39FE7F497F7FF1F93876782A69781
:1073C00003C70700A1471377F70FE313F71617EA70
:1073D000FF1F130AAA4983476A0097E6FF1F238D00
:1073E000F66C97E7FF1F83C7D74891C7FD5797E60D
:1073F000FF1F2383F66C97E5FF1F83C5354797E78B
:10740000FF1FA38BB76A97E7FF1F83C7274693F930
:1074100007089306000493F70706639DD74A93076E
:10742000A0096387F51463E4B7109307F00563843C
:10743000F548930750096382F52801440DABFD57C9
:1074400017E7FF1F2309F766E1B5FD5717E7FF1F91
:107450002302F76675BD17A50100130525F5977082
:107460000100E780C05B97E7FF1F93876777A697C8
:1074700003C40700814917EAFF1F130AAA571374B0
:10748000F40F97AA0100938AEAF263C78904294599
:1074900097700100E780A045854717E7FF1FA30904
:1074A000F75417E7FF1F2306875417E7FF1F230F23
:1074B000F76037E700E0B70640002320D718010047
:1074C0000100378600408347A60293F7370F230554
:1074D000F6022320D7102DBDB3073A0183C507005C
:1074E0005685850997700100E780803B79BF854705
:1074F00017E7FF1F230EF74E21BD17E7FF1F1307E6
:10750000276E26970347070097E6FF1FA380F642E2
:1075100097E6FF1F238DE64017E7FF1F2308F75A62
:10752000C5BB854717E7FF1F2302F740D5B3930775
:10753000400A638DF5349307200B6388F536930773
:10754000100AE39CF5EE83072A00014463D1074249
:1075500097E7FF1F83C7B73193F63700638E061A8C
:107560000546638EC62209466399C61A1D4775A251
:1075700017E5FF1F0345A52FC94717EAFF1F034A59
:107580001A2F97E5FF1F83C5A52E17E4FF1F03449D
:10759000342E6319F510CD476316FA10930770085F
:1075A000639CF5021307300FB7170E006308E40061
:1075B0001307900DB7B704006314E40817E7FF1F23
:1075C0002322F750BE8517A50100130525DF97700C
:1075D0000100E780E02C95B593078008639DF500D6
:1075E00033048040B77746001374F40F938787CD38
:1075F000B3D78702E1B793079008639AF500330485
:10760000804091671374F40F9387C766D5B79307CB
:10761000A008639BF50033048040B7173D00137446
:10762000F40F93870790E9B79307B008639AF500C2
:107630003304804091671374F40F938797D04DBF44
:1076400093F5F5078D47639BF50033048040B797AA
:107650005B001374F40F938707D859BF8947639B66
:10766000F50033048040B7770B001374F40F938751
:10767000071BBDBF8547639AF50033048040DD6773
:107680001374F40F938767E3A5B789E93304804047
:107690008D671374F40F938777DC99BFF167938735
:1076A000072029BF97000000E78000A7A285528528
:1076B00097000000E78040A649B39305610017E5F5
:1076C000FF1F0345C51A17E4FF1F0344541A970010
:1076D0000000E78000B59305710022859700000047
:1076E000E78020B43C0017E7FF1F2327F74E8347AE
:1076F00061002304F10083477100A304F10089476E
:1077000017E7FF1F230AF73A8357810017E7FF1F88
:10771000231EF7140944A1AC154793F64700B3366E
:10772000D00093F78703850685C32146638BC70680
:107730006146638AC706130680026388C70613067C
:1077400080036393C700914717E6FF1F230ED636C9
:1077500097E6FF1FA38AF63697E7FF1F2387E736D2
:1077600017E7FF1F0347C7109376070497E7FF1F2C
:1077700083C717108DEE1377770C93067008630C90
:10778000D7021377F7078D46631ED70AB307F04079
:10779000B7955B0093F7F70F938505D881A8194734
:1077A000ADBF854755B7894745B78D4771BF93062C
:1077B00070086311D7021307300FB7150E006389E5
:1077C000E7021307900DB7B504006383E7021307C0
:1077D000700845BF9306800C6311D702B307F040D1
:1077E000B775460093F7F70F938585CDB3D5F502AE
:1077F00097E7FF1F23A8B72CF9B39306900C631AE1
:10780000D700B307F040916593F7F70F9385C566EE
:10781000F1BF9306A00C631BD700B307F040B71568
:107820003D0093F7F70F93850590C9B79306B00C09
:10783000E319D7F4B307F040916593F7F70F9385F9
:1078400095D06DB78946631BD700B307F040B77575
:107850000B0093F7F70F9385051B49BF8546631A05
:10786000D700B307F040DD6593F7F70F938565E325
:10787000B5BF09EBB307F0408D6593F7F70F93851C
:1078800075DCADB7F165938505209DB783472A0068
:10789000C18B99C7854717E7FF1F2302F72271BEE7
:1078A00097E7FF1F238D072049BE854717E7FF1F76
:1078B000A30DF72059B63C0017E7FF1F232EF73022
:1078C0000947930700032314F10097E6FF1F238560
:1078D000E61E2DBD63990758A94763EBB74417A768
:1078E00001001307E7958A05BA959C41BA978287EC
:1078F00017E4FF1F0344B4F7094A630C440F636C99
:107900008A0885476309F40A9307F00F17E7FF1FFA
:107910000347871A63F6E70017E7FF1F230EF718E0
:1079200017EAFF1F034A4A19930700041374FA0F5A
:1079300063F447011304000497E7FF1F9387C729E7
:1079400083AA0700228617E5FF1F130525F2D685B7
:10795000330A8A40A29A97700100E78000E997E70E
:10796000FF1F238B471597E7FF1F23A7572797E78D
:10797000FF1F83C7771415476399E762B7E700E0F5
:107980003707400023A0E71801000100B786004038
:107990002380860285A58D47630CF40A9947E31579
:1079A000F4F697A701009387279017E7FF1F232579
:1079B000F722A947A1BF17E7FF1F0347072397E750
:1079C000FF1F93876711494697A501009385C596C8
:1079D0006306870097A50100938505923E85977001
:1079E0000100E78080E017E7FF1F2327A71EC94794
:1079F00031BF97E6FF1F83C6461F054797E7FF1F66
:107A00009387870D6394E6023E851306700297A55F
:107A100001009385E58F97700100E78000DD17E78F
:107A2000FF1F232BA71A93077002CDB53E851306BF
:107A3000300497A501009385E58797700100E780E2
:107A4000C0DA17E7FF1F2329A718930730047DBD6D
:107A500097E5FF1F83C5A5E117A50100130545970D
:107A600097700100E780C0E3854A17EBFF1F034BC7
:107A7000CB1797E5FF1F83C585DF17A50100130509
:107A8000259563185B0B97700100E78060E197E72D
:107A9000FF1F83C7C7DDB5CBE368F4E617A4010079
:107AA0001304C48D638C670117A401001304848D33
:107AB0006386470117A401001304448E2285977042
:107AC0000100E78080FE1375F50F93071500860708
:107AD00017E7FF1F2302F7008D4717E7FF1FA30DCE
:107AE000F7FE97E7FF1F938727FF0147BE861376B0
:107AF000F70F89076365A60297E7FF1F23AED70C30
:107B000097E7FF1F83C747FD11B59797010093873C
:107B1000E77F17E7FF1F2321F70C9147C5BB33060B
:107B2000E40003460600A380070005072380C70082
:107B30007DBF97700100E780A0D697E7FF1F83C73E
:107B400007D3E1D7E362F4DC17A401001304048037
:107B5000638C5701179401001304C47F63864701A7
:107B600017A4010013048480228597700100E78028
:107B7000C0F31375F50F93071500860717E7FF1F6E
:107B8000230CF7F48D4717E7FF1FA307F7F497E7D8
:107B9000FF1F938767F40147BE861376F70F8907A7
:107BA000E37CA6F43306E40003460600A380070046
:107BB00005072380C700D5B797E5FF1F83C525CBF1
:107BC00017A501001305858197700100E78040CD5E
:107BD00097E7FF1F83C717F093E7470017E7FF1FDB
:107BE000A30AF7EE83472A0017E7FF1FA302F7EE69
:107BF000A9B0179501001305A57F97700100E780D4
:107C000000E297E7FF1F9387A7EC83C7070017E7FA
:107C1000FF1F230DF7C417E4FF1F0344E4E93334C7
:107C20008000B1B3179501001305C57D9770010061
:107C3000E780E0DE97E7FF1F83C7D7E993E70701F7
:107C400017E7FF1FA308F7E883472A0017E7FF1F7E
:107C50002300F7E86FF06FFE179501001305C57B51
:107C600097700100E780A0DB03470A007D8B51EF8E
:107C7000B787004003C767021377C70B1367270056
:107C80002383E70203C7A7021377C70B13672700F5
:107C90002385E70203C7E7021377C70B13672700A3
:107CA0002387E70203C727031377C70B1367270050
:107CB0002389E702854717E7FF1F2309F7C617E760
:107CC000FF1F2307F7D217E7FF1F2305F7DE17E78C
:107CD000FF1F2302F7DE97E7FF1FA38907C497E77B
:107CE000FF1FA38707D097E7FF1FA38507DC97E750
:107CF000FF1FA38207DC97E7FF1FA38907DC97E735
:107D0000FF1FA38407EE6FF04FF389476312F7025A
:107D100097E7FF1F83C7C7B59146638CD70863E019
:107D2000F604638EE70C6369F70A05476380E70E84
:107D3000FD5717E7FF1FA301F7D837074000B7E744
:107D400000E023A0E71801000100B78600401306F9
:107D5000F0FC2381C60223A0E7106FF06FDB13074E
:107D600020086382E7086362F70213071008E391B3
:107D7000E7FC378700408347670293F7C70B93E719
:107D800027002303F7026FF04FEB130730086389D6
:107D9000E70213074008E39DE7F837870040834771
:107DA000270393F7C70B93E727002309F7026FF028
:107DB000CFE8378700408347270393F73707F5B7A6
:107DC000378700408347E70293F7C70B93E7270005
:107DD0002307F7026FF06FE6378700408347E7021B
:107DE00093F73707F5B7378700408347A70293F724
:107DF000C70B93E727002305F7026FF00FE43787DF
:107E000000408347A70293F73707F5B7378700404D
:107E10008347670293F73707ADB71795010013053E
:107E2000A56097700100E78080BF97E7FF1F238F51
:107E300007A2D5B3179501001305056097700100DF
:107E4000E780E0BD97E7FF1F239207A297E7FF1F98
:107E5000938787C603C40700894763F387000944F3
:107E60001374F40F29B613070002E393E7EC639948
:107E7000090A638FF500930720026381F5081795BF
:107E800001001305E55E97700100E78060A14DB524
:107E9000179501001305055B97700100E78020B876
:107EA0000144179B0100130B2B5BA14AB3078A0007
:107EB00083C507005A85050497700100E780409E3E
:107EC000E31654FF179501001305C5B19770010023
:107ED000E780E0B417E4FF1F0344849911E497E7B7
:107EE000FF1F2387079661B48947E313F4E48547AE
:107EF00017E7FF1F230EF7946FF02FD417E6FF1F2D
:107F00000346F69697E5FF1F83C565961795010012
:107F10001305055597700100E78080986FF0EFD149
:107F2000638FF50493071002E39BF5F497E5FF1FB9
:107F300083C50594179501001305855497700100BA
:107F4000E780009697E7FF1F23A847C997E7FF1F21
:107F5000938747B7944383D7470017E7FF1F03472B
:107F6000C7B617E6FF1F2323D6901D4497E6FF1FD1
:107F70002390F69097E7FF1F238DE78ECDBA97E504
:107F8000FF1F83C5E58E179501001305E550977017
:107F90000100E780E09097E7FF1F238B078A97E7B0
:107FA000FF1F2395078C6FF0EFF62547E388E79CCA
:107FB00019476391E702B786004023808602B7E73E
:107FC00000E03707400023A0E71801000100130676
:107FD00000FC41B31307100A6391E702B786004023
:107FE00023808602B7E700E03707400023A0E718A8
:107FF00001000100130680FCA9BB1307A009E38F51
:10800000E7FC1307400AE38BE7FC13072002E38732
:10801000E7960547E384E796B7E700E037074000B7
:1080200023A0E718E392099601000100B7860040FB
:1080300023808602130620FC29BB17E7FF1F034796
:10804000B7A76308F71E63E7E7029547630EF70ECD
:1080500099476308F704B786004023800602B7E714
:1080600000E03707400023A0E718010001001306D5
:10807000A0FCC5B19307F005630AF7009307500908
:108080006306F70093071002E317F7FCB7E700E079
:108090003707400023A0E71801000100B786004021
:1080A00051BF97E9FF1F83C929A193070004CE8A16
:1080B00063F43701930A000497E7FF1F9387C7B162
:1080C00003AA070013F4FA0F2286D28517D5FF1FE3
:1080D0001305C57997600100E7802071B387894057
:1080E000529417E7FF1F2309F79C97E7FF1F23A56B
:1080F00087AE638E0902B787004023805703B7E637
:1081000000E03706400023A0C6180100010003C7A5
:108110002702134707042381E70203C727021377C7
:10812000C70F2381E70223A0C6106FF06F9EB786AA
:10813000004023800602B7E700E03707400023A095
:10814000E71801000100FDB537870040834737007D
:1081500097E6FF1F83C6D69793F70708D58FA3012D
:10816000F700B7064000B7E700E023A0D7180100EA
:1081700001001306A0FC2301C70223A0D7106FF053
:108180002F9997E7FF1F9387A7A5A69783C7070097
:1081900093F7F70FD9CF97E7FF1F83C707A5D1EB59
:1081A00017E7FF1F03475791930700026313F70870
:1081B00097D7FF1F9387876B03AB070097DAFF1FE3
:1081C00083CA0A6B17DAFF1F034A9A6A97D9FF1FFF
:1081D00083C9296AD2875687CE865A8697D5FF1FCC
:1081E00083C50567179501001305852C976001006D
:1081F000E780006B97E7FF1F23A6678D97E7FF1FB8
:108200002384578D97E7FF1FA380478D97E7FF1FB4
:10821000238D378B97D7FF1FA38B8762B7E700E0CB
:108220003707400023A0E71801000100B78600408F
:10823000D1B3B7E700E03707400023A0E7180100FB
:108240000100B786004025B529472381E702094789
:108250002383E7022385E7022387E7022389E702D6
:108260006FF06F8F03C76700118B6309079083C797
:108270005700918BB5CF17E7FF1F03470797854737
:108280006313F70697E7FF1FA381E78497D7FF1FC4
:10829000238E076897D7FF1F238C077497E7FF1F6C
:1082A000238A078097E7FF1F2387078097D7FF1F41
:1082B000A38E076697D7FF1FA38C077297D7FF1F60
:1082C000A38A077E97D7FF1FA387077E97D7FF1F35
:1082D000A38E077E97E7FF1FA3890790B78700400B
:1082E00011476FF06F8917D7FF1FA302F75679BFA9
:1082F000854717D7FF1F230BF76217D7FF1F2309E7
:10830000F76E17D7FF1F2307F77A17D7FF1F23042E
:10831000F77A69BF854717D7FF1F2309F76017D77B
:10832000FF1F2307F76C17D7FF1F2305F77817D711
:10833000FF1F2302F77817D7FF1FA309075E17D780
:10834000FF1FA307076A17D7FF1FA305077697D755
:10835000FF1FA38207768280411106C697000000A6
:10836000E78080FBB787004023800700130740FCAD
:108370002386E7001307C004A386E70017D7FF1F73
:108380001307C74E2398E70017D7FF1F130707529D
:10839000239AE70017D7FF1F1307875D239CE70089
:1083A00017D7FF1F13070769239EE700294723817B
:1083B000E70209472383E7022385E7022387E702D1
:1083C0002389E702A3810700930600F8A380D70062
:1083D000930690022380D700FD562383D700238184
:1083E000E700B706400037E700E02320D71003C7B7
:1083F000170013671700A380E700B24097D7FF1F4D
:108400002398076C41018280411106C69700000045
:10841000E78080F0B787004023800700130700FC47
:108420002386E7003147A386E70017D7FF1F13070E
:10843000E7432398E70017D7FF1F13072747239A1F
:10844000E70017D7FF1F1307A752239CE700294710
:108450002381E70209472383E7022385E702A381FB
:108460000700930600F8A380D700930690022380AC
:10847000D700FD562383D7002381E700B7064000CD
:1084800037E700E02320D71003C717001367170052
:10849000A380E700B24097D7FF1F239B07624101EB
:1084A0008280F1679387072017D7FF1F232CF7607F
:1084B000854717D7FF1F2319F760A14717D7FF1F5D
:1084C0002305F76097D7FF1FA381076097D7FF1F8A
:1084D000238E075E97D7FF1F238C073697D7FF1F82
:1084E000A3870736814717D5FF1F1305A536FD550E
:1084F00017D6FF1F1306C6362947B306F50023809B
:10850000B600B306F600238006008507E397E7FE72
:1085100097D7FF1F2384076C97D7FF1FA380076C93
:1085200097D7FF1F238D076A97D7FF1FA387075889
:1085300097D7FF1FA385075897D7FF1F238007589A
:1085400097D7FF1F238B075697D7FF1F238A0756FE
:1085500097D7FF1FA384075697D7FF1F238107567E
:1085600097D7FF1FA38D0766828017D7FF1F03478A
:10857000C76785476316F70017030000670003E924
:1085800017030000670083DD411122C406C617D718
:10859000FF1F0347876585472E8613F4F50FAA85CD
:1085A0006317F70417D5FF1F130585409760010077
:1085B000E780A02397D7FF1F238C0742B78700408F
:1085C00023848702B7E600E03706400023A0C618E0
:1085D0000100010003C7A7021377C70F2385E70235
:1085E000B240224423A0C61001454101828017D524
:1085F000FF1F1305A52F97600100E780001F97D785
:10860000FF1F23850732B787004023828702B7E622
:1086100000E03706400023A0C6180100010003C790
:1086200067021377C70F2383E7025DBF411106C6B8
:1086300097000000E78020E7B240410117030000E7
:108640006700E3F2411106C697F0FFFFE780C0C460
:1086500097D7FF1F83C7972DA1CB97D5FF1F83C542
:10866000052D89C917D5FF1F1305852C97E0FFFF3E
:10867000E780207097D7FF1FA38A072A97D7FF1F8D
:108680002386074437E700E0B70640002320D718C9
:1086900001000100378600408347660293F7370FD9
:1086A0002303F6022320D710B2404101828041C942
:1086B000D9C597D7FF1F83C7A741D1C3011122CCCA
:1086C0004AC84EC656C25AC006CE26CA52C42E89C1
:1086D000AA890144930A0004371B0300637724032B
:1086E000B3078940C207C183BE8463F4FA009304D0
:1086F0000004C204C180130A1BD497D7FF1F83C78D
:10870000E7229DE37D1A631C0A00F2406244D244D2
:108710004249B249224A924A024B0561828097F04F
:10872000FFFFE78060B7D1BF338589002694A68517
:10873000420497000000E78060E5418045B78280F1
:1087400097D7FF1F9387074E18429C4383D6450057
:108750000345070083C5C700035646006396A5007E
:1087600083D5E700638DD502011106CE2386A700CD
:108770002397D700B705CF00DC4B9385757D0507A0
:108780007D162EC2230001003AC42316C100231710
:10879000D10099C30A858297F24005618280828068
:1087A000DC4DDC4B81CFB7E70400904503A3870580
:1087B000914517D5FF1F03452547028382806D71C0
:1087C0003C083EC6B707E500232291103EC8AA84A4
:1087D0003C083285232611103ECA23248110232011
:1087E00021112E8997300000E780E0552A84979563
:1087F0000100938565CF178501001305E5B79760E4
:108800000100E780E009A28517950100130545DE08
:1088100097600100E780C008294597600100E78064
:10882000000DB705CB009385757D6800971000009B
:10883000E780005FA285680097300000E780004372
:10884000014781467000CA85268597200000E78091
:10885000808205CD2A84979501009385E5C8178508
:108860000100130565B197600100E7806003A285F0
:1088700017950100130585D897600100E780400235
:10888000294597600100E78080068320C1100324FA
:10889000811083244110032901105161828097D7F0
:1088A000FF1F9387273818429C43797122D406D63C
:1088B0000348070083C807012A8483D6450003556F
:1088C00046006396080183D82701638DD802238868
:1088D000070105072399D7003708CC00DC4B1308A4
:1088E000787D3ACC1307F5FF42CA23080100231E06
:1088F000E100231FD10099C7080832C62EC4829711
:108900003246A245228597000000E78080EBB250F6
:108910002254456182806D713C083EC0B707E50076
:108920003EC23C083EC4232611102324811023227A
:108930009110231701002318010023190100231AA5
:108940000100231B010097B7FF1F83D7A7A999E355
:10895000C167FD172316F10097B7FF1F83D7A7A89C
:1089600091EB97D7FF1F9387E72B9C439C43DC47F2
:1089700083D7070017B4FF1F1304C4A6584C23174E
:10898000F10083574400484B2318F10031E19795DB
:108990000100938565BC178501001305E59D97606F
:1089A0000100E780E0EF17950100130525BC9760F3
:1089B0000100E780E0EE294597600100E78020F3A1
:1089C0008320C110032481108324411051618280CF
:1089D00097B7FF1F83C777A189EBB7E70400BC57A0
:1089E00082975C4C23AA0700E1BFFD1797B6FF1FD3
:1089F000A38DF69E03560701834704014C470A8561
:108A0000230BF10097300000E780602397D7FF1F0A
:108A1000938747219C430147814688430A866C001F
:108A200097100000E7802065AA8429C1979501006E
:108A3000938585B2178501001305059497600100A1
:108A4000E78000E6A685179501001305E5B297605B
:108A50000100E780E0E4294597600100E78020E914
:108A6000584CB7E70400BC57484B9DBF97B7FF1F52
:108A700083C7B797F5D7B7E70400BC4F10448545C7
:108A800017D5FF1F0345451A82971DBF5C4EDC4B6F
:108A9000B9CFB1CD411122C4178501001305C58D91
:108AA0002E8497950100938565A906C697600100FD
:108AB000E78000DFA285179501001305A5AE97603A
:108AC0000100E780E0DD294597600100E78020E2B2
:108AD000B7E704002244B24003A3870517D5FF1F60
:108AE00003458514130640069145410102838280A7
:108AF000411122C417B4FF1F1304848C1C4C06C6FA
:108B000089C7DC4399C34C488297584CB7E70400A7
:108B1000BC57484B82975C4CB240224423AA0700C2
:108B20004101828017B7FF1F1307878B8347070018
:108B30009306F00B850793F7F70F63E9F60097B6F6
:108B4000FF1F238FF688034507008280930700F8F4
:108B5000FDB7835745006386071001114AC817B94E
:108B6000FF1F1309298852C4032AC90106CE22CC4B
:108B700003274A0126CA4EC656C2F15735E31307EA
:108B8000D00DFD57636EC704B7E9040083A709073A
:108B90002A841305860042054181B284AE8A8297F9
:108BA000232AAA000325C9015C49A9E7979501007A
:108BB0009385C596177501001305057C9760010024
:108BC000E78000CE17950100130505A69760010008
:108BD000E78000CD294597600100E78040D1DD574F
:108BE000F2406244D2444249B249224A924A3E8506
:108BF0000561828093874400B705CF002319F500F3
:108C00009385757D310597100000E780602103256D
:108C1000C90183456400310597300000E7800005F5
:108C20000325C9012686D685310597300000E780E7
:108C300000017146A2854A8597600100E780E0BA8D
:108C4000504419CA83A78905854517D5FF1F0345D9
:108C5000A5FD8297814769B797000000E780E0CBC8
:108C6000D5BFFD573E858280411126C297A4FF1FC4
:108C700093844477D84C22C437E404003C54484BD6
:108C800006C68297DC4C0323C4052244B2409244BA
:108C900023AA070017D5FF1F034505F985454101A4
:108CA0000283411126C297D4FF1F9384A4F79C40EE
:108CB00006C622C44AC0D5C3DC43C5C35CC1230079
:108CC000B5002A849795010093858580177501006A
:108CD0001305856A97600100E78080BC294597608D
:108CE0000100E780C0C09C4023A4070023A2070026
:108CF00097A7FF1F9387C76CDC4FDC4B91C72955A3
:108D000097000000E78000DF97A7FF1F9387876D1C
:108D1000DC4FDC4B89C797000000E78020F537E97E
:108D200004008327C905894517D5FF1F0345C5EFF3
:108D300082978327C905914517D5FF1F0345C5EEC7
:108D400082979C4003A347016309030022852244C4
:108D5000B2409244024941010283B240224492440B
:108D60000249410182800111328506CE22CC26CAF9
:108D70002E8497300000E78000FDAA8497850100CB
:108D800093854578177501001305055F976001000D
:108D9000E78000B103078400035664008355440054
:108DA000A686179501001305E58197600100E7800D
:108DB00020AF294597600100E78060B397A7FF1FA8
:108DC00083C76760639D9700014597000000E780B7
:108DD00060D281450A8597000000E780C0ECF24030
:108DE0006244D244056182806D7123248110232660
:108DF00011102322911093F745002E8463870714E6
:108E00003C083EC0B707E5003EC23C083EC42317FD
:108E100001002318010023190100231A0100231B5C
:108E2000010097A7FF1F83D7A75999E3C167FD17D3
:108E30002316F10097A7FF1F83D7A75891EB97D769
:108E4000FF1F938727DE9C439C43DC4783D70700A3
:108E500017A7FF1F1307C7562317F100544F835757
:108E600047002318F100DC4AA1E7978501009385AC
:108E7000A56D177501001305255097600100E78067
:108E800020A2178501001305656E97600100E78039
:108E900020A1294597600100E78060A513454400A3
:108EA0008320C110032481108324411051618280EA
:108EB00097A7FF1F83C737512555D9C3FD1717A69D
:108EC000FF1FA302F65003D6060183470701CC46D5
:108ED0000A85230BF10097300000E78040D697D732
:108EE000FF1F938727D49C4317A7FF1F1307474DE6
:108EF000978601009386866A88430A866C009710DD
:108F00000000E7804017AA8451D997850100938516
:108F1000A563177501001305254697600100E780DA
:108F20002098A68517850100130505659760010047
:108F3000E7800097294597600100E780409B2685E0
:108F400097000000E78000BB91BF93F725009DC705
:108F5000B7E70400BC47414681452808829725555C
:108F600097000000E78000B928089305F00F9700EC
:108F70000000E78040D3134524001DB793F7150088
:108F8000014599DF97000000E78020991345140000
:108F900001BF5C4D411106C688C317D7FF1F2323AD
:108FA000F7C8B7E7040083A70708170500001305F3
:108FB000E5E38297B24097D7FF1F2387A7C60145F5
:108FC0004101828001113335A000A307A100B7E75A
:108FD000040083A7471706CE1306F1008545130545
:108FE00050308297F240056182808280411122C414
:108FF00006C697D7FF1F83C7A7C4014489EF97B759
:10900000FF1F83C77720054499E717C4FF1F034458
:10901000E45F13441400228597000000E780C0FA43
:10902000178501001305056C09E417850100130578
:10903000656C2244B240410117630100670043861A
:10904000797122D4A30F010037E404008327841729
:1090500026D24AD006D6AA842E891305503093050D
:10906000F10132C6829732468347F101931506011A
:10907000C18185CB01452EC697000000E780C0F472
:1090800083274417B2454A8626858297054597006F
:109090000000E78060F3B2502254925402594561B7
:1090A0008280832744174A8626858297EDB741112F
:1090B0009397050122C406C626C2C1872E8463D4B5
:1090C0000702B7E40400FC5417A5FF1F03458534CD
:1090D000829719C1BC5482972165218DB2402244E8
:1090E00092444101828093F715008DC7B7E70400D1
:1090F00083A7471A17A6FF1F1306C63097D5FF1F71
:10910000938545B317A5FF1F0345C53082971345C7
:109110001400E9B793F7250099CFB7E70400BC4FD7
:1091200013060064894517A5FF1F0345A52E8297E6
:109130001345240065B793F7850095C7B7E704008A
:1091400003A8871A1307401F97A7FF1F83C7872C01
:1091500081466146994517D5FF1F0355A5AE029874
:1091600013458400A5BF93F745000145A5DBB7E48F
:10917000040083A7041817D5FF1F0355A5AC8297D9
:10918000BC4C13060064914517A5FF1F03458528B5
:1091900082971345440099B797D7FF1F83D787AAB3
:1091A0006398A70217D7FF1F231FB7A817D7FF1F62
:1091B000231CC7A817D7FF1F2319D7A82E861785EA
:1091C000010013056558BE85175301006700436D04
:1091D000178501001305C558176301006700238434
:1091E0000357450097D7FF1F83D7C7A5631AF70416
:1091F000C1674111F91722C417D7FF1F2324F7A411
:1092000037E4040097D7FF1F23A007A497D7FF1FB9
:10921000A38807A27C4C06C6894517A5FF1F0345F6
:10922000651F82977C4C914517A5FF1F0345851E3E
:1092300082972244B240410117030000670043DBDC
:10924000178501001305C551175301006700237DE1
:109250007D15954763E2A71C178701001307474652
:109260000A053A951C41011122CC06CEBA972E84EC
:109270008287178501001305254F97500100E7806D
:10928000007AA1A203C7250099476311F7022E8532
:1092900097000000E78000F5834564001785010012
:1092A0001305854D97500100E780805F97B7FF1F3A
:1092B000238C07F4178501001305C54D7DBF03C737
:1092C000250095476319F702C16717D7FF1F03579A
:1092D0006797F91703D5A5006309F702B7E70400FC
:1092E00083A7C7178297178501001305A54B9750D1
:1092F0000100E780C072854717B7FF1F2306F7F00C
:10930000178501001305854C8DBF97D7FF1F239B41
:10931000A79283D7E50097D6FF1F2396F69283D7AF
:10932000050197D6FF1F2391F69283D7250197D683
:10933000FF1F239CF69097D7FF1FA3830790631B03
:10934000E502B7E70400BC4F096613060690A14585
:1093500017A5FF1F0345050C82970356E4008355AC
:10936000A400178501001305254597500100E780EB
:10937000205351B79307700F2316F100B7E704008D
:1093800083A7870D17A6FF1F0346C6086C008297A8
:109390004DF9854717D7FF1FA304F78A5DB71785D7
:1093A000010013056543D1BD83C525009147639234
:1093B000F502178501001305A54397500100E780CA
:1093C000006697000000E780A0C2F2406244056199
:1093D000828099476392F502228597000000E7801A
:1093E00060E083456400178501001305E538975058
:1093F0000100E780E04AD1BF9547639AF5008347B3
:109400001400E1F3178501001305C540BDB51785AC
:1094100001001305A540E1BF82806D7123248110F6
:109420002326111023229110328401CD8947630A2B
:10943000F5028320C110032481108324411051615F
:109440008280178501001305253EAE8497500100E8
:10945000E780E05CA285268597C0FFFFE780E011EA
:10946000C9BFB7E70400FC472800829717850100B1
:109470001305453C97500100E780605A83478100FF
:1094800039C41307000B6380E7021387A70513771E
:10949000F70F8D4663EDE602A285280097D0FFFF07
:1094A000E780C08079B78547E3F587F88345910069
:1094B0001775010013058521B335B00097B7FF1F5D
:1094C0002384B7BC97500100E780803D9DB70347D8
:1094D0009100A207D98F35671307D7556385E70831
:1094E0006368F7022D671307B7556387E70631678F
:1094F0001307C755638AE70429671307A7556394C1
:10950000E702A285280097D0FFFFE78080B815B753
:1095100039679306E765638DD70663E9F60013079D
:10952000E7556380E706A28528003DB73D679306AF
:10953000F7556386D7061307F766E396E7FE97D0DD
:10954000FFFFE78000D1F5B50146A285280097D03E
:10955000FFFFE78040A1F1BDA285280097D0FFFF63
:10956000E78060B1F9B58947E3F587EC9305E4FF3F
:10957000C205C1811305A10097A0FFFFE780C0C409
:109580004DBDA285280097D0FFFFE78080B155B57B
:10959000A285280097D0FFFFE78040BC59BD97D037
:1095A000FFFFE780C0C471B5411122C417A4FF1F9B
:1095B000130484E7AA86178601001306E6112285A4
:1095C000C14506C697500100E780A04603574400F6
:1095D00097A7FF1F938747E62393E700035764008D
:1095E0002394E700B240224441018280411106C623
:1095F00097000000E78080FBB7E7040083A787148B
:1096000017A6FF1F130646E2D54501458297B240D3
:109610004D4697A5FF1F938525E213057030410144
:1096200017030000670003A261712324811A37E445
:109630000400832704082326111A2322911A2320C9
:10964000211B232E311917050000130585A68297CB
:1096500017A9FF1F130909DC994785442300A900B6
:10966000231CF100978501009385050BE1471775D1
:109670000100130565D0231CF1082308910097C948
:10968000FF1F9389090997500100E780602183D566
:109690000900178501001305250797500100E78091
:1096A0002020294597500100E780602403D5090058
:1096B000896997000000E78060EF8327441710084E
:1096C00085451305503082978327441717A6FF1F3F
:1096D000130686D6CD45130570308297832744172D
:1096E00017A6FF1F130646D3B545130560308297B2
:1096F0008327441730088945130510318297832743
:109700004417300989451305203182978327441572
:10971000938509900D458297832744159385099079
:1097200011458297A305910023069100230891001B
:1097300002CD230C010083278416300991451305BF
:1097400070408297832784161306B1008545130560
:1097500000408297832784167000854513051040CA
:109760008297832784163008854513052040829709
:109770008327841610088545130550408297832758
:1097800004157D558297832744137D5582977D5517
:1097900097A0FFFFE78000EE8327440C829797A0F5
:1097A000FFFFE78040C98327841417A6FF1F130615
:1097B000A6C7D5450145829789471306700F814595
:1097C00028092306F1009790FFFFE780C0928D479C
:1097D0001306000881452808230CF1089790FFFF25
:1097E000E78060919147230CF10097770100938700
:1097F00027AA984383C747003AC8230AF10097D0A5
:10980000FFFFE78040B670008545054597A0FFFF44
:10981000E78060ED30099305700F094597A0FFFFC1
:10982000E78060EC3008930500080D4597A0FFFF26
:10983000E78060EB10089545114597A0FFFFE78092
:1098400080EAC16717C7FF1F1307C73FF9171CC37B
:109850002322070017A5FF1F130585BB97A0FFFF55
:10986000E78040E78327C41D17C5FF1F1305053C8C
:1098700082973C4803450900854582978320C11A99
:109880000324811A8324411A0329011A8329C11947
:109890005D618280C16717C8FF1F0358A83AF91796
:1098A0006301F8083DCDB5CD011126CAB7E4040027
:1098B00083A7841222CC2E862315B10006CE2A84DB
:1098C00001478146ED45428582972AC611ED1785ED
:1098D0000100130565E597500100E7804014F24050
:1098E0006244D24405618280FC440356A100A285F3
:1098F00082972C0017C5FF1F0355C53497A0FFFFA3
:10990000E78000EA69DD17850100130525E397501C
:109910000100E780C01083A7C412ED45280082979C
:109920007DBF8280411106C61DC9854717A7FF1F4D
:10993000A309F7AE354697A5FF1F9385E5AD13053F
:10994000603097A7FF1F238F07AC97F0FFFFE780DA
:10995000606FB240410117F3FFFF6700636997A78B
:10996000FF1FA38007ACF9B7C16717C5FF1F0355D9
:10997000652DF9176307F500B7E7040003A3C717C0
:1099800002838280854717C7FF1F230BF72A0145F3
:1099900017F3FFFF670043631783FFFFE7020371BD
:1099A0002A8408452E89B28919C900C1971500007B
:1099B0009385A586610597300100E7808001814489
:1099C0007D5A97100000E780E03963C7A404814402
:1099D00097100000E780003A63C8A40497C7FF1FF0
:1099E0009387C7269C43DC47B307F940918723023E
:1099F000F400638309048327C900B307F440958703
:109A0000A302F4001C4C89C79C4799C32285829706
:109A10001783FFFF6700C36C5C4413971400850431
:109A2000BA972390470171BF1C481397140085040F
:109A3000BA972390070069BF832789000547B307BA
:109A4000F4409587A302F40083570400638EE70275
:109A50008DC309476384E7040D47E395E7FA9787C9
:109A600001009387E72F1CCC97870100938747302D
:109A700011A897870100938727F61CCC97870100D0
:109A8000938787F65CC8BDBF978701009387C7E1BE
:109A90001CCC97870100938727E2EDB797870100D9
:109AA0009387C7301CCC9787010093872731D9BF94
:109AB00095E51783FFFFE7020361004618448347DB
:109AC000940075839D8B6317F70097100000E78063
:109AD00060B448C41783FFFF670023618280178347
:109AE000FFFFE702A35C13893500C16442094111FD
:109AF000AA890144F11413590901054A2EC6971089
:109B00000000E7802026B2456348A40001454101DA
:109B10001783FFFF6700C35C83A7090013171400B6
:109B2000BA9783D707006388B7006394970063747C
:109B30002A010504E1B70545D9BF1783FFFFE702F6
:109B40000356AA892E89328BB6843A8ABE8A97A098
:109B50000000E78020FB71C9268597200000E78080
:109B600020098D4763E7A7007D551783FFFF670036
:109B7000835683DB440097100000E780A0242A84EA
:109B800097100000E78040259307740031443305A7
:109B9000850263CDA70297100000E780A0229710EE
:109BA0000000E78020222A8497100000E780C0226E
:109BB0009307740031443305850263C3A7049710EB
:109BC0000000E78020209307450029A89710000097
:109BD000E7808020330585021307F0179307C0172D
:109BE000E35FA7FA2D55E3C277F963040B02D6862B
:109BF0005286A6854A8597200100E78020BAB5B72E
:109C000097100000E780401D330585029307C5FFCC
:109C1000D1BF832749001385C90083D5270097004A
:109C20000000E78000EC61F581B769553DBF97C73B
:109C3000FF1F239FA70097C7FF1F9387270190430C
:109C400081470C463307F500420741836393B70011
:109C500082805446139847008507C2962390E600F9
:109C6000D5B797C7FF1F938767FE9C4303C587003F
:109C7000828017C5FF1F0355A5FD82801783FFFF54
:109C8000E7026344C1671387D7FF630BE502636A8A
:109C9000A700F1176300F50201451783FFFF670076
:109CA000C3441387E7FF6302E502FD171D8D1335DB
:109CB0001500E5B797500000E780C0267D15C5BFA9
:109CC00097500000E78040FBD5BF97500000E78029
:109CD00060F9EDB71783FFFFE702E33E4111AA8465
:109CE00001442EC697100000E780C008B2456348C3
:109CF000A400014541011783FFFF6700033F9C4813
:109D0000131514003E9583570500E385B7FE05043F
:109D1000C9BF03485500814693F7F60F63E5070175
:109D200081473E858280584593975600BA9703D75E
:109D300027006316B70003D70700E304C7FE8506B4
:109D4000E1BF8346450001479377F70F63E4D700EF
:109D5000814711A81C45131657000507B29703D673
:109D60000700E313B6FE3E8582801783FFFFE702FC
:109D7000E33393170501C18797CAFF1F938A0AED42
:109D8000635BF00883A70A00C0479C4703570400A1
:109D9000198D420541816368F500014422851783CE
:109DA000FFFF6700E33312052A94CDBFDC4713940D
:109DB0004900014A3E94834744006341FA02014A44
:109DC000834754006349FA028509C20993D90901FE
:109DD00083A70A009847E3EBE9FCC1B71C441319B9
:109DE0005A00A6853E994A8597000000E780C0EE9C
:109DF00005E1050AC9B75C4413195A00A6853E99C6
:109E00004A8597000000E78020ED19E1050A4DBF63
:109E1000E30C09FA61B7AA8481495DBF1783FFFF8C
:109E2000E702632A1C452A8481E79307C5001CC505
:109E30001C44231204001CC09307F00F63EDB7000D
:109E400093F5F50F228597200000E78020E2178325
:109E5000FFFF6700832993940501C167C18063F9FF
:109E6000F500A685228597200000E78040E5C5B76C
:109E7000C18193F5F50F228597200000E78000DF70
:109E8000A685228597200000E78040E0C9B797C7E4
:109E9000FF1F9387A7DB884382801C4599C797C71C
:109EA000FF1F23A5A7DA014582807D55828097C7D1
:109EB000FF1F9387A7D998438347450048479207D8
:109EC0003E9582801783FFFFE702E31F6171004523
:109ED0001C183EC6B70780013EC81C183ECA8357EF
:109EE000440002CE02D002CC231EF100834784003E
:109EF0002A8902D22301F1023C083ED402D69700FF
:109F00000000E78000FB835705002316F1029750FD
:109F10000000E78060C42307A1025C400355640091
:109F2000F18313F717008347F10252055181F99B22
:109F3000D98FA307F10297100100E780807539CD12
:109F4000AA840355050097A00000E78080BC83D752
:109F500004002AD26800231CF10083D72400231DAB
:109F6000F1001C4803D647008C4397200000E7808F
:109F700000CD8347B400CA86178601001306468CBD
:109F80008117A305F4006C00481097200100E780BA
:109F9000E0805D611783FFFF670023152155D5BF62
:109FA0001C45B1CF03C5A700894613576500630B55
:109FB000D7028D46630ED70285466300D70213078A
:109FC00040063305E50203C7B700418B15CB83C7B5
:109FD000B700BD8B3355F54082801375F503130729
:109FE000803EC5B709671375F50313070771D1BF25
:109FF000372709001375F5031307077CD9B7014507
:10A0000082801783FFFFE702030C03A98500630C1E
:10A0100009048347B900AE8493F7070E85C303454F
:10A020009900930520030D810505B305B502884409
:10A03000610597300100E780E0A935A02E859700E3
:10A040000000E78020F62A8419CD97000000E78001
:10A05000605C8325C900B307B54063FA87002E947E
:10A06000B305A440E9F51783FFFF670003088545A2
:10A070007DBF1783FFFFE70203052A8403D5050090
:10A08000011132C636C43AC22EC002CA02CC02CE78
:10A0900097A00000E780E0A782452ACA22852ECC3F
:10A0A00097000000E780E0E003570500231EE10071
:10A0B00097500000E78040AAA24632469247230FFD
:10A0C000A10036874C08B286228501469700000021
:10A0D000E780E0A605611783FFFF67000301178390
:10A0E000FFFFE70243FE61711C183EC6B7078001FF
:10A0F0003EC81C183ECA3C0800453ED4AA8402CC87
:10A1000002CE02D002D202D697000000E78060DAC9
:10A110008357050035592316F10297500000E78058
:10A12000A0A32307A10209C48357440081EB21594E
:10A130004A855D611783FFFF670023FB03556400B9
:10A140005205518197100100E780A0542A8965D1FA
:10A150008347B40093F7070E99C71305840197301E
:10A160000100E780609983574400231EF100834774
:10A1700084002301F1025C4003550900D98313F7E1
:10A18000070883471102231CA10093F7F707D98F13
:10A19000A300F10283572900231DF1005C40F183E5
:10A1A00013F717008347F102F99BD98FA307F10238
:10A1B00097A00000E780E0952AD235D98347940024
:10A1C0006800139757008347B400FD8BD98FA30510
:10A1D000F4001C4803D647008C4397200000E7801A
:10A1E00000A6A68717770100130787657400054648
:10A1F0004C10268597000000E78060942A890DD9CD
:10A200008347B400A685FD8BA305F40097000000EA
:10A21000E78060DF31BF1783FFFFE702C3EA8324D3
:10A2200085FE2A844111268597000000E78080D7AB
:10A23000834734FF93F7070E8DCB2AC626859700F8
:10A240000000E78060C809CD834734FFB245FD8B2D
:10A25000A309F4FE91C5228597300100E78080872D
:10A2600041011783FFFF670043E87DD98327C4FFBF
:10A270002685829775F5834734FF93F7070E91C7BC
:10A28000228597300100E7802087032584FE970010
:10A290000000E78000E5E9B71783FFFFE702A3DFCF
:10A2A0009C4141112A8903C7070089472E84935690
:10A2B00067006380F6040D466388C6049307F007C1
:10A2C0006304F7022E8597200000E780C0A7AA84C8
:10A2D0008149C16B130C490097C7FF1F93870797EC
:10A2E0009C43984763E4E90441011783FFFF67003B
:10A2F00043DE03D745008547E3F8E7FE2E85972028
:10A300000000E780A0A9E1B703D74500E3FEE7FC22
:10A310002E8597200000E78000A3AA84228597203D
:10A320000000E78060A4C204C98C5DB7DC47035518
:10A33000A900139A49003E9A93170501C187635DEE
:10A34000F00083570A006397A70263E7740383272B
:10A35000CA00034D5A002DA0A1672167A98F1307DA
:10A36000F7EFE374F7FE6397090097000000E780BA
:10A37000209161FD85098DB783278A00034D4A002E
:10A38000835DA90003576900216A138BC7003AC691
:10A39000814A33CA4D01631E5D0197C7FF1F938732
:10A3A000678B9C43E1DBA286628681452685829786
:10A3B000D1B7A1679387F7EF930C4BFF63F2470385
:10A3C000B2455A8597F0FFFFE780A0710DC10327C2
:10A3D0008B00104709CE10436382C4023107D5BFFA
:10A3E000EE85668597000000E780008F71F99386FF
:10A3F0001A0093FAF60F130B0B0271BF8356440039
:10A400005C43E3E9F6F622853AC697100000E78040
:10A41000807DA1679387D7042A8A035D4400324771
:10A4200063E897008347D90093E707F8A306F9008C
:10A430001C4766852286E2858297C1670844FD171E
:10A44000337AFA00529508C02312A40125B797B7B2
:10A45000FF1F9387A77F9843814715C31447814700
:10A4600063FFD500939745004C47BE9519C903C7B4
:10A47000550081476375E600DC451606B2973E85B8
:10A48000828003C745008147E37BE6FE16069C45B4
:10A49000F5B71783FFFFE70263C1AA892E8A8144BB
:10A4A00097BAFF1F938A8A7A83A70A00984763E6C0
:10A4B000E4001783FFFF6700A3C2DC471394440046
:10A4C00001493E9413BB140083474400634BF900D9
:10A4D000014913BB140083475400634FF9008504FE
:10A4E000E1B70844931759005287DA860146A285DE
:10A4F0003E9582990509C9BF484493175900528770
:10A50000DA860546A2853E9582990509E9B7178343
:10A51000FFFFE70243BB814517F5FFFF1305054821
:10A5200097B7FF1F2396077297000000E780A0F6F9
:10A530001783FFFF670063BB97B7FF1F9387077100
:10A540009C4395C31783FFFFE702E3B7814517F5E7
:10A55000FFFF1305A54497000000E780C0F31783B1
:10A56000FFFF670083B882801783FFFFE70203B411
:10A5700037E404008327841241112315E100AE89DA
:10A580003289368A3A8681460147ED45AA84829708
:10A590002AC621C90356A100D28597400100E78051
:10A5A000C0248327C413CE8526858297058905C9D3
:10A5B0008327440D2314210101462C002685829710
:10A5C0002A8401C9B7E7040083A7C712ED45280014
:10A5D0008297228541011783FFFF670063B04944DA
:10A5E000D5B76554FDB75C41FD175CC18280178308
:10A5F000FFFFE70243ADB7E70400FC5F8297954792
:10A600003305F50281450D811783FFFF6700E3AD38
:10A610001783FFFFE70223ABB7E70400FC5F8297D5
:10A6200095473305F5020D811783FFFF6700E3AB04
:10A630001783FFFFE70223A9B7E7040083A7870B6F
:10A640000355050082971783FFFF670003AA17834E
:10A65000FFFFE70243A7035505003287AE86179632
:10A66000FF1F035686E397B5FF1F9385E55E9700AE
:10A670000000E780A0EF1783FFFF670003A71783A1
:10A68000FFFFE70243A4B7E7040083A7C717829739
:10A690001783FFFF670063A51783FFFFE702A3A2ED
:10A6A000B7E7040083A7871397B5FF1F9385C55AA3
:10A6B000829701451783FFFF670023A31783FFFFDE
:10A6C000E70263A0B7E7040083A7C71F814517957A
:10A6D000FF1F035585D882971783FFFF6700E3A00C
:10A6E0001783FFFFE702239EB7E7040083A78713C2
:10A6F00097B5FF1F93854557829701451783FFFF45
:10A700006700A39E1783FFFFE702E39BB7E7040000
:10A7100083A7C71F81451795FF1F035505DA829749
:10A720001783FFFF6700639C1783FFFFE702A3996E
:10A730002E8597800000E780E0AF97800000E780DB
:10A74000E0EC1783FFFF6700439A1783FFFFE702E0
:10A75000839797800000E780E0F61783FFFF67008C
:10A76000C3985C49E1175CC95CC583572501A10703
:10A770002319F50083570501A1072318F5008280EE
:10A78000F1473305F50297B7FF1F9387E74F9C43C7
:10A790003E9582808D476315F60803D746008547AE
:10A7A00063F0E7081783FFFFE702E39136853684FD
:10A7B0002E8997100000E780005929C9835744006B
:10A7C00093140501C18063E397042285971000006C
:10A7D000E7806057FD14231294009307A0026300E2
:10A7E000F5029307B0026307F50293079002631F17
:10A7F000F500228597000100E780C08501A8014689
:10A80000CA85228597A00000E78060B01783FFFF0C
:10A810006700A38D228597100000E780C003FDB775
:10A82000828097B6FF1F938666469C42014599CF6A
:10A830009843D44217B6FF1F232AE6446396D700F5
:10A8400097B6FF1F23A6E6441385C7FE82801783B1
:10A85000FFFFE702438797000000E780A04B7144A9
:10A8600033058502914597900000E78020E911E5C6
:10A8700065551783FFFF6700438797B7FF1F23A323
:10A88000A74097000000E780E04833058502914526
:10A8900097900000E78080E661DD97B7FF1F23A552
:10A8A000A73E97000000E780E04697B7FF1F23957B
:10A8B000A73C97000000E780E04597B7FF1F239E65
:10A8C000A73A977701009387E7FC17B7FF1F232963
:10A8D000F73A97070000938707E917B7FF1F232F61
:10A8E000F738014579B71773FFFFE702C37DAA85E3
:10A8F00017B5FF1F1305453897100000E780C05BB0
:10A900001773FFFF6700637E1773FFFFE702A37BE8
:10A9100097000000E78060FD97100000E780405B33
:10A9200097B7FF1F938787369C4391CF1387C7FE46
:10A9300019CB83D5C7FF17B5FF1F1305A535972082
:10A940000100E78020191773FFFF6700037A177370
:10A95000FFFFE702437797000000E780C0EC09CDD6
:10A96000834785002A8493F7070499EB0355E50094
:10A9700097000000E78080F91773FFFF6700E37618
:10A980008347C5009304450117B9FF1F1309093018
:10A9900085E3832709005CC997B7FF1F23A8972E7B
:10A9A00083274900F1FB97B7FF1F23A3972EE9B731
:10A9B000FD172306F500610597800000E780C0D6EB
:10A9C0008307840063CB07048347840093E707F879
:10A9D0002304F400B7E704009C5F82974205A9476F
:10A9E00041813375F5028347840093F707FCC98FD3
:10A9F0002304F4008347D4003E951C402318A40090
:10AA000089CF984319CB8347C400504081458507BF
:10AA10003305F502420541810297832709005CC88E
:10AA200097B7FF1F23A497268327490089E797B785
:10AA3000FF1F23AF97248347C4009DDF8355040184
:10AA400017B5FF1F1305052597200100E780800833
:10AA500025B71773FFFFE702036797B7FF1F9387B9
:10AA6000A7489C4701448583858B85E3AE84B285E6
:10AA70003A8697100000E780804B2A8419C597100A
:10AA80000000E780C041829408CC22851773FFFF45
:10AA90006700A3651773FFFFE702436141112E8929
:10AAA00032C6AA8997000000E780C03132471306FA
:10AAB0000502CA86970500009385C5CC17B5FF1F10
:10AAC0001305851B97000000E780E0F82A8425C95C
:10AAD0009304C50097000000E780E0411946AA856D
:10AAE000268597100000E7808015854526859710FC
:10AAF0000000E780601117750100130565D74E95BA
:10AB000083450500268597100000E78020165C48E5
:10AB100031468145A1075CC85CC483572401E11715
:10AB20002319F40083570401E1172318F4001C4C87
:10AB30003E859770FFFFE780005CA3042501228516
:10AB400041011773FFFF6700A3591773FFFFE70267
:10AB500083574111AA842EC632C497100000E780A3
:10AB60006036004DB2452246834784000CC050C079
:10AB700093F7F70393E707042304F4002318040072
:10AB8000268597100000E780803183479400A9460E
:10AB90002317A40013D7370005073307D7029D8B6F
:10ABA00085072306F400A306E40083C70401D84800
:10ABB0008507230FF7FE17B7FF1F1307270D58430D
:10ABC000232A04009307440129E317B7FF1F232119
:10ABD000F70C17B7FF1F232BF70A17B4FF1F130437
:10ABE000640B228597200100E78000E11C44858BDF
:10ABF0005D8D19E58145228597200100E78080ED74
:10AC000041011773FFFF6700434E1CC317B7FF1FB7
:10AC10002320F708D9B71773FFFFE702C34A970548
:10AC20000000938565B7014597000000E78000B0FC
:10AC300001451773FFFF6700434B1773FFFFE702E0
:10AC4000834897000000E78080B01773FFFF67001C
:10AC5000C3498347C500A5E31773FFFFE702A34677
:10AC60002A840355E50097000000E78000C821C151
:10AC70008347840093F7F7FB2304F4001C4091C73B
:10AC8000DC4381C74C400145829797000000E78074
:10AC900080B917B5FF1F1305E5FF97200100E78076
:10ACA000A0E50355E40097000000E78020C6177375
:10ACB000FFFF6700834382801773FFFFE702A34013
:10ACC00097B7FF1F938787FC97050000938565C89A
:10ACD00017B5FF1F130505FC23A0070023A20700DB
:10ACE00097200100E780E0CE1773FFFF6700E33F86
:10ACF0001C4D91CFDC4381CF1773FFFFE702A33CCC
:10AD00008345070082971773FFFF6700033E828029
:10AD100097B7FF1F938747FA9C4303C507008280BC
:10AD200097B7FF1F938747F99C4303C5170082809D
:10AD300097B7FF1F938747F89C4303C5270082807E
:10AD400097B7FF1F938747F79C4303C5470082804F
:10AD500097B7FF1F938747F69C4303C53700828050
:10AD600097B7FF1F938747F59C4303C55700828021
:10AD700097B7FF1F938747F49C4303C56700828002
:10AD800097B7FF1F938747F39C4303C577008280E3
:10AD900097B7FF1F938747F29C4303C587008280C4
:10ADA00097B7FF1F938747F19C4303C597008280A5
:10ADB00097B7FF1F938747F09C4303C5A700828086
:10ADC00097B7FF1F938747EF9C4303C5B70011E177
:10ADD0001D45828097B7FF1F938707EE9C4303C5ED
:10ADE000C700828097B7FF1F938707ED9C4303C579
:10ADF000D700828097B7FF1F938707EC9C4303C55A
:10AE0000E700828097B7FF1F938707EB9C4303D52A
:10AE10000701828097B7FF1F938707EA9C4303C50A
:10AE20002701828097B7FF1F938707E99C4303D5CB
:10AE30004701828097B7FF1F938707E89C4303D59C
:10AE40006701828097B7FF1F938707E79C4303D56D
:10AE50008701828097B7FF1F938707E69C4303C54E
:10AE6000A701828097B7FF1F938707E59C4303C51F
:10AE7000B701828097B7FF1F938707E49C4303C500
:10AE8000C701828097B7FF1F938707E39C4303C5E1
:10AE9000D701828097B7FF1F938707E29C438857AB
:10AEA000828097B7FF1F938727E19C4303D5C70292
:10AEB000828097B7FF1F938727E09C4303D5E70263
:10AEC00019E11305800C828097B7FF1F9387C7DEB7
:10AED0009C4303C50703828097B7FF1F9387C7DD95
:10AEE0009C43C85B828097B7FF1F938767DC8843CA
:10AEF000828097B7FF1F9387E7DB8843828019E141
:10AF00007D558280F5DE984265DFFDD917B7FF1FBA
:10AF1000130787FD1847AA877155058B631D072402
:10AF200003C507001547E37DA7FC03C737001305DA
:10AF3000F0057D171377F70FE364E5FC03C35700B3
:10AF4000E30003FC83C86700E38C08FA03C77700BB
:10AF5000494579171377F70FE364E5FA03C7A700AC
:10AF600011481305F7FF1375F50FE36BA8F803CE2F
:10AF700097000D481305FEFF1375F50FE362A8F85F
:10AF800003C8B7006309080065181378F80F1305A4
:10AF9000600DE36705F703C5C70079487915137598
:10AFA000F50FE36FA8F403C8D7000D457D1813789B
:10AFB000F80FE36705F503D80701930E4017511802
:10AFC000420813580801E3ED0EF303C8E7007D18AB
:10AFD0001378F80FE36605F303C827017D1813788B
:10AFE000F80FE36F05F103C88700C54E7518137895
:10AFF000F80FE3E70EF103D86701856E938EBEE08C
:10B000006D18420813580801E3EC0EEF03D847010E
:10B010006D18420813580801E3E40EEF03D88701C6
:10B020007918420813580801E36C05ED03C8A7011D
:10B030007D181378F80FE36505ED03C5B7011D48CA
:10B040007D151375F50FE36DA8EA03C5D7017148A7
:10B0500079151375F50FE365A8EA03D5E701130821
:10B06000E00F7D1542054181E36CA8E803C50702A6
:10B07000494879151375F50FE364A8E8C85301C969
:10B0800037C834005915130858BFE36BA8E603A866
:10B09000870237C53400130555BF5918E36205E729
:10B0A00017B5FF1F2328C5C003C6050117B5FF1F2D
:10B0B0002324F5C00545E375C5E403D82501D0492F
:10B0C00033760603E31E06E203C61501E30A06E231
:10B0D00017B6FF1F232EB6BC83C527000146638722
:10B0E000A50003C61700F1453306B60283C7070360
:10B0F0009305C00272971A071307C70516031A971C
:10B1000096084697B387B70241553E973297420754
:10B1100041836362E8061773FFFFE702C3FA3685CF
:10B1200097800000E780A06897000100E780204832
:10B130002A8497A00000E780805A2A9497F00000A4
:10B14000E78060262A9497900000E780A0812A94E7
:10B1500097F0FFFFE780E06F2A9497400000E780B8
:10B1600060932A9497700000E780A09C2295177343
:10B17000FFFF670083F782801773FFFFE702A3F4E6
:10B180004111A307A10097A00000E780A0C5930587
:10B19000F100170500001305E5B597F0FFFFE78004
:10B1A000802F014541011773FFFF670003F41773F8
:10B1B000FFFFE702C3EE17B4FF1F1304E4D2032816
:10B1C000840079599368180097B4FF1F23A214D301
:10B1D0001378180063100802BA84BE89368B328A4D
:10B1E0002E89AA8A97F0FFFFE780E0A77D152695B4
:10B1F00019E531594A851773FFFF6700C3ED97F0D2
:10B20000FFFFE78040A67D152695A167E353F5FE75
:10B2100097B7FF1F9387070498433E8C814B01CB60
:10B22000014597F00000E7802044933B15004A85D4
:10B23000DA865686D28597900000E780C04D2A892D
:10B2400011CD1C44F99B17B7FF1F2323F7CA83278F
:10B250000C00CDD3E3800BFA829769BF268597B7A0
:10B26000FF1F23A507C897F0FFFFE780809C41469A
:10B27000CE8517B5FF1F1305A5D097300100E780D5
:10B28000C05697D00000E78040990325040B97D063
:10B290000000E780009D054597D00000E78000A4EE
:10B2A000054597000000E78060EDA9B797B7FF1F3D
:10B2B000938787C39C47858BEDC71773FFFFE70212
:10B2C00083E017B5FF1F1305E5C997B7FF1F23AD2F
:10B2D00007C097B7FF1F23AB07C097B7FF1F23A96E
:10B2E00007C097200100E780208197500000E78089
:10B2F000E0F597100100E780A04C97100100E7806F
:10B30000A05297B7FF1F9387A7BC9C4391C70545E1
:10B3100097800000E780402097B7FF1F938707A51D
:10B320009C4399C741657D1597700000E78040A256
:10B3300097F00000E780E03D97D00000E780808F25
:10B3400097B7FF1F938707CF9C4313971701635647
:10B35000070097F00000E78000AD97B7FF1F23A11B
:10B3600007C297B7FF1F23AF07C097B7FF1F23ADD3
:10B3700007C097B7FF1F23AB07C097000000E78007
:10B38000008C97000000E780007297F0FFFFE780D5
:10B39000401897F00000E78040D61773FFFF670062
:10B3A000C3D4828097B7FF1F938707B488438280F6
:10B3B0001773FFFFE70223D197800000E7806075D5
:10B3C00097800000E780C0771773FFFF6700E3D125
:10B3D0001773FFFFE70283CD2A849304140201113F
:10B3E0002E85B289A685214636C63A899730010056
:10B3F000E780403D0DE9B24638082686CE85130524
:10B40000940497500000E780604121462C084A854B
:10B4100097300100E780003B133515000561177375
:10B42000FFFF6700E3CB0145D5BF1773FFFFE702BE
:10B4300083C99305450617B5FF1F13052588971087
:10B440000100E78020691773FFFF670003CA1773C5
:10B45000FFFFE70243C741112EC697F0FFFFE780C9
:10B46000601BB24588C141011773FFFF6700E3C746
:10B470001773FFFFE70283C3AA842E84978000001E
:10B48000E780006CAA898545228597000000E78047
:10B49000E07D83C7E4011389940899E313890403C9
:10B4A000CE85228597000000E780407C21469305E9
:10B4B0001902228597000000E780607897B7FF1F88
:10B4C000938787A28C43228597100000E780C08273
:10B4D000214693858402228597000000E78020762C
:10B4E0001773FFFF6700C3BF1773FFFFE70223BB9C
:10B4F000397197F00000E780E0B49305400661E9F8
:10B5000097800000E78000606302051497A7FF1F83
:10B5100083C7877C13B7170097A6FF1F238EE67A91
:10B52000014499CFC16417B9FF1F1309E99B93091F
:10B53000400EFD1497000000E780C0866342A40A15
:10B5400097F0FFFFE780000D4169B7290900096AFC
:10B55000FD7A2A8B81447D199389F97B130A0A713C
:10B56000938A8AC797000000E780C08363D7A4044A
:10B570001304400EB387840217B7FF1F1307C79643
:10B580000324070B3E948357C4016382270B1840A2
:10B590003307EB4063EAE900834744008507B3873C
:10B5A0004703D6976365F70801468145094597F03B
:10B5B000FFFFE780604EAA8B29E597400000E780F7
:10B5C000808385476317F50689659385057117A5FF
:10B5D000FF1F1305A56E97100100E780A04F95A0EF
:10B5E000B30734030327090BBA9703D7C7016308CE
:10B5F000970003C75700A38207002382E7000504D2
:10B6000015BF9305C500228597000000E78080E6FE
:10B610005E852286976501009385C52697F0FFFF1A
:10B62000E780E0525E8597100000E780608A85041D
:10B6300015BF97B7FF1F9387278B9C478D83858BFB
:10B64000C1F721611773FFFF6700E3A80146854535
:10B65000094502D002D202D402D697F0FFFFE7805C
:10B66000A043AA8479DD97F00000E780E09C13896D
:10B67000C4002A8481454A8597000000E780005F66
:10B680000C4041464A8597000000E780405B8329D3
:10B6900044006385090C4E8502D802DA02DC02DE22
:10B6A00097300100E78060402ACE141005462C0830
:10B6B00008184ECC97500000E780E00A1375F50F8C
:10B6C00051ED8355840093E525004A8597000000DD
:10B6D000E780E05E11460C104A8597000000E78085
:10B6E00000560146976501009385451A268597F017
:10B6F000FFFFE780C045268597000000E780407D7A
:10B700005C40A1D3014685450D4597F0FFFFE780DA
:10B71000A038AA841DD548401389C4009730010081
:10B72000E780A0382AC64A8597000000E780404C91
:10B730003246636FC5004C404A8597000000E780A1
:10B74000005001468145268597F0FFFFE7802040A5
:10B75000268597000000E780A077E5B58355840033
:10B76000ADB71773FFFFE702039697A7FF1F9387F5
:10B77000A7779C471DC193E7870017A5FF1F1305F7
:10B78000E55317A7FF1F2325F77697100100E780E1
:10B7900040321773FFFF67004395DD9B17A7FF1F1C
:10B7A0002328F77497300000E780E0647DF117A547
:10B7B000FF1F1305A55097100100E780E033D1BFAC
:10B7C0001773FFFFE702A38D4169AA892E8AB28A07
:10B7D000368BBA8B814417ACFF1F130CEC70930CA3
:10B7E000400E7D1997F0FFFFE780C05B63C4A400A3
:10B7F00001443DA03384940383270C0B3E9483576C
:10B80000C401638627055A87D6865286CE851305DE
:10B81000040397000000E780E0BB01C923800B0010
:10B8200022851773FFFF6700038B8347F40185C3ED
:10B830005A87D6865286CE85130594089700000055
:10B84000E78040B909C585472380FB00D1BF850447
:10B8500051BF835745006380071E1773FFFFE70240
:10B86000E38401112A8497000000E780C04D09C9D4
:10B8700085476309F50605611773FFFF6700438677
:10B8800097E00000E780007C7DF58357440049473E
:10B89000ED9BE392E7FEC145228597000000E7801B
:10B8A0004033AA84228597000000E780204F035789
:10B8B000440002CE91472A89631AF7002285970037
:10B8C0000000E780A0513C082ACC3ECE97E0000063
:10B8D000E78080765C55C5D374084A86A685054501
:10B8E000829751BF03574400D147E3F6E7F8032A94
:10B8F0000400C169014997AAFF1F938AEA5E130BEE
:10B90000400EFD1997F0FFFFE780C049634FA90E75
:10B910002285032A040097000000E780C042A14569
:10B920002A89228597000000E780A02AAA84228520
:10B9300097000000E780804A14402A86AA89780888
:10B940002685CA8597000000E780C0E7AA8405D550
:10B9500003C7F40189476315F7008347C10181DFFD
:10B960005546D2851385640097300100E780E0E7F3
:10B97000014597800000E780C01901C583D7C40145
:10B98000A5E797A7FF1F938727569C479355190054
:10B99000858913D73700058B01CF8983858B639900
:10B9A000B70001452EC697000000E780C0DBB24516
:10B9B0004E8597800000E780601F0346C1012A84FE
:10B9C00093751900268597900000E780E03935C10E
:10B9D000268597800000E780E018268511C0014584
:10B9E00097800000E780004C97300000E780A0407F
:10B9F0008547E312F5E883C754001307F00FE38C83
:10BA0000E7E68507A382F400BDB5B304690383A705
:10BA10000A0BBE9483D7C401638B37015546D28588
:10BA20001385640097300100E780C0D955DD050912
:10BA3000D1BD5DD86DB782801763FFFFE702036752
:10BA400097800000E780000C05C1C164014417A97C
:10BA5000FF1F130969499309400EFD1497F0FFFF7A
:10BA6000E7804034634EA40017A5FF1F130505258A
:10BA700097100100E780E0031763FFFF670043664C
:10BA8000330534038327090B3E958357C50163882B
:10BA900097002312050097800000E780A00C0504A2
:10BAA00075BF97A7FF1F938727449C478D83858B7E
:10BAB0008DE31763FFFFE702036117A5FF1F13055F
:10BAC000E51F97100100E78020031763FFFF670061
:10BAD000C36182801763FFFFE702E35E9705000002
:10BAE0009385C5A017A5FF1F1305451D97100100DD
:10BAF000E78020EE1763FFFF6700235F1763FFFFF8
:10BB0000E702635C8841B7E70400BC5B05054205BA
:10BB10004181829709C585472300F5000505176314
:10BB2000FFFF6700835C83C7F5FF2E858507A38F22
:10BB3000F5FE828083C7F5FFFD1793F7F70FA38FFC
:10BB4000F5FE99EF1763FFFFE702E357B7E704003D
:10BB5000BC571385F5FF82971763FFFF6700E35813
:10BB600082801C41035745008D8FBA951CC123125A
:10BB7000B5003E85828093D78500A2051441DD8DF6
:10BB8000835745001387E6FF18C189072312F50084
:10BB900013D685004111238FB6FEA38FC6FE410147
:10BBA000828018419307F7FF1CC183574500850722
:10BBB0002312F500A30FB7FE8280835745008D8FB7
:10BBC0002312F5001C41BE950CC12E858280AA87E8
:10BBD00003D7470008410D8FAA952392E7008CC335
:10BBE0008280184108453305A7408280835745006D
:10BBF000035765001D8F1C4108453385A740330559
:10BC0000A74082801763FFFFE702E34B41112EC676
:10BC10002A8497000000E780A0FDB2456373B50059
:10BC200001A0835744000840BE952312B4003E95FE
:10BC300041011763FFFF6700434B1763FFFFE702F4
:10BC4000834841112E84B28532C697000000E780F8
:10BC5000A0FB3246A28597300100E78000B9410180
:10BC60001763FFFF670063481763FFFFE702A34501
:10BC70002E84854597000000E78000F923008500A9
:10BC80001763FFFF670063461763FFFFE702A343E5
:10BC900041112317B100894597000000E780C0F6E5
:10BCA0008347E1002300F5008347F100A300F5007E
:10BCB00041011763FFFF670043431763FFFFE7027C
:10BCC000834093D78500A2054111DD8D2317B10074
:10BCD000894597000000E78020F38347E1002300B7
:10BCE000F5008347F100A300F50041011763FFFF52
:10BCF0006700A33F1763FFFFE702E33C139785014B
:10BD000093D78501C166938606F0D98F13D7850036
:10BD1000758FD98FA2053707FF00F98D4111DD8D91
:10BD20002EC6914597000000E78000EE6C0011469A
:10BD300097300100E78060AB41011763FFFF6700A8
:10BD4000C33A1763FFFFE70203381C41854503C46C
:10BD5000070097000000E78080E622851763FFFF59
:10BD60006700A3381763FFFFE702E3351C41411169
:10BD7000894503C7070083C717002307E100A3070E
:10BD8000F10097000000E78080E30355E1004101E6
:10BD90001763FFFF670063351763FFFFE702A332F6
:10BDA0001C414111894503C7070083C717002307BA
:10BDB000E100A307F10097000000E78040E083570F
:10BDC000E100410113D58700A2075D8D4205418145
:10BDD0001763FFFF670063311763FFFFE702A32EBE
:10BDE0000C4141112A841146680097300100E78018
:10BDF000C09F9145228597000000E78040DCB24754
:10BE0000C166938606F01397870113D58701598D74
:10BE100013D78700758F598DA2073707FF00F98F59
:10BE20005D8D41011763FFFF6700232C1C45BE9504
:10BE30000CC18280AE87944391E6584101EF0CC15A
:10BE40005CC1828003C7570013671700A382E70015
:10BE5000B687D5B70CC3EDB7AA87084119CD1841ED
:10BE6000D44398C36313D500D8C32A870346570029
:10BE70009376160081E6232007008280944381CACE
:10BE80008C4203A847008CC363930601CCC3799A04
:10BE900014C3A302C7003687D1BF1C45DC471D8DE4
:10BEA000B777DBB6938777DB09853305F502420563
:10BEB00041818280F147B385F50248452E95828005
:10BEC0008347450085072302F50082801763FFFF43
:10BED000E702631F2A8409E41763FFFF6700E3207A
:10BEE00083474400F5DBFD1793F7F70F2302F400B7
:10BEF000E5F71C4403D7270005072391E700DC433F
:10BF000099C3228582974C4889CD83475400898BF9
:10BF100099E71C4422859C479C439C478297232A8F
:10BF200004000040232004007DB71763FFFFE702F1
:10BF300083198357250041112EC681EB01442285C8
:10BF400041011763FFFF6700431A0357050081474C
:10BF5000F146E305F7FEB385D702404585072E94E9
:10BF60008345440008C4F5F5B247AA8481E7232A33
:10BF7000040009A81C456C0022859C439C438297C1
:10BF800048C84DDD85472312F400B2472320040042
:10BF9000231804002319F4005C485CC483D72400F0
:10BFA000FD172391F40061BF1763FFFFE702A311A0
:10BFB00097A7FF1F938787D2884323260500232452
:10BFC0000500410597100100E78000B31763FFFFEC
:10BFD0006700A3111763FFFFE702E30E17A4FF1F1B
:10BFE0001304C4CF1C40411199CF9C472300B500D6
:10BFF0002AC65CC197000000E78040FB1C40DC4380
:10C0000099C33245829741011763FFFF6700E30D33
:10C010000347450029E3584DAA877D551DCF176377
:10C02000FFFFE702430A1CC3DC4797A6FF1F23A7B5
:10C03000E6CAF156130507012390D70097050000C3
:10C040009385050297100100E780A09801451763CA
:10C05000FFFF670083097D55828082801763FFFFA1
:10C06000E702630601116146814528009760FFFFE2
:10C07000E780600897A7FF1F938747C69C43280067
:10C080009305F00FDC473EC697000000E780C0F440
:10C0900005611763FFFF6700430597A7FF1F93879D
:10C0A000E7C39C43D847A1679387C702631EF70A7B
:10C0B000397106DE22DC26DA80004AD84ED652D408
:10C0C00056D23285B28497000000E780C0C7AA89A3
:10C0D000268597000000E78020C92318A4FC268548
:10C0E00097000000E78040C82319A4FC268597002C
:10C0F0000000E78060C783D744000A8A231AA4FCA3
:10C10000858393F7F70F230EF4FC8607BD0793F79B
:10C11000073F3301F1408A8A01498347C4FD6367C1
:10C12000F902CE85130584FC232C54FD97000000F2
:10C13000E78080EA5281130104FCF2506254D25429
:10C140004259B259225A925A21618280268597001B
:10C150000000E78060C193171900D6970509239066
:10C16000A7001379F90F55BF828097A7FF1F938708
:10C17000E7B69C43D847A1679387A702631AF70ADB
:10C18000397106DE22DC26DA80004AD84ED652D437
:10C1900056D23285B28497000000E780C0BAAA89DF
:10C1A000268597000000E78020BCFD572318A4FCDB
:10C1B00026852319F4FC97000000E780E0BA83D7B6
:10C1C00044000A8A231AA4FC858393F7F70F230EF1
:10C1D000F4FC8607BD0793F7073F3301F1408A8AD5
:10C1E00001498347C4FD6367F902CE85130584FCCA
:10C1F000232C54FD97000000E78000DE52811301DC
:10C2000004FCF2506254D2544259B259225A925A02
:10C2100021618280268597000000E780E0B49317B3
:10C220001900D69705092390A7001379F90F55BF78
:10C23000828097A7FF1F938767AA9C43D847A1676F
:10C2400089076310F70A397106DE22DC26DA8000DE
:10C250004AD84ED652D456D2328532899700000041
:10C26000E78060AEAA894A8597000000E780C0AFEA
:10C27000835749000A8A2318A4FC858393F7F70F94
:10C28000230CF4FC8607BD0793F7073F3301F14009
:10C290008A8A8144834784FD63E7F402CE851305CF
:10C2A00084FC232A54FD97000000E780E0D25281ED
:10C2B000130104FCF2506254D2544259B259225A2A
:10C2C000925A216182804A8597000000E780C0A9C8
:10C2D00093971400D69785042390A70093F4F40F46
:10C2E00055BF828097A7FF1F9387479F9C43D847DE
:10C2F000A1679387E704631EF70A397106DE22DC23
:10C3000026DA80004AD84ED652D456D23285B2842C
:10C3100097000000E78020A3AA89268597000000E7
:10C32000E78080A42318A4FC268597000000E780FE
:10C33000A0A3231AA4FC268597000000E780C0A2D2
:10C3400083D744000A8A2319A4FC858393F7F70F47
:10C35000230EF4FC8607BD0793F7073F3301F14036
:10C360008A8A01498347C4FD6367F902CE851305B4
:10C3700084FC232C54FD97000000E780E0C5528127
:10C38000130104FCF2506254D2544259B259225A59
:10C39000925A21618280268597000000E780C09C28
:10C3A00093171900D69705092390A7001379F90F61
:10C3B00055BF828097A7FF1F938747929C43D8471A
:10C3C000A1679387C704631AF70A397106DE22DC76
:10C3D00026DA80004AD84ED652D456D23285B2845C
:10C3E00097000000E7802096AA8926859700000024
:10C3F000E7808097FD572318A4FC2685231AF4FCB8
:10C4000097000000E780409683D744000A8A2319EA
:10C41000A4FC858393F7F70F230EF4FC8607BD0772
:10C4200093F7073F3301F1408A8A01498347C4FDEE
:10C430006367F902CE85130584FC232C54FD970015
:10C440000000E78060B95281130104FCF25062548D
:10C45000D2544259B259225A925A21618280268579
:10C4600097000000E780409093171900D6970509C0
:10C470002390A7001379F90F55BF828097A7FF1F5C
:10C480009387C7859C43D847A167DD076317F704E7
:10C490001763FFFFE70223C3797132853284970067
:10C4A0000000E780408A2AC6228597000000E780C6
:10C4B000A08B2311A102228597000000E780A088AD
:10C4C000B2452300A102280897000000E780C0B011
:10C4D00045611763FFFF670043C182809797FF1F85
:10C4E0009387C77F9C43D847A167938787046317C7
:10C4F000F7041763FFFFE70203BD797132853284C9
:10C5000097000000E78020842AC62285970000005B
:10C51000E78080852311A102228597000000E78033
:10C520008082B2452300A102280897000000E7801E
:10C53000A0AA45611763FFFF670023BB828097971E
:10C54000FF1F9387A7799C43D847A1679387A704C8
:10C550006312F7021763FFFFE702E3B60111280039
:10C56000814597000000E78020A705611763FFFF62
:10C570006700A3B782809797FF1F938727769C4316
:10C58000D847A167938757026319F7021763FFFF24
:10C59000E70263B30111328597F0FFFFE780A07ACD
:10C5A0002308A1008145280097000000E780C0A271
:10C5B00005611763FFFF670043B382809797FF1FF2
:10C5C0009387C7719C43D847A1679387E702631B92
:10C5D000F7041763FFFFE70203AF011132853284CE
:10C5E00097F0FFFFE7804078AA84228597F0FFFF4D
:10C5F000E7808077854709E9228597F0FFFFE7808C
:10C6000080744205B337A0002800814523189100AB
:10C610003ECA97000000E780209C05611763FFFF7A
:10C620006700A3AC82809797FF1F9387276B9C437B
:10C63000D84799476313F7081763FFFFE702A3A8DA
:10C6400079713285328497F0FFFFE780C06F2AC688
:10C65000228597F0FFFFE78020712310A102228539
:10C6600097F0FFFFE780206E2301A102228597F05B
:10C67000FFFFE780406DA301A102228597F0FFFF35
:10C68000E780606C2302A102228597F0FFFFE7801C
:10C69000806B2313A102228597F0FFFFE780A06A39
:10C6A000B2452314A102280897000000E780C09239
:10C6B00045611763FFFF670043A382809797FF1FC1
:10C6C0009387C7619C43D847A1679387C7036313C8
:10C6D000F7081763FFFFE702039F79713285328401
:10C6E00097F0FFFFE78020662AC6228597F0FFFFBC
:10C6F000E78080672310A102228597F0FFFFE78083
:10C70000A0662311A102228597F0FFFFE780A063B6
:10C710002302A102228597F0FFFFE780C062A302F7
:10C72000A102228597F0FFFFE780E0612303A102C9
:10C73000228597F0FFFFE7800061B245A303A102C5
:10C74000280897000000E780208945611763FFFFF4
:10C750006700A39982801763FFFFE702C396011168
:10C760002A8497F0FFFFE780005EAA84228597F075
:10C77000FFFFE780605F228597F0FFFFE780C05EE4
:10C78000035744008D4763F7E700228597F0FFFFCA
:10C79000E780805D228597F0FFFFE780E05C28005E
:10C7A000A68597000000E780208305611763FFFFDF
:10C7B0006700A3939797FF1F938747529C43D847DF
:10C7C000A167FD07631FF7001763FFFFE702A38F51
:10C7D000328597000000E78040F81763FFFF67008D
:10C7E000C39082809797FF1F9387474F9C43D847FA
:10C7F000A167E5076315F7081763FFFFE702A38C3E
:10C8000079713285328497F0FFFFE780C0532AC6E2
:10C81000228597F0FFFFE7802055228597F0FFFFE4
:10C82000E78080542310A102228597F0FFFFE78064
:10C83000A053520551812311A10222852302010236
:10C8400097F0FFFFE7802050A302A102228597F016
:10C85000FFFFE780404F2303A102228597F0FFFFEF
:10C86000E780604EB245A303A102280897F0FFFFBE
:10C87000E780807645611763FFFF6700038782804A
:10C880009797FF1F938787459C43D847A167938756
:10C89000E703631FF7001763FFFFE702C3823285D8
:10C8A00097000000E78060EB1763FFFF6700E383FA
:10C8B00082809797FF1F938767429C43D847A16761
:10C8C00093874704631EF7021753FFFFE702A37F16
:10C8D00079713285328497F0FFFFE780C0462AC61F
:10C8E000228597F0FFFFE7802048B245280897F09F
:10C8F000FFFFE780606E45611753FFFF6700E37E2F
:10C9000082809797FF1F9387673D9C43D847A16715
:10C91000938787026310F7041753FFFFE702A37A98
:10C9200079713285328497F0FFFFE780C0412AC6D3
:10C93000228597F0FFFFE7800041B2452300A10266
:10C94000280897F0FFFFE780206945611753FFFF34
:10C950006700A37982801753FFFFE702C3760111B6
:10C9600097F0FFFFE780203EAA85280097F0FFFFA1
:10C97000E780806605611753FFFF6700037797978D
:10C98000FF1F9387A7359C43D847A167D107631F33
:10C99000F7001753FFFFE70203733285970000008B
:10C9A000E780A0FB1753FFFF6700237482809797EF
:10C9B000FF1F9387A7329C43D847A167C507631F12
:10C9C000F7001753FFFFE70203703285970000005E
:10C9D000E780A0F81753FFFF6700237182809797C5
:10C9E000FF1F9387A72F9C43D847A167B907631FF1
:10C9F000F7001753FFFFE702036D32859700000031
:10CA0000E780A0F51753FFFF6700236E828097979A
:10CA1000FF1F9387A72C9C43D847A167AD07631FCF
:10CA2000F7001753FFFFE702036A32859700000003
:10CA3000E780A0F21753FFFF6700236B8280979770
:10CA4000FF1F9387A7299C43D84789476318F7029C
:10CA50001753FFFFE70223670111328532C897F0B1
:10CA6000FFFFE780402EAA85280097F0FFFFE780B0
:10CA7000A05605611753FFFF6700236782809797D1
:10CA8000FF1F9387A7259C43D847A1678D07631194
:10CA9000F7041753FFFFE702036301113285328465
:10CAA00097F0FFFFE780202A13066100AA844C005C
:10CAB000228597300000E780C0232800A68597F0E4
:10CAC000FFFFE780605105611753FFFF6700E361D7
:10CAD00082809797FF1F9387A7209C4381CFDC43D9
:10CAE00091CB1753FFFFE702035E82971753FFFFB7
:10CAF0006700A35F82801753FFFFE702C35C797171
:10CB00003C08AE843ED2A165B7070A002A843ED411
:10CB100048103C08DD053ED636C432C63AC297D02E
:10CB2000FFFFE780E02F12474810BA8597F0FFFF1C
:10CB3000E780C01332464810B28597F0FFFFE780C8
:10CB4000E014A2464810B68597F0FFFFE780001278
:10CB5000501001478146A685228597D0FFFFE780C8
:10CB6000805145611753FFFF670023581753FFFF9C
:10CB7000E702635501117C000329C501AE843ECA5A
:10CB8000A165B70707002A843ECC48087C00C5058C
:10CB90003ECE97D0FFFFE780A0288345D900480804
:10CBA00097F0FFFFE780800C500801478146A6857B
:10CBB000228597D0FFFFE780004C05611753FFFFE8
:10CBC0006700A3521753FFFFE702E34F83C79500A7
:10CBD00093F7F707A384F50097000000E78040F97A
:10CBE0001753FFFF670063501753FFFFE702A34D82
:10CBF00079713C08AE843ED2A165B70709002A844A
:10CC00003ED448103C08938545043ED632C636C40F
:10CC100097D0FFFFE780C020A2464810B68597F066
:10CC2000FFFFE780A00432464810B28597F0FFFF6F
:10CC3000E780C005501001478146A685228597D020
:10CC4000FFFFE780404345611753FFFF6700E3495B
:10CC50001753FFFFE702234783C7950041112A843A
:10CC600093F7F707A384F50032852EC697F0FFFFF0
:10CC7000E780800F85672AC46370F5029770000013
:10CC8000E78020E92246B24509ED11478146228519
:10CC900097000000E78060E641011753FFFF67003F
:10CCA000C34401478346F501DDB71753FFFFE70291
:10CCB000E33F01113C003ECAB7070A003ECC3C00EE
:10CCC0003ECE83C79500AA89328593F7F707A384E0
:10CCD000F5002E8497F0FFFFE78000098567637DEC
:10CCE000F504A165AA8493858504480897D0FFFFC1
:10CCF000E7800013268597700000E78080E12A898D
:10CD000029E19145480897F0FFFFE78020F6A685C6
:10CD1000480897F0FFFFE78060F7CA85480897F05A
:10CD2000FFFFE780A0F4014781465008A2854E85A9
:10CD300097D0FFFFE780203405611753FFFF67009E
:10CD4000233A8145480897F0FFFFE78020F2034926
:10CD5000090275BF1753FFFFE702433579711C10B5
:10CD60003ECAB7070F003ECC404D1C10AA84AE89C6
:10CD70004808994532C636893ECE97D0FFFFE780F6
:10CD8000200A32464808B28597F0FFFFE78000EEA0
:10CD9000630C0902A545480897F0FFFFE780C0E64D
:10CDA0002546CA8597200100E78020A45008014746
:10CDB0008146CE85268597D0FFFFE780C02B456151
:10CDC0001753FFFF6700C3318355C402480897F02B
:10CDD000FFFFE780A0EB0355E402814505C58547C9
:10CDE00085456301F502C167FD179305F00F630BDD
:10CDF000F5007D1597700000E780208E93051500E3
:10CE000093F5F50F480897F0FFFFE78020E683458C
:10CE10000403480897F0FFFFE78040E583451403CB
:10CE2000480897F0FFFFE78060E483552403480833
:10CE300097F0FFFFE78080E583554403480897F0AB
:10CE4000FFFFE780A0E49DB71753FFFFE702A3278A
:10CE500083C795008146014693F7F707A384F50041
:10CE600097000000E78040EF1753FFFF6700E327BC
:10CE70001753FFFFE702232579713E841C103ECA39
:10CE80002E89B7070F00A1653ECCFD051C10AA84B2
:10CE9000480842C03AC23ECE36C432C697D0FFFFE1
:10CEA000E78000F832464808B28597F0FFFFE78038
:10CEB000E0DBA2464808B68597F0FFFFE78000DD7B
:10CEC00012474808BA8597F0FFFFE78020DC024848
:10CED000630C08029145480897F0FFFFE780C0D235
:10CEE0001146A28597200100E78020905008014755
:10CEF0008146CA85268597D0FFFFE780C017456128
:10CF00001753FFFF6700631E8945480897F0FFFF2E
:10CF1000E78080CF834704002300F5008347140097
:10CF2000A300F500E1B71753FFFFE702231883C7FB
:10CF3000950001112A8A93F7F707A384F50032853B
:10CF4000AE8432C697F0FFFFE78000E232462A89BE
:10CF5000328597F0FFFFE78000DF85676373F90292
:10CF6000AA894A8597700000E780A0BA2A8419ED43
:10CF7000114781464A86A685528597000000E780C2
:10CF8000C0B705611753FFFF670083159387E9FF5B
:10CF900093F7F70F0547E366F7FE8347F50195EB37
:10CFA0008947E380F9FE8346F401528501474A86AA
:10CFB000A68597000000E78040B4A167D90748081C
:10CFC0003ECC230A010002CE97000000E780A0B00B
:10CFD0004DBF639EE7008947639EF90093071020C9
:10CFE000231FF50097700000E780C0B76DBF0947A9
:10CFF000E39BE7FA8D47E398F9FA228597700000E2
:10D00000E78080DF9797FF1F938787EC9C4399E722
:10D010009797FF1F938787D59C4399C703D5040033
:10D0200097800000E780A0CE231F040022855DBF0B
:10D030001753FFFFE702230901113C003ECAB7075F
:10D040000B003ECC3C003ECE83C795002A8932853A
:10D0500093F7F707A384F500AE8497F0FFFFE7800E
:10D06000A0D093170501C187635AF006A1652A84F1
:10D070009385E502480897D0FFFFE78060DAA28534
:10D08000480897F0FFFFE78060C09797FF1F9387DE
:10D09000E7CD9C43A9EB01449375F40F480897F042
:10D0A000FFFFE780A0BC9355844093F5F50F480837
:10D0B00097F0FFFFE78080BB9355044193F5F50F90
:10D0C000480897F0FFFFE78060BA014781465008A3
:10D0D000A6854A8597D0FFFFE780E0F905611753E1
:10D0E000FFFF67008300416585460546A2857D15E3
:10D0F00097500000E78060BD59DD510597000100A1
:10D10000E780808F130440063344850271B71753BC
:10D11000FFFFE70243FB0111B70706003EC683C7C6
:10D12000950021642A8993F7F707A384F500AE845C
:10D1300028009305A4040AC40AC897D0FFFFE7801B
:10D1400020CE300001478146A6854A8597D0FFFF53
:10D15000E78060F297E0FFFFE780801513049404F6
:10D16000480822CC230A010002CE97000000E78085
:10D17000809605611753FFFF670023F71753FFFFE2
:10D18000E702C3F2C1642A8901449799FF1F93897A
:10D19000A9D5130A8002FD1497E0FFFFE78080C144
:10D1A0006347A40001451753FFFF670063F3B3070C
:10D1B000440303A7C90ABA9703D707006306970079
:10D1C00083D72700638427010504F9B70545E1BF2C
:10D1D0001753FFFFE70283ED2A8A2E8999C123A006
:10D1E000050081498144979AFF1F938AAAAF614B3A
:10D1F00097E0FFFFE78040C263C7A4004E85175346
:10D20000FFFF6700E3ED3384640383A70A003E94C5
:10D210008357040099E763040900232089008504EB
:10D22000C1BF4146D2851305440097100100E78035
:10D23000605975F5A289E5B71753FFFFE70203E7C9
:10D2400039717C083ED4B7070A003ED67C083ED828
:10D2500083C795002A8A328593F7F707A384F500E0
:10D260002E8932C697F0FFFFE78000B085676373B1
:10D27000F5083246AA84328597F0FFFFE780A0AC1C
:10D280008547AA8963E8A706A165938585042810C8
:10D2900097D0FFFFE780C0B8268597700000E78031
:10D2A00040872A8429ED9145281097F0FFFFE780F9
:10D2B000E09BA685281097F0FFFFE780209DCE8594
:10D2C000281097F0FFFFE780609A014781463010F1
:10D2D000CA85528597D0FFFFE780E0D9A167938781
:10D2E000770448183EDC230A010202DE97F0FFFFB4
:10D2F000E780607E21611753FFFF670063DE814591
:10D30000281097F0FFFFE7806096A685281097F019
:10D31000FFFFE780A0979797FF1F938767F39C43D2
:10D3200081CB22856389090097D00000E7804024E3
:10D330008345040271B797D00000E780C022CDBFBB
:10D340001753FFFFE70283D683C795004111AA89CF
:10D3500093F7F707A384F5003285AE84328A97F0FD
:10D36000FFFFE78060A08567637FF5022A899760E9
:10D370000000E780007A2A84914631C58347F50191
:10D3800005476387E70291C70D476366F704AD461B
:10D390001DA89305050303250A00414697100100C7
:10D3A000E78040420DE941011753FFFF670043D377
:10D3B0009305950803250A00414697100100E78070
:10D3C0006040814669F54A86A6854E859700000033
:10D3D000E780C081C9BF83250A00130594089770B0
:10D3E0000000E780A02919C1C146F1BF9797FF1F30
:10D3F000938707AE9C4399E79797FF1F93870797FB
:10D400009C4399C7228597800000E780208A69FDA8
:10D410008547A30FF400228597B00000E780608461
:10D42000228597600000E780E0734E8581464A863A
:10D43000A68597F0FFFFE780607BA167938757047D
:10D4400048003EC42302010002C697F0FFFFE780B8
:10D45000806891BF1753FFFFE70263C483C795003D
:10D460004111AA8993F7F707A384F50032852E8925
:10D47000B28A97F0FFFFE780208F85676374F50E0F
:10D48000AA8497600000E780C0682A840DED416B94
:10D49000014A979BFF1F938B2BA5130C400E7D1BFE
:10D4A00019A833048A0383A70B0B3E948357C40146
:10D4B00063836705050A97E0FFFFE780A08EE342DC
:10D4C000AAFE95460DA08357C50163969702930562
:10D4D000050303A50A00414697100100E780802E4E
:10D4E000994611E181462686CA854E8597F0FFFF51
:10D4F000E780C06F85A883A50A0013050403977011
:10D500000000E780A017C14679FD2285231E940004
:10D5100097A00000E780E074228597600000E78014
:10D5200060649797FF1F9387A7D29C43A9C32300EA
:10D530000402228597D00000E78040F04E858146A6
:10D540002686CA8597F0FFFFE780406AA167938728
:10D55000070448003EC42302010002C697F0FFFF03
:10D56000E780605741011753FFFF6700C3B6894743
:10D570002300F402E1B7397106DE22DC4AD88000CC
:10D5800052D456D25AD026DA4ED65ECE2E8A328960
:10D590002A8B97D0FFFFE780E07D06057105419952
:10D5A0008A8A3301A140232224FC231404FC97D04F
:10D5B000FFFFE780207C83479A000605350593F737
:10D5C000F7072315A4FCA304FA004A85232624FCAC
:10D5D00097E0FFFFE780407993170501C18763401B
:10D5E000F0025681130104FCF2506254D2544259A5
:10D5F000B259225A925A025BF24B21618280AA846C
:10D600004A8597E0FFFFE7802076AA894A8597E060
:10D61000FFFFE7806075A1659385C5022A89130520
:10D6200044FC97C0FFFFE780A07F268597C0FFFFDF
:10D63000E780E073854511C94A86CE8597C0FFFF14
:10D64000E780606DAA8B21E98945130544FC97E0CA
:10D65000FFFFE780A061A685130544FC97E0FFFF6C
:10D66000E780C062CE85130544FC97E0FFFFE780AA
:10D67000E061CA85130544FC97E0FFFFE780006185
:10D6800001478146130644FCD2855A8597D0FFFF97
:10D69000E780609EB9B78145130544FC97E0FFFF22
:10D6A000E780C05CA685130544FC97E0FFFFE78098
:10D6B000E05DCE85130544FC97E0FFFFE780005D49
:10D6C000CA85130544FC97E0FFFFE780205C814496
:10D6D00097D0FFFFE780006AE3D4A4FA83A70B0189
:10D6E00013971400BA9783D5070099C5130544FC16
:10D6F00097E0FFFFE78080598504D9BF797106D68E
:10D7000022D44AD000184ECE52CC56CA26D25AC87D
:10D71000AE893289AA8A97D0FFFFE780A065060507
:10D72000690541990A8A3301A140232A24FC231C5C
:10D7300004FC97D0FFFFE780E06383C799000605EC
:10D740002D0593F7F707231DA4FCA384F9004A8550
:10D75000232E24FC97E0FFFFE7800061931705016B
:10D76000C187634FF0005281130104FDB25022546F
:10D7700092540259F249624AD24A424B4561828030
:10D78000AA844A8597E0FFFFE780005EA165938544
:10D79000A5022A89130544FD97C0FFFFE780406872
:10D7A000268597C0FFFFE780805C854509C9CA854B
:10D7B00097C0FFFFE78020592A8B29E1894513058F
:10D7C00044FD97E0FFFFE780604AA685130544FD0E
:10D7D00097E0FFFFE780804BCA85130544FD97E083
:10D7E000FFFFE780A04A01478146130644FDCE852E
:10D7F000568597D0FFFFE7800088B5B781451305B0
:10D8000044FD97E0FFFFE7806046A685130544FDD1
:10D8100097E0FFFFE7808047CA85130544FD97E046
:10D82000FFFFE780A046814497D0FFFFE780805448
:10D83000E3DBA4FA83270B0113971400BA9783D56F
:10D84000070099C5130544FD97E0FFFFE7800044FA
:10D850008504D9BF1753FFFFE702E38683474500DE
:10D86000404DD5EFFD575DC483469400094763637F
:10D87000D70A0346B400854663EEC6088306E40073
:10D8800063CA06085C45F9562390D7009787FF1FA7
:10D8900083C7874599E3A304E4009787FF1F938715
:10D8A000E74C9C4381E78947A306F4009797FF1F45
:10D8B0009387079A9C4381E789472306F4009705DD
:10D8C000000093854506AA841305040197F0000023
:10D8D000E7802010FD57231AF40281471CDC014821
:10D8E0009787FF1F23AE873E9787FF1F9387873F4A
:10D8F000232E040304C0804397D0FFFFE780C0516C
:10D9000061463306C502814522859740FFFFE780C7
:10D91000807E81473E851743FFFF6700037DFD57EB
:10D92000D5BF1743FFFFE702037A2A840355450258
:10D9300097600000E780E01D19E5231E04001743EF
:10D94000FFFF6700837A8357E401F5DB930504FF4B
:10D95000174501001305452D97E00000E780E0140E
:10D96000F9BF1743FFFFE70203762E89A165411136
:10D970009385E5032A8436C432C6BE843AC297C072
:10D98000FFFFE780E04912472285BA8597E0FFFF55
:10D99000E780C02D32462285B28597E0FFFFE78001
:10D9A000E02EA2462285B68597E0FFFFE780002E95
:10D9B000630309029145228597E0FFFFE780C024B9
:10D9C0001146A68597100100E78020E24101174328
:10D9D000FFFF670083718945228597E0FFFFE7809D
:10D9E000A02283C704002300F50083C71400A3000E
:10D9F000F500E9BF1743FFFFE702E36C83C795001B
:10DA0000444D054793F7F707A384F5001C424111E5
:10DA100083C707006367F7062E842A89B1C003C74E
:10DA2000D400630FF7021787FF1F1307273418432B
:10DA300005C3A386F40097A00000E780404A83C78F
:10DA4000D40099E741657D1597400000E78040309C
:10DA500083D72403918B89C797E00000E780C01328
:10DA60004A85A28597F0FFFFE7808010A167C10774
:10DA700048003EC42302010002C697F0FFFFE78082
:10DA8000800541011743FFFF670023661743FFFF2F
:10DA9000E702636303D745008D47AA8441112E84B2
:10DAA00032892E8563E3E70297E0FFFFE780C02B12
:10DAB000AA8523000900268597C0FFFFE780A028DC
:10DAC00041011743FFFF6700436297E0FFFFE780D4
:10DAD000A0292AC6228597E0FFFFE780E028B2450B
:10DAE00085472A862300F900268597C0FFFFE78037
:10DAF0008022F9B7397106DE22DC26DA80004ED6A4
:10DB000052D456D24AD85AD05ECEAE89B284AA8AAE
:10DB100097D0FFFFE78000250605130525024199F0
:10DB20000A8A3301A140232224FC231404FC97D049
:10DB3000FFFFE780202383C7990006054D0593F773
:10DB4000F7072315A4FCA384F9002685232624FCCB
:10DB500097E0FFFFE780402193170501C1876340ED
:10DB6000F0025281130104FCF2506254D254425923
:10DB7000B259225A925A025BF24B21618280AA8BDF
:10DB800003AB040097C0FFFFE780601E51E583D719
:10DB9000440001498544F11793B71700A301F4FC31
:10DBA000834734FCA165C9C79385E504130544FC8C
:10DBB00097C0FFFFE780C026A685130544FC97E0C9
:10DBC000FFFFE780A00ADE85130544FC97E0FFFF16
:10DBD000E780C00B834734FC114691E30946DA85A0
:10DBE000130544FC97E0FFFFE78060058144630A6A
:10DBF0000900416B7D1B97D0FFFFE780A01663CC27
:10DC0000A40201478146130644FCCE85568597C081
:10DC1000FFFFE7804046B1B7A685130634FC9700A6
:10DC20000000E780E0E6933415002A8986048DBF62
:10DC30009385C504A5BF8327C90013971400BA971D
:10DC400083D5070063886501130544FC97E0FFFF57
:10DC5000E780C003850445B71743FFFFE70223446D
:10DC600079711C103EC4B7070F003EC61C103EC899
:10DC700083C79500AA8A328593F7F707A384F50036
:10DC8000AE89328497E0FFFFE780000E931705010D
:10DC9000C187635AF0062A8A228597E0FFFFE78052
:10DCA000A00C2A895285032B040097C0FFFFE78050
:10DCB000000C39ED8357440081440544F11793B7B4
:10DCC0001700A303F10083457100DA872287CA8613
:10DCD0005286280097000000E780E0C8014781468F
:10DCE0003000CE85568597C0FFFFE780C038A1671A
:10DCF0009387D70348083ECC230A810026CE97F0AD
:10DD0000FFFFE78040DD45611743FFFF6700A33C4D
:10DD1000A2851306710097000000E78060D7AA84EF
:10DD2000094455D13544E30055FB4A8597F0FFFF80
:10DD3000E78000450D4441D9014497D0FFFFE780BB
:10DD40006002634DA400C16B0144FD1B97D0FFFF2F
:10DD5000E7804001634EA4001544B5B7DC441317B7
:10DD60001400BA9783D70700638327030504F1B72C
:10DD7000D84493171400BA9703D70700631B7701A1
:10DD800023902701268597A00000E78080DB0144CF
:10DD90001DBF050465BF1743FFFFE702233183C79B
:10DDA000950041112A8A93F7F707A384F50032857D
:10DDB0002E89328497E0FFFFE78000FB931705016F
:10DDC000C1876353F006AA89228597E0FFFFE780A9
:10DDD000A0F92311A1004E85832A040097C0FFFFFC
:10DDE000E780E0F839E58357440085440144F117A2
:10DDF00093B71700A300F100034811000357210057
:10DE0000D6875285CE862686CA8597F0FFFFE780A3
:10DE10006006A167F10748003EC42302910022C6B4
:10DE200097F0FFFFE78020CB41011743FFFF67001A
:10DE3000232BA2851306110097000000E78040C540
:10DE40002A84894455D98357210011678544BA979C
:10DE5000C2071167C1831307F7EFE36FF7F89787DE
:10DE6000FF1F9387E7069C4381CB8545130521005F
:10DE700097500000E780207583552100228581445A
:10DE800097C0FFFFE78040E525D9231005002285D4
:10DE900097A00000E78040CD85B71743FFFFE7025A
:10DEA000032083C7950041112A8B93F7F707A384BA
:10DEB000F50032852E8A328497E0FFFFE780C0EAC2
:10DEC00093170501C1876351F006AA8A228597E05E
:10DED000FFFFE78060E92A895685832B040097C0FD
:10DEE000FFFFE780C0E831E58357440081440544E3
:10DEF000F11793B71700A301F10003483100DE8743
:10DF00005A854A87D6862286D28597F0FFFFE7801A
:10DF100060F6A167ED0748003EC42302810026C6D3
:10DF200097F0FFFFE78020BB41011743FFFF670029
:10DF3000831AA2851306310097000000E78040B5E0
:10DF4000AA8409445DD99167CA97C2071167C18342
:10DF50001307F7EF0544E362F7FACA8597C0FFFF9E
:10DF6000E78080D7014451F9814997D0FFFFE780CE
:10DF700060E063DBA900984893971900BA9703D72C
:10DF8000070005EF2390270197D0FFFFE78080DE91
:10DF90001544E384A9F6268597A00000E780C0BC5D
:10DFA0009787FF1F9387C7F29C430144B9D74A85DF
:10DFB00097500000E780C05889B785097DB717439F
:10DFC000FFFFE702A30E79713E847C083EC82E8ACB
:10DFD000B7071400A1653ECAE5057C08AA890808B0
:10DFE00036C4428932C6BA8AC6843ECC97C0FFFF87
:10DFF000E78000E3CA85080897E0FFFFE78000C7D5
:10E0000032460808B28597E0FFFFE78020C8A246A5
:10E01000630A09049D45080897E0FFFFE780C0BE3A
:10E020001D4681459740FFFFE780E00C63890A08A1
:10E030009145080897E0FFFFE78000BD1146A685DF
:10E0400097000100E780607A100801478146D28579
:10E050004E8597C0FFFFE780000245611743FFFF31
:10E0600067000308B685080897E0FFFFE78000C255
:10E070001C400808D8439355C7018589120751836E
:10E08000B205D98D97E0FFFFE78040C01C4008082B
:10E0900083C5870097E0FFFFE78040BD1C4008086C
:10E0A00083C5A70097E0FFFFE78040BC1C4008083D
:10E0B00083C5970097E0FFFFE78040BB85BF894598
:10E0C000080897E0FFFFE78020B483C7040023001F
:10E0D000F50083C71400A300F500BDB71743FFFF89
:10E0E000E702C3FC83C795004111AA8993F7F7079C
:10E0F000A384F5003285AE84328497E0FFFFE78089
:10E10000A0C693170501C187635DF0042A89032A1D
:10E11000040097C0FFFFE78080C519E983574400DA
:10E120000548F11793B71700A307F100814631A8FE
:10E130001306F100A28597000000E78060951DC5D9
:10E140001C459DC783D6470001480347F10093074C
:10E150008500D2884A86A6854E8597000000E78014
:10E1600040E641011743FFFF670083F709487DBF81
:10E170001D486DBF1743FFFFE70243F365715C085D
:10E180003EC4B7077B013EC65C083EC883C7950006
:10E190002A8A328593F7F707A384F500AE8997E0C2
:10E1A000FFFFE78040BA8357E100E1C789452800B7
:10E1B00097C0FFFFE780C0C68145280097E0FFFFBA
:10E1C000E780C0AA97C0FFFFE780A0CC9787FF1F1A
:10E1D000938707089C431784FF1F0344E4B0AA8475
:10E1E0003334800099C3136424009787FF1F9387FB
:10E1F000E7B79C4399C3136444009787FF1F938735
:10E2000027CD9C4399C31364840083D50400280060
:10E21000014997E0FFFFE78060A783D5240028002D
:10E2200097E0FFFFE78080A683D54400280097E0B1
:10E23000FFFFE780A0A597D0FFFFE780A0AE931572
:10E240000501C181280097E0FFFFE78020A4A28597
:10E25000280097E0FFFFE78060A39C446360F90219
:10E26000014781463000CE85528597C0FFFFE78089
:10E2700080E059611743FFFF670083E6DC44131415
:10E28000490028003E9497E0FFFFE78060968347AF
:10E2900044000347540089070607BA978607E36AD4
:10E2A000F5FC835524002800814A97E0FFFFE780B2
:10E2B000E09D83454400280097E0FFFFE780009B36
:10E2C00083455400280097E0FFFFE780209A8347AA
:10E2D000440063C9FA00814A8347540063C1FA02CB
:10E2E0000509A5BF1C4413975A002800BA9783D587
:10E2F0000700850A97E0FFFFE7804099C9BF032B1D
:10E30000C40093975A0028003E9B83552B00850A32
:10E3100097E0FFFFE780809783550B00280097E088
:10E32000FFFFE780A0964DBF1743FFFFE702A3D989
:10E330005C4993E717005CC997A00000E78020B60E
:10E340001743FFFF670063DA1743FFFFE702A3D716
:10E350002E84814597F0FFFFE780C0E705C583570E
:10E360000500FD172310F50009C48357250023106D
:10E37000F40097000000E78060FB01451743FFFFB2
:10E380006700A3D631457DD823100400C5BF1743CD
:10E39000FFFFE702A3D183C7950041112A8A93F7B3
:10E3A000F707A384F50032852E89328497E0FFFFBA
:10E3B000E780809B93170501C1876356F006AA8901
:10E3C000C145228597E0FFFFE780A0802A8B4E851C
:10E3D000832A040097C0FFFFE780609931E98357E3
:10E3E0004400231101000544F11793B71700A3005F
:10E3F000F10081440348110003572100D68752855C
:10E40000CE862286CA8597F0FFFFE780A0A6A16787
:10E410009387170248003EC42302810026C697E076
:10E42000FFFFE780406B41011743FFFF670043CBCD
:10E4300013061100A28597F0FFFFE7806065AA84AC
:10E4400009E523110100094475B7930521005A8598
:10E4500097000000E78080EF835721002A84D9DBF2
:10E460009787FF1F9387C7A69C4381CB85451305DC
:10E47000210097500000E780001583552100268574
:10E48000314497C0FFFFE78020852DD5231005007C
:10E49000268597900000E780206D0144A1BF1743B7
:10E4A000FFFFE70243C241112E896C00AA8402C615
:10E4B00097F0FFFFE78000D20DC103570500050765
:10E4C0002310E50097000000E78040E681473E8585
:10E4D00041011743FFFF670043C13247954765DBA2
:10E4E000CA85268597300000E780400DC147E3408C
:10E4F00005FE3244854741462310F4008357090046
:10E50000A685130544002311F40097000100E7805D
:10E51000C02D228545BF1743FFFFE70223B983C7FC
:10E5200095004111AA8A93F7F707A384F500328575
:10E53000AE89328497E0FFFFE780008393170501DF
:10E54000C1876356F0062A8AC145228597D0FFFF0E
:10E55000E7802068AA845285032B040097C0FFFF40
:10E56000E780E08031E983574400231101008544AE
:10E57000F11793B71700A300F100014403481100FD
:10E5800003572100DA875685D2862686CE8597F0F6
:10E59000FFFFE780208EA1679387070248003EC4F3
:10E5A0002302910022C697E0FFFFE780C05241019D
:10E5B0001743FFFF6700C3B2A2851306110097F04F
:10E5C000FFFFE780E04C2A8409E52311010089441C
:10E5D00075B726859305210097000000E78060EC61
:10E5E000AA8449FD83552100228597B0FFFFE7806B
:10E5F000A06E49F5014997C0FFFFE780A077635DF2
:10E60000A900184893171900BA9703D707000DEF10
:10E61000035721002390E70097C0FFFFE780807534
:10E62000630625039787FF1F9387878A9C4399C7B3
:10E630000355210097500000E78080F022859790D5
:10E640000000E78060521DBF050975B795443DB7CE
:10E6500005C19307F00F630FF500C547630CF50084
:10E660009307F5FF05453315F5004205418182808A
:10E670000145828041657D158280B9E91743FFFF1E
:10E68000E70263A403450603328497000000E78095
:10E6900060FC9305803EB305B502C205C18181CD02
:10E6A0000357E402854763F8E7001305040197E088
:10E6B0000000E78020428357E40241677D176385AD
:10E6C000E700FD172317F4021743FFFF6700E3A1DC
:10E6D00082801743FFFFE702839C004283C79500B7
:10E6E000444D0349140093F7F707A384F5008347CB
:10E6F0000400220911673369F900A167B347F900E3
:10E7000041112A8BAE8A63ECE70E8347240013077E
:10E71000C00EB91793F7F70F6373F7100347340070
:10E72000C14763EEE70E834744001307E00793C732
:10E7300007086371F70C8349840083477400A209BA
:10E74000B3E9F900856763F7F90A034A6400834770
:10E7500054004E85220A336AFA0097500000E78081
:10E76000403B61C123962403834B3400137AFA00A3
:10E77000239A34032388740323994403938904015F
:10E78000631C090023A60402239804024E8597E027
:10E790000000E78060363DA0034924004A859700C9
:10E7A0000000E78020EB2397A402834744004E85B6
:10E7B000A388F402E38D0BFCE30B09FC97E0000057
:10E7C000E780202F97900000E78000738146014684
:10E7D000D6855A8597E0FFFFE7800058A1679387A9
:10E7E00097033EC423020100480002C697E0FFFFE2
:10E7F000E780602E41011743FFFF6700C38D85440A
:10E80000A2862686D6855A8597E0FFFFE780C0540A
:10E81000A167938797033EC423029100F1B7BD44DB
:10E82000C5B79144F1BF1743FFFFE70223880111E9
:10E830001C08404D3EC2B7070F003EC41C083EC630
:10E840002A89AE8997C0FFFFE780A0DA585C1C5C7C
:10E850006346B70E6394E50063E2A70E3385A740D5
:10E86000B3B7A700B305B7401306803E81469D8D20
:10E8700097000100E78080B793140501C180A1656E
:10E880009385C503480097B0FFFFE7806059814535
:10E89000480097D0FFFFE780603D8355040448009F
:10E8A00097D0FFFFE780803E83552404480097D02F
:10E8B000FFFFE780A03D814589CCC167FD17930527
:10E8C000F00F6388F400268597500000E780E0E0B1
:10E8D000AA85480097D0FFFFE780403903554404DC
:10E8E000814501CDC167FD179305F00F6307F50062
:10E8F00097500000E78060DEAA85480097D0FFFFB0
:10E90000E780C03683456404480097D0FFFFE78066
:10E91000E03583457404480097D0FFFFE780003559
:10E92000500001478146CE854A8597B0FFFFE780BA
:10E93000807405611733FFFF6700837A814481B7D4
:10E940001733FFFFE702237883C7950093F7F70794
:10E95000A384F50097000000E78020ED1733FFFF48
:10E960006700A3781733FFFFE702437483C795005E
:10E970004111404D93F7F707A384F5002A8A3285A9
:10E98000B284AE8997D0FFFFE780003E2A8B2685B0
:10E9900097D0FFFFE780403D2A89268597D0FFFF6B
:10E9A000E780603A93170B0163CA0702E177CA97C1
:10E9B000C207C183116763E3E70293070910C20727
:10E9C000C1831307B00F637BF70093170901C18759
:10E9D000AA8A634AF000C54763FE57014101173315
:10E9E000FFFF6700E36F97B0FFFFE780C028E317E2
:10E9F00025FFD5B763080B026306090281446389CA
:10EA00000A02B7077F0023106405231124057CC088
:10EA1000568597000000E780E0C39304803EB3046E
:10EA2000950239A0B7077F00232004047CC08144ED
:10EA30000355240497E00000E780A0A3A1C497C079
:10EA4000FFFFE78000BB269593D7F441333795004D
:10EA5000AE97BA9708DC5CDCCE8552859700000043
:10EA6000E780A0DC99E023220404A1679387B70321
:10EA700048003EC42302010002C697E0FFFFE78082
:10EA80008005A9BF814701481CDC232E0403E9B798
:10EA90001733FFFFE702236397C0FFFFE780C0370C
:10EAA000E1473305F502914597500000E78000C526
:10EAB000E55711C59777FF1F23A6A72281473E85FB
:10EAC0001733FFFF6700636285471777FF1F230D2A
:10EAD000F72082801733FFFFE702E35E9777FF1F7F
:10EAE0009387072080433DC0835704046390A706A3
:10EAF00083572404639CB7043689B28497C0FFFF10
:10EB0000E78020AF5C5C63C3B7046395B7001C5C0F
:10EB100063EEA7028347640463F3F400A68723032C
:10EB2000F4048347740463F39700A687A303F404F3
:10EB30008357440441677D176385E70085072312E7
:10EB4000F4043C4481C7CA85268582971733FFFFAA
:10EB50006700A3599777FF1F938787189C43014548
:10EB600099C303C5870082801733FFFFE702A355CF
:10EB70000111B70707003EC683C79500584D0AC468
:10EB800093F7F7070AC8A384F5002A89AE8411CB4E
:10EB90001C4283C707002304F70097900000E7801A
:10EBA0000034216493055402280097B0FFFFE780EA
:10EBB000202797000000E78020FAAA85280097D038
:10EBC000FFFFE780A00A300001478146A6854A85FD
:10EBD00097B0FFFFE780204A13044402480822CC84
:10EBE000230A010002CE97E0FFFFE780C0EE056137
:10EBF0001733FFFF6700634F1733FFFFE702A34C94
:10EC000001117C003ECAB70707003ECC7C003ECE17
:10EC100083C795002E84AA8493F7F707A384F50091
:10EC2000A16593855502480897B0FFFFE780401F14
:10EC300097000000E78040F2AA85480897D0FFFFC0
:10EC4000E780C002500801478146A285268597B01B
:10EC5000FFFFE780404205611733FFFF6700E3488D
:10EC60009777FF1F9387C7079C43094599C303C53F
:10EC7000970082809777FF1F938787069C430945FB
:10EC800099C303C5D70082809777FF1F93874705F5
:10EC90009C43014599C303C5A70082801733FFFF3A
:10ECA000E702C3400111B70708003EC683C79500BD
:10ECB000404D0AC493F7F7070AC8A384F5002A89D0
:10ECC000AE8429C41442854703C7060063E0E70AFF
:10ECD00083479400094681496380C702B307F74020
:10ECE000A304E400B339F00083C716002305F40041
:10ECF00097900000E780A01E03572403058B19C7D7
:10ED00006386090097D00000E78000E9216493053D
:10ED10008402280097B0FFFFE78080109700000072
:10ED2000E78040F4AA85280097D0FFFFE78000F431
:10ED300097000000E78080F5AA85280097D0FFFFA4
:10ED4000E780C0F2014781463000A6854A8597B02A
:10ED5000FFFFE780403213047402480822CC230AE4
:10ED6000010002CE97E0FFFFE780E0D60561173390
:10ED7000FFFF6700E3361733FFFFE702C3340111DB
:10ED80007C003ECAB70708003ECC7C003ECE83C75D
:10ED900095002E84AA8493F7F707A384F500A16554
:10EDA00093858502480897B0FFFFE78060079700CA
:10EDB0000000E78020EBAA85480897D0FFFFE78096
:10EDC000E0EA97000000E78060ECAA85480897D049
:10EDD000FFFFE780A0E9500801478146A28526850C
:10EDE00097B0FFFFE780202905611733FFFF670019
:10EDF000C32F9777FF1F9387A7EE9C43014599C3C5
:10EE000003C5B70082801733FFFFE702C32B011150
:10EE1000B70707003EC683C79500404D0AC493F765
:10EE2000F7070AC8A384F5002A89AE8405C81C42E6
:10EE3000054783C707006368F7060347B400630FFD
:10EE4000F700A305F40097900000E780400983478E
:10EE5000B400B9CF97D0FFFFE78040BE216493058F
:10EE6000B400280097B0FFFFE78080FB9700000008
:10EE7000E78060F8AA85280097D0FFFFE78000DFD1
:10EE8000014781463000A6854A8597B0FFFFE7809D
:10EE9000801E2904480822CC230A010002CE97E0F4
:10EEA000FFFFE78040C305611733FFFF6700E323DF
:10EEB00097D0FFFFE78020BF55B71733FFFFE7026A
:10EEC000832001117C003ECAB70707003ECC7C00BE
:10EED0003ECE83C795002E84AA8493F7F707A384B8
:10EEE000F500A165AD05480897B0FFFFE78040F346
:10EEF00097000000E78020F0AA85480897D0FFFF20
:10EF0000E780C0D6500801478146A285268597B084
:10EF1000FFFFE780401605611733FFFF6700E31C22
:10EF20009777FF1F9387C7DB9C43094599C303C5A8
:10EF3000C70082801733FFFFE702E31801117C004E
:10EF4000AE843ECAA165B70707002A843ECCD1052E
:10EF50007C0048083ECE97B0FFFFE78060EC97004A
:10EF60000000E78020FCAA85480897D0FFFFE780D3
:10EF7000E0CF500801478146A685228597B0FFFF64
:10EF8000E780600F05611733FFFF67000316173333
:10EF9000FFFFE702431383C7950093F7F707A384A6
:10EFA000F50097000000E78020F91733FFFF6700A6
:10EFB000C3131733FFFFE702630F83C795000329CD
:10EFC000C501411193F7F707A384F5001C4283C9DB
:10EFD0000700854763E637079777FF1F9387472723
:10EFE0009C432E84AA8485CF97000000E78080F39D
:10EFF00089476306F502630409028347C9006380F9
:10F0000037032306390197900000E78040ED8357CE
:10F010002903898B89C797D00000E780E0B7268550
:10F02000A28597000000E78020F1A167CD07480086
:10F030003EC42302010002C697E0FFFFE780A0A9BB
:10F0400041011733FFFF6700A3099777FF1F9387DD
:10F0500027C99C431D4599C303C5E7008280173328
:10F06000FFFFE70243060111B70707003EC683C74B
:10F070009500584D0AC493F7F7070AC8A384F50012
:10F080002A89AE8415C71C4283C70700939687015F
:10F09000E18663C4060685466381D7068346E7009A
:10F0A0006388F6002307F70097900000E78020E3CD
:10F0B00021649305E400280097B0FFFFE78040D665
:10F0C00097000000E780A0F8AA85280097D0FFFFEE
:10F0D000E780C0B9014781463000A6854A8597B0D0
:10F0E000FFFFE78040F93504480822CC230A0100DD
:10F0F00002CE97E0FFFFE780009E05611733FFFF18
:10F100006700A3FE1733FFFFE702E3FB01117C005A
:10F110003ECAB70707003ECC7C003ECE83C79500B1
:10F120002E84AA8493F7F707A384F500A165B90597
:10F13000480897B0FFFFE780A0CE97000000E78067
:10F1400000F1AA85480897D0FFFFE78020B2500859
:10F1500001478146A285268597B0FFFFE780A0F191
:10F1600005611733FFFF670043F81733FFFFE7021E
:10F17000E3F3AA8401441779FF1F1309A9B6E149F3
:10F1800097C0FFFFE78040C96344A400014519A868
:10F1900033053403832709003E9583572500639781
:10F1A000970011051733FFFF670083F30504C9BFFC
:10F1B000032E8500630A0E121773FF1F130343D13A
:10F1C00003230300631503002943639006120323FE
:10F1D0004E01631503001D43639907101733FFFFAA
:10F1E000E702E3EBC689428A3E89BA8AB684328B4B
:10F1F000AE8B2A84B5E103554E0019E501431A850B
:10F200001733FFFF670023EDA167A98F116763FB29
:10F21000E70097000000E78080F5814597F0FFFF49
:10F22000E780C0120844B70700E05841F98F18453D
:10F230005CC1B707001FF98F1CC55C4991C7610508
:10F2400097E00000E780408BE38A09FA22859790D7
:10F250000000E78060C65DB7328597C00000E78098
:10F2600040430D4349DD1C44116703D54700A167A6
:10F27000A98F63FBE70097000000E78040EF81451E
:10F2800097F0FFFFE780800C0323840093164B0167
:10F29000D1828347B300035663008588FD8BA305A5
:10F2A000F300FD777D8E558EFD76FD16B204F18E4E
:10F2B00083274301C58E231273012313D300230434
:10F2C000530123052301A3044301BDDF228597B029
:10F2D000FFFFE78020CDAA850844B5D1610597D00E
:10F2E0000000E780207F8DB71D431A858280173389
:10F2F000FFFFE702A3DB0569AA84AE89328A0144D5
:10F30000FD5A7D1997C0FFFFE780C0A56347A400A1
:10F3100001451733FFFF6700A3DCD844931714009F
:10F32000BA9703D70700631F37032390570163077A
:10F330000A00268597900000E780A0809C449DC32A
:10F3400083D76700B3F72701639E3701D28801484E
:10F350008147014781460146814526859700000087
:10F36000E78040E5050479BF1733FFFFE70203D4C8
:10F3700079711C103EC4B7070F003EC61C103EC872
:10F3800083C79500AA8A328593F7F707A384F5000F
:10F390002E89328497D0FFFFE780009D93170501E7
:10F3A000C187635AF006AA89228597D0FFFFE780BC
:10F3B000A09B2A8A4E85032B040097B0FFFFE780AD
:10F3C000009B39ED8357440081440544F11793B7FE
:10F3D0001700A303F10083457100DA872287D286E4
:10F3E0004E86280097E0FFFFE780E05701478146FF
:10F3F0003000CA85568597B0FFFFE780C0C7A16778
:10F400009387F70348083ECC230A810026CE97D085
:10F41000FFFFE780406C45611733FFFF670043CC77
:10F42000A2851306710097E0FFFFE7806066AA845B
:10F43000094455D1528597E0FFFFE78060D40D4421
:10F4400059D90546D285268597000000E78060EAF5
:10F450002A8451B71733FFFFE702E3C6835507003D
:10F460000346270041112A842E8532C62EC497E018
:10F47000FFFFE780E0D001C93246A2452285970010
:10F480000000E78000E741011733FFFF6700E3C595
:10F490001733FFFFE702A3C083C795004111AA8A73
:10F4A00093F7F707A384F5003285AE89328497D0AD
:10F4B000FFFFE780608B93170501C1876357F00A50
:10F4C000C1452A8A228597C0FFFFE78080702A8D78
:10F4D000228597D0FFFFE78020892A89228597D04F
:10F4E000FFFFE7804086930705F893F7F70F1307B0
:10F4F000E007AA8B637BF706228597D0FFFFE780A2
:10F5000080842A8C228597D0FFFFE780C083AA8C55
:10F510005285032B040097B0FFFFE780408539E94F
:10F5200083574400231101008144F11793B717005A
:10F53000A300F1000544034711008356210093877F
:10F5400084005685DA8822885286CE8597F0FFFFA0
:10F55000E78020A7A167E90748003EC42302810095
:10F5600026C697D0FFFFE780005741011733FFFF02
:10F57000670063B613061100A28597E0FFFFE780DE
:10F580002051AA8409E52311010009446DB79305B0
:10F5900021006A8597F0FFFFE780A0F02A8441FDF3
:10F5A000835521009356C900131649018548668882
:10F5B000E2875E87858A5182268597000000E78072
:10F5C00060BF2A848DBF1733FFFFE70243AD83C7B7
:10F5D000950041112A8B93F7F707A384F500328534
:10F5E000AE89328497C0FFFFE7800078931705014A
:10F5F000C1876352F00A2A8A228597C0FFFFE780FD
:10F60000A076AA8A228597C0FFFFE780E0752A8945
:10F61000228597C0FFFFE7800073930705F893F7F3
:10F62000F70F1307E0072A8C6377F706228597C048
:10F63000FFFFE7804071AA8C228597C0FFFFE7801B
:10F6400080702A8D5285832B040097A0FFFFE780EE
:10F65000007239E58357440085440144F11793B79C
:10F660001700A301F10003473100930784005A8576
:10F67000DE882688D6865286CE8597F0FFFFE78003
:10F6800040948D4748003EC42302910022C697D083
:10F69000FFFFE780404441011733FFFF6700A3A34A
:10F6A000A2851306310097E0FFFFE780603E2A84C1
:10F6B000894455D99356C9001316490185486A886B
:10F6C000E6876287858A5182D68597000000E780A9
:10F6D00060AEAA8449BF1733FFFFE702239D2A8942
:10F6E00081440144617A916A176BFF1F130B4B7EB3
:10F6F00097B0FFFFE780006863C7A4002285173337
:10F70000FFFF6700E39D8327090093991400CE97BC
:10F7100003D507003307450142074183636457035C
:10F7200005C103270B0019C785453E85974000009A
:10F73000E78060E9832709000504CE97239007003E
:10F7400085047DB797000000E78060A28327090049
:10F750000504CE972390070065D5814597F0FFFFFC
:10F76000E780C0BEF1BF1733FFFFE702239483C7D2
:10F77000950041112A8A93F7F707A384F500328593
:10F780002E89328497C0FFFFE780005E9317050142
:10F79000C187635AF004AA89832A040097A0FFFF57
:10F7A000E780E05C31E58357440085440144F1176C
:10F7B00093B71700A301F10003483100D6875285A3
:10F7C0000147CE862686CA8597D0FFFFE780806AEC
:10F7D000A167F50748003EC42302910022C697D0D6
:10F7E000FFFFE780402F41011733FFFF6700438F82
:10F7F000A2851306310097E0FFFFE78060292A8485
:10F8000089445DD99767FF1F9387876C9C4381CF9D
:10F81000044997B0FFFFE780E055AA852685974009
:10F820000000E78040DA1305040197000000E7803C
:10F83000C0EA228597800000E78000338144ADBF95
:10F840001733FFFFE702A38583C795004111AA8AFA
:10F8500093F7F707A384F5003285AE89328423112C
:10F86000010097C0FFFFE780205093170501C18773
:10F870006354F0062A8AC145228597C0FFFFE780BE
:10F880004035AA8B5285032B040097A0FFFFE78029
:10F89000004E21E98357440085440144F11793B792
:10F8A0001700A300F1000348110003572100DA8775
:10F8B0005685D2862686CE8597D0FFFFE780805B6F
:10F8C000A1679387270248003EC42302910022C605
:10F8D00097D0FFFFE780202041011723FFFF67003B
:10F8E000837FA2851306110097E0FFFFE780401A8F
:10F8F0002A8489444DD99767FF1F9387675D984392
:10F900003E8901CF044997B0FFFFE780A046AA8552
:10F91000268597400000E78000CB1305040197007F
:10F920000000E78080DB97B0FFFFE780A0449544AC
:10F930003DD9930521005E8597F0FFFFE78060B613
:10F94000AA8435F11C480357210022852390E70043
:10F9500097800000E780402183270900A9D703553D
:10F96000210097400000E780A0BD35BF1723FFFFAF
:10F97000E702E37283C795004111AA8A93F7F7075C
:10F98000A384F5003285AE89328497C0FFFFE780FB
:10F99000A03D93170501C1876351F0062A8A22858D
:10F9A00097C0FFFFE780403C2A895285032B040063
:10F9B00097A0FFFFE780A03B31E5835744008544D3
:10F9C0000144F11793B71700A301F1000348310078
:10F9D000DA8756854A87D2862686CE8597D0FFFF5E
:10F9E000E7804049A167F90748003EC4230291001F
:10F9F00022C697D0FFFFE780000E41011723FFFFCB
:10FA00006700636DA2851306310097E0FFFFE78072
:10FA100020082A8489445DD99167CA97C207116773
:10FA2000C1831307F7EF8544E362F7FA9767FF1F77
:10FA30009387074A9843BE8B01CF044997B0FFFFD5
:10FA4000E7804033AA85268597400000E780A0B76D
:10FA50001305040197000000E78020C897B0FFFF5E
:10FA6000E780403195443DD11C4822858144239054
:10FA7000270197800000E780200F83A70B00B9D7EC
:10FA80004A8597400000E780A0AB89B71723FFFFA6
:10FA9000E70263632A844105B28497000000E7808F
:10FAA000C0C311C5228597800000E780E00B814626
:10FAB0000146A685228597800000E780C04E1C4C39
:10FAC00089C7DC4799C3228582971723FFFF670008
:10FAD000C3619767FF1F9387A7209C43014599C384
:10FAE0001385070182809767FF1F9387671F8843ED
:10FAF00082801723FFFFE702035D9317C600DD8DA9
:10FB0000C2054111C1812A8432C697C0FFFFE78038
:10FB1000E0173246228511829375F60F97C0FFFFDA
:10FB2000E780C01441011723FFFF6700035C172320
:10FB3000FFFFE702A35779713C083ED2B7070C00DC
:10FB40003ED43C083ED683C79500AE842A8993F7FD
:10FB5000F707A384F500A16593853504481097A0A5
:10FB6000FFFFE780E02BC165FD150144176AFF1F09
:10FB7000130A8A37930A400EAE892E8B2EC697B091
:10FB8000FFFFE78020224205931704014181C183D2
:10FB9000B24563E9A702C167FD176387F500481006
:10FBA00097C0FFFFE780800E501001478146A68571
:10FBB0004A8597A0FFFFE780004C45611723FFFFB0
:10FBC000670003523307540383270A0BBA9703D6FF
:10FBD000C701630A3601638A3501481097000000A7
:10FBE000E78060F1DA85050451BFB285EDBF1723C8
:10FBF000FFFFE702C34A79717C083EC8B7071100CE
:10FC00003ECA7C083ECC83C79500AA89328593F70B
:10FC1000F707A384F5002E8997C0FFFFE780C01483
:10FC200085676378F504A165AA848905080897A00B
:10FC3000FFFFE780E01E268597400000E78060ED2B
:10FC4000133415000A04A285080897C0FFFFE78057
:10FC5000E001A685080897C0FFFFE780200325CCB8
:10FC6000014781461008CA854E8597A0FFFFE780AF
:10FC7000804045611723FFFF6700E345B307540346
:10FC80000327CA0ABA9703D70700631C970003D655
:10FC9000270063806505080897000000E780A0E55D
:10FCA000DE8505042EC697B0FFFFE780A010420551
:10FCB000931704014181C183B245E3E1A7FCC16709
:10FCC000FD17E38FF5F8080897C0FFFFE78000FCF9
:10FCD00041BFB285F9B7C165FD150144176AFF1F21
:10FCE000130A8A20930A80022E8BAE8B65BF1723DE
:10FCF000FFFFE702433D1841834717008346070093
:10FD0000A207D58FD207D1832390F5008347270020
:10FD1000034717008D45A207D98F91832310F60062
:10FD200097C0FFFFE780A0E91723FFFF6700E33BD1
:10FD30001723FFFFE7028337C16401441769FF1FE0
:10FD40001309891A93098002FD1497B0FFFFE78019
:10FD500060066347A40001451723FFFF670043388F
:10FD6000330534038327C90A3E9583570500E3858D
:10FD700097FE0504D9BF1723FFFFE70223332A8A22
:10FD8000AE89B284B68A97400000E78080D819E532
:10FD900091473E851723FFFF670083342A894E85EC
:10FDA00097C00000E780E08E2A84638E0A048D47A6
:10FDB0006DD103570500C547E31D47FD0347F90112
:10FDC0008546AD47E317D7FC8347450081CF4146C1
:10FDD000A6855D0597F00000E780C09E814755D954
:10FDE000AD4745BF130965012302E500CA85268595
:10FDF00097100000E780606231C1A547E38B0AF8E5
:10FE00002302040079B705C183570500E39247F93F
:10FE10004146A685190597F00000E780A09A814722
:10FE20002DD99947BDB74E8597000000E78080F037
:10FE30002A84954739DD130955004DBF4146A685F3
:10FE400023104401231134011305190097F0000019
:10FE5000E780A099228597800000E780A0EA81478B
:10FE60000DBF1723FFFFE702032679717C003ECC0C
:10FE7000B7070A003ECE7C003ED083C79500B2840F
:10FE80002E8493F7F707A384F5001306A1002A89AF
:10FE90002C00268597000000E780A0E5A1652808D2
:10FEA0008D0597A0FFFFE780A0F790408355A10044
:10FEB00003558100854697000000E78000ECAA8486
:10FEC000AA85280897C0FFFFE78040DA0356A10003
:10FED00083558100280897000000E780C0C13008E2
:10FEE00001478146A2854A8597A0FFFFE780A018B9
:10FEF000854748103ED42302910202D697D0FFFFD7
:10FF0000E78060BD45611723FFFF6700031E1723CD
:10FF1000FFFFE702431B79717C003ECCB7070A0064
:10FF20003ECE7C003ED083C79500B2842E8493F7EA
:10FF3000F707A384F5001306A1002A892C00268563
:10FF400097000000E780E0DAA16528088D0597A0FA
:10FF5000FFFFE780E0EC90408355A100035581004E
:10FF6000814697000000E78040E1AA84AA8528081E
:10FF700097C0FFFFE78080CF0356A1008355810023
:10FF8000280897000000E78000B730080147814645
:10FF9000A2854A8597A0FFFFE780E00D4810230265
:10FFA000910202D402D697D0FFFFE780C0B245612C
:10FFB0001723FFFF670063131723FFFFE702A31058
:10FFC00097000000E78060DB1723FFFF6700E31165
:10FFD0009767FF1F938707D1884382801723FFFF0E
:10FFE000E702630E835725004111AE842A8423075C
:10FFF000B10017F5FFFF130525466C002316F1002D
:020000040001F9
:1000000097A0FFFFE780204991C4228597800000D8
:10001000E780E0D6FD572310F40013062002814547
:10002000130554009720FFFFE780E00C41011723E0
:10003000FFFF6700830B1723FFFFE7022307797198
:100040007C003ECCB7070A003ECE7C003ED083C782
:100050009500AA89AE8493F7F7073285A384F5004B
:100060001306A1002C0097000000E78080C803550C
:100070008100114497400000E780A0A915C50355F1
:10008000A100014497B00000E780A06011CD0357A4
:1000900005008357810045446318F70085459700A4
:1000A0000000E780E0F30144216993053900280846
:1000B00097A0FFFFE780C0D6A285280897C0FFFF62
:1000C000E780C0BA0356A100835581002808970035
:1000D0000000E78040A2300801478146A6854E8592
:1000E00097A0FFFFE78020F948104AD4230281023D
:1000F00002D697D0FFFFE780009E45611723FFFFE0
:10010000670003FE1723FFFFE70243FA9767FF1F0D
:10011000938707BD2A8488432E8915C50357450355
:100120008357C4016311F702232605022318050231
:10013000410597D00000E780209C63060900978066
:100140000000E78060DB81449769FF1F9389C9D96C
:10015000130A800297B0FFFFE780C0C563C4A40400
:100160009767FF1F938787C09C4399C70355C401B6
:1001700097200000E780C0BD6307090022859780B3
:100180000000E780C0A01306400E8145228597201D
:10019000FFFFE78040F6FD57231EF4001723FFFF03
:1001A000670003F43385440383A7C90A3E950357C8
:1001B00005008357C4016317F700CA859700000044
:1001C000E78000E2850479B71723FFFFE70203EE1B
:1001D00083C795004111AA8993F7F707A384F50017
:1001E0003285AE8497C0FFFFE78000B885676378EB
:1001F000F5042A8997400000E780A091014401CDD1
:1002000083D70400314463882701854597000000A7
:10021000E78080EF01444E85A2864A86A68597D066
:10022000FFFFE780A09CA1679387170448003EC4A6
:100230002302810002C697D0FFFFE780C0894101F9
:100240001723FFFF6700C3E91723FFFFE70203E659
:100250009767FF1F9387C7A8804329C4014597C0AC
:100260000000E780002181470148C1641CDC232E87
:100270000403232004041769FF1F1309E9C601447E
:100280009309400EFD1497B0FFFFE780A0B1634FC4
:10029000A400814517F5FFFF1305857F97A0FFFF99
:1002A000E780601F1723FFFF670083E333053403F4
:1002B0008327090B3E958357C501638797008545C2
:1002C00097000000E78040E4050475BF93570501DF
:1002D00013D78700A380F50093170501C183A1837D
:1002E0002380E5002381F500A381A50082801723E8
:1002F000FFFFE70243DD2300050083C71500A300CD
:10030000F50083C725002301F50083C73500A3014D
:10031000F50083C745002302F50083C75500A302FB
:10032000F50083C7650093059500A303050023032B
:10033000F50023040500328597000000E78040F9AE
:100340001723FFFF670063DA1723FFFFE70203D6D7
:100350004111E9540DCD85CD93F9C5FF2E842A892D
:10036000AA84338AA900B7EA040063189A020D88A8
:10037000854411CCB7E704009C5F82972AC6228689
:100380006C003305390197E00000E78000462685C0
:1003900041011723FFFF6700A3D483A78A039104B9
:1003A000829793170501C183A183A38EF4FE93570F
:1003B0000501238FF4FEA183238EA4FEA38FF4FEF8
:1003C0006DB763E6D5021723FFFFE702C3CFB287FD
:1003D00041113686BE8536C697E00000E780E040D2
:1003E000B246410136851723FFFF670003D08146DF
:1003F00036858280838705001387F5003D05FD87DC
:1004000093F77708834607007D158606B58FA3000E
:10041000F5006307B7007D17834717009D83DDB79D
:1004200082801723FFFFE70203CAB7E7040083A710
:10043000070932872A863A858297133515001723D4
:10044000FFFF670083CA15C181478DC11723FFFFD6
:10045000E70263C7414697E00000E780003985471F
:100460003E851723FFFF670043C881473E85828092
:100470001DCD1723FFFFE70203C5414681452A84AE
:100480009720FFFFE78020C74146814513050403FD
:100490009720FFFFE78020C60147C167232204049D
:1004A00038C87CC805451723FFFF670003C4014512
:1004B000828081473DCDB5CD1723FFFFE702A3C062
:1004C000B2842E891306800581452A849720FFFF78
:1004D000E78060C2CA8524C4268597000000E780B3
:1004E000C0F64146814522859720FFFFE780A0C0E6
:1004F0003044A285228597000000E780C0F2930473
:100500000401A285268597000000E780E0EEA6851D
:100510001305040297000000E78000EE2285970093
:100520000000E78020F585473E851723FFFF670021
:10053000C3BB3E8582801723FFFFE70223B741112B
:10054000E9540DCD85CD93F9C5FF2E842A89AA845F
:10055000338AA900B7EA0400639844030D888144F4
:1005600011CCB7E704009C5F82972AC622866C00F4
:100570003305390197E00000E780202726854101F7
:100580001723FFFF6700C3B583A78A0391048297EF
:1005900093170501C183A183A38EF4FE9357050130
:1005A000238FF4FEA183238EA4FEA38FF4FE6DB7E8
:1005B00065CD1723FFFFE70263AFB28411E605455F
:1005C0001723FFFF6700C3B12A842E890145EDD9A7
:1005D0003C487848B3E6E700E5D69386F7FFB3B723
:1005E000F6007D17032A4404BA9734C87CC8630513
:1005F0000A06C14913050A03B38949412295637D5F
:100600003601B2862E86A68597000000E780A0DB23
:100610007C40BE9464C065B7CE862E86CE8597009A
:100620000000E78040DAC114D2944E9923220404DA
:10063000A2879306040103C7070003C607038507C3
:10064000318FA38FE7FEE398F6FE3044A285228522
:1006500097000000E78020DD2699C14933069940C4
:1006600063EC9900A9DCA686A68513050403970010
:100670000000E78040D579BF8147B306F400330717
:10068000F6000347070083C5060085072D8F2380EA
:10069000E600E39437FF3044A285228597000000EE
:1006A000E78060D8C1145DBF014582800DC117236A
:1006B000FFFFE70243A11306800581459720FFFF56
:1006C000E78060A305451723FFFF670003A20145EC
:1006D0008280814749C5C1C51723FFFFE702A39E5A
:1006E000FC4141462E84AA846399C7041386050100
:1006F000A2878146C14503C7070003C507038507D5
:10070000298F3305D600034505008506298FA38F61
:10071000E7FEE392B6FE3044A285268597000000EE
:10072000E78060D0228597000000E78060F8854769
:100730003E851723FFFF6700439B138507031D8E2C
:10074000814522959720FFFFE780E09A7C401307C0
:1007500000F813060402A2972388E70251BF3E85E2
:1007600082801723FFFFE70203966D712E84B28407
:10077000AA8590102800368997000000E780A0D352
:1007800009EDD55725A050400C40280097000000E7
:10079000E78040E27DD5FD142104F5F42C004A8564
:1007A00097000000E78020F3814761DD3E855161BD
:1007B0001723FFFF670063931723FFFFE702A39050
:1007C00041112EC432C62C00054697000000E78078
:1007D00080F941011723FFFF670023911723FFFFD3
:1007E000E702638E01112A842EC602C802CA02CC17
:1007F00002CE97E00000E780402BB2462A86A28511
:10080000080897000000E78060FB1375F50F05618D
:100810001723FFFF6700638D1723FFFFE702A38AFB
:100820007971B2872A8421462308B100130511018A
:10083000BE853AC436C697E00000E78000FBB246AA
:1008400093059101368597000000E78060A8228516
:10085000141035460C0897000000E78020F62A8423
:10086000224701E921460C103A8597E00000E78015
:10087000C0F7228545611723FFFF67000387172311
:10088000FFFFE70243847171AE84AA850A85328432
:1008900097000000E78060BB11C90A86A685228503
:1008A00097000000E78020B8814711E1C5473E85E9
:1008B0004D611723FFFF670043831713FFFFE70214
:1008C000837D1D712A8AB289BE843546854713050A
:1008D00011012E8CB68A3A8BC28C468D2308F1000A
:1008E00097E00000E78060F010100C085285231F8D
:1008F000010097000000E780C0F82A843DEDA14781
:100900006313FD089307900591E0E5473546E285BE
:100910001305110113990A012308F1001359090164
:1009200097E00000E78060EC1357890093978A00F6
:10093000D98F90080C085285231FF1009700000002
:10094000E78020F42A8415E9A1E49387FA009183D3
:100950001379F9003EC6631309004149668B81444F
:10096000C14B854DB247639F970C6A868C003385D7
:100970005C0197E00000E78040E7228525611713BE
:10098000FFFF6700037593079004C9F0A547BDBF3B
:10099000834701050947C14B2308F100834711052F
:1009A000A58FA308F10093872400814463E1FB0431
:1009B000014714083386E6008C08B386E400BA9534
:1009C000DA9683C6060083C505000507AD8E2300B1
:1009D000D600E390E7FE4147639CE70490080C08CB
:1009E000528597000000E780C0E925D181A0B306B9
:1009F0009B00BA871008B305F60090083E9603C521
:100A000006000346060085078506298E2380C5005B
:100A1000E39277FF998F90080C085285BE94970057
:100A20000000E78000E68947014749D12A84B1B731
:100A300090083E96034606001408BE962380C60022
:100A4000850759BFB2478504638797148147180803
:100A5000B306F70098083E973386F900034707006E
:100A6000034606008507318F2380E600E39177FF78
:100A700090080C08528597000000E78080E05DF543
:100A80003546E285130511012308B10197E0000006
:100A9000E780A0D5139704014183939784002183B5
:100AA000D98F10180C085285231FF1009700000001
:100AB000E78020DD25FD814710183387F9003E9639
:100AC0000347070003460600B306FB008507318F86
:100AD0002380E600E39277FF65A81808B306F700C5
:100AE00098083E973386F90003470700034606003F
:100AF0008507318F2380E600E3E127FFCA87639EE5
:100B0000770990080C08528597000000E78060D7AD
:100B100011FD81479800B306F700900818103E9722
:100B20003E9603470700034606008507318F238062
:100B3000E600E39177FF3546E285130511012308AE
:100B4000B10197E00000E78040CA13970401418398
:100B5000939784002183D98F10180C085285231F86
:100B6000F10097000000E780C0D1E31105EC814758
:100B700010183387F9003E96034707000346060026
:100B8000B306FB008507318F2380E600E3E227FFF1
:100B9000C109410BC1BB814785B79408BE9683C686
:100BA000060018083E972300D700850789BF638099
:100BB00006321713FFFFE702034E59712A84BE89DC
:100BC000B28B85473546130511022E8B468C428920
:100BD000BA8A368A2300F10297E00000E780E0C07D
:100BE00010180C1022852317010297000000E780DF
:100BF00040C963180512A147631FFC0693079005BF
:100C000063930900E5473546DA851305110293140D
:100C10000A012300F102C18097E00000E780E0BCF8
:100C200093178A0013D78400D98F90080C1022855F
:100C30002317F10297000000E780A0C47DE16392D2
:100C400009049307FA00BD88918391E0C144C2076B
:100C5000C183DE8C814A3EC6414DB24763E2FA0E43
:100C60006286B3854B01881097E00000E78080B56D
:100C70004DC93D557DA093079004E39609F8A5471B
:100C800059B7834701050947C14C2300F102834747
:100C90001105B3C7F900A300F10293872900814928
:100CA00063E1FC04814618103306D7008C083387B3
:100CB000D900B69556970347070083C505008506FA
:100CC0002D8F2300E600E390D7FE41476390E706AF
:100CD00090080C10228597000000E78080BA35D17B
:100CE00089A0B3863A01BA871010B305F6009008C0
:100CF0003E9603C506000346060085078506298E35
:100D00002380C500E39297FF3387EC4090080C10D6
:100D10002285BA9997000000E780A0B6894701476D
:100D200041D165611713FFFF6700A33A90083E9613
:100D3000034606001410BE962380C600850779B7C7
:100D4000B247850A93990A01939D8A0093D90901B4
:100D50006391570F85473546DA8513051102230045
:100D6000F10293D9890097E00000E78000A8B3ED75
:100D70003D0190000C1022852317B103970000005D
:100D8000E78020B059FD8147A68963EA9706268649
:100D90000C084A8597E00000E78020A581471810DD
:100DA000B306F700100898083E973E9603470700E1
:100DB000034606008507318F2380E600E3E197FEB6
:100DC000639FA90590080C10228597000000E7801A
:100DD00040AB21F981479810B306F7009008181826
:100DE0003E973E9603470700034606008507318F6E
:100DF0002380E600E391A7FF4109C10CB9BD1808A3
:100E00009000B306F7003E963387FC0003470700C7
:100E1000034606008507318F2380E600B5B79808A2
:100E20004E97034707001C10CE972380E7008509E3
:100E300041BF85473546DA85130511022300F102CB
:100E400093D9890097E00000E780209AB3ED3D0137
:100E500090000C1022852317B10397000000E78053
:100E600040A2E31005EC814718089000B306F70094
:100E70003E963387FC0003470700034606008507BC
:100E8000318F2380E600E391A7FF41460C084A8595
:100E900097E00000E780609581471810B306F700DF
:100EA000100898083E973E96034707000346060041
:100EB0008507318F2380E600E391A7FF90080C108F
:100EC000228597000000E780C09B1DD599BD7D5508
:100ED00082801713FFFFE702031F01112A842E856A
:100EE00093055100328902C002C202C402C69304B3
:100EF000740097F0FFFFE780A03D1D46A68513050F
:100F0000910097E00000E780408E10088A854A85AE
:100F100097000000E780E09619ED93071400180889
:100F200083C607000346070085070507B18EA38F18
:100F3000D7FEE397F4FE05611713FFFF6700E31A7E
:100F40001713FFFFE70283162E848C414111AA89F3
:100F5000838715003289914463D30700A1449757D2
:100F6000FF1F9387E72E9C43A1C7C1CA8D4723105B
:100F7000F10083C725004A852301F10083C73500AE
:100F8000A301F10083C745002302F10083C7550088
:100F9000A302F10083C7650093059100A30301003C
:100FA0002303F1002304010097F0FFFFE7804032A4
:100FB0000C404A860A8597F0FFFFE78080330328BC
:100FC000040083564400A6881D0881470147E516A2
:100FD00042868A854E8597000000E780408E2A89E8
:100FE00019E5A685228597B0FFFFE780E0C14A8515
:100FF00041011713FFFF6700A30E4A860A8597F089
:10100000FFFFE780002F6DB71713FFFFE702030A0A
:101010002E848C414111AA8983871500328991441D
:1010200063D30700A1449757FF1F938767229C4310
:10103000A1C7C1C68D472310F10083C725004A858B
:101040002301F10083C73500A301F10083C74500E8
:101050002302F10083C75500A302F10083C7650096
:1010600093059100A30301002303F1002304010071
:1010700097F0FFFFE780C0250C404A860A8597F06D
:10108000FFFFE780002783564400032804008A8579
:10109000858EC2061D08C1822312D400A68881470E
:1010A0000147E51642864E8597000000E78060B054
:1010B00041011713FFFF6700A3024A860A8597F0D4
:1010C000FFFFE78000234DBF1713FFFFE702A3FFD9
:1010D000B335B000011185052A891315F601336572
:1010E00015012308B1009305110136843AC632C0B8
:1010F0003EC442C297F0FFFFE780801DA24712481E
:10110000425593D68700230BF10093059101935725
:101110008800A30AD100A30BF100230C010197F072
:10112000FFFFE780E01A3247024603280400B33786
:10113000E000835644009207914411C2A1444A85BD
:10114000A68842860C0897F0FFFFE78040772A893F
:1011500019E5A685228597B0FFFFE780E0AA4A85BA
:1011600005611713FFFF670043F81713FFFFE7023E
:10117000E3F301113EC68647B335B0008505AA8961
:101180001315F6015D8D2308B10093051101368416
:101190003A89B28442C446C297F0FFFFE780401309
:1011A00022489248164593578800A30AF1009305F8
:1011B000910193D78800230B0101A30BF100230CAD
:1011C000110197F0FFFFE780A010324710408356CF
:1011D0004400B337E000920703280900914891C00A
:1011E000A1480C084E8597000000E780809CAA84E7
:1011F00001E9835544004A8597B0FFFFE780C0A00E
:10120000268505611713FFFF670083EDAA959307F5
:10121000F00F171701001307A7A46317B50013C534
:10122000F7FF1375F50F828005058346F5FFB58F2F
:10123000BA9783C70700D5B70357450014419307F2
:10124000F00F171601001306A6A136974207418337
:10125000139506014181631BE500AD8FB29703C56D
:101260000700130515F3133515008280850603C5A5
:10127000F6FFA98FB29783C70700D9BF1713FFFFE7
:10128000E70263E4B28736842E86BA86AA853E8555
:10129000BA8497F0FFFFE7806052634F0500228514
:1012A00097E00000E78060802A86A686A2852685D2
:1012B00097F0FFFFE78080501713FFFF6700E3E21E
:1012C0001713FFFFE70283DE5D712A8BAE8A1715C5
:1012D0000100130565962C00B284368ABA893E89CE
:1012E00097F0FFFFE780C04F2A845DE1341041464C
:1012F000DA85280097F0FFFFE780404C2A8449E90F
:101300008547A303F100A6C2930771002408BEC459
:10131000A68685470D462C18281002DC02DED6C0B2
:10132000BEC697F0FFFFE78000442A8435E183477B
:101330007102A6860D4693F7F7072300FA00C1470E
:101340003EDE2C188947281026DCA303F10097F015
:10135000FFFFE78040412A8405ED4146A6854E8582
:1013600097D00000E78060488D47A6860D462C1870
:101370002810A303F10097F0FFFFE780C03E2A8406
:1013800001E94146A6854A8597D00000E780E045FF
:10139000228561611713FFFF670083D41713FFFFD6
:1013A000E70263D297F70000938707EF984383C75C
:1013B000470079712A89AE84171501001305458805
:1013C0000C083AC42306F10097F0FFFFE780404184
:1013D0002A8405ED14104146CA85080897F0FFFFDE
:1013E000E780C03D2A8415E1140815462C0008103A
:1013F00097F0FFFFE780803C2A8401E921462C0812
:10140000268597D00000E780403E2285456117136E
:10141000FFFF670083CD1713FFFFE702C3CA97F7EB
:101420000000938767E79C477971AA842E8417157B
:101430000100130565810C083EC697F0FFFFE780A9
:10144000203A0DE914104146A685080897F0FFFFE1
:10145000E780C03605E1140811466C00081097F0CB
:10146000FFFFE780A03519E58347F10193F7F70304
:101470002300F40045611713FFFF670003C717132C
:10148000FFFFE70243C43688A14881470147E5468C
:1014900097F0FFFFE780A0421713FFFF6700E3C448
:1014A0001713FFFFE70223C23688A148814701478F
:1014B000E54697F0FFFFE780C06F1713FFFF670057
:1014C000C3C21713FFFFE70203C001112A842E8550
:1014D0000C0832C697F0FFFFE780803009ED3247F5
:1014E000970601009386C6741008C14522859700AF
:1014F0000000E780E0D805611713FFFF6700E3BE37
:101500001713FFFFE70223BC4111C1472EC032C4AD
:101510008A8509463EC23EC697F0FFFFE780A024B9
:1015200041011713FFFF670043BC1713FFFFE702DA
:1015300083B94111AE8613061009AA850A8502C037
:1015400002C202C402C697F0FFFFE78020274101D4
:101550001713FFFF670063B91713FFFFE702A3B676
:101560003287970601009386A66E2E8693050002A9
:1015700097000000E780C0D01713FFFF6700E3B6B5
:101580001713FFFFE70223B47971C1472ACC2ED08D
:1015900032D42C080D4628003ECE3ED23ED602C4A0
:1015A00002C602C802CA97F0FFFFE780C01B456170
:1015B0001713FFFF670063B31713FFFFE702A3B022
:1015C0000111AA842E84170501001305E5688A8598
:1015D00097F0FFFFE780C02015E514084146A68577
:1015E0000A8597F0FFFFE780601D09ED8347E10161
:1015F0000347F101A207D98FCA07C9836177D98F41
:101600002310F40005611713FFFF670003AE15CD2B
:101610001713FFFFE70223AB9747FF1F938707715D
:1016200090439745FF1F9385A5701745FF1F13052E
:10163000E56B97D00000E78000C51745FF1F130535
:10164000E56A1713FFFF670043AA1745FF1F13053D
:10165000E56982808DCD1713FFFFE702C3A6974788
:10166000FF1F9387A76C944301112E840A86974528
:10167000FF1F9385E56B97D00000E78040C60A8581
:101680000294014505611713FFFF670003A67D550E
:1016900082801713FFFFE70203A397D00000E780C3
:1016A00080D19747FF1F23A3A76817F5FFFF1305F6
:1016B000E5C997B00000E780C0741713FFFF67000B
:1016C000C3A21747FF1F1307A76893171500084306
:1016D0003E95FD572310F50082801713FFFFE702A8
:1016E000839E2A84084009E51713FFFF6700E39FE4
:1016F0001C4158401CC06313E5005CC08347550083
:1017000023200500F99BA302F50097A0FFFFE780C7
:10171000207CC9BF1713FFFFE70243999747FF1FBC
:101720009387076598432A8411CB8347350093F745
:10173000070289C70355050089450297130544012F
:1017400097B00000E780403B835504000355E40058
:1017500097300000E780A00C485819C597A0FFFFFC
:10176000E7800077232A0402130584039700000012
:10177000E780E0F68144B1499790FFFFE780C06DB4
:1017800063CBA402834734002320040493F727FC8F
:10179000A301F40000489790FFFFE780E06C131668
:1017A0001500814522859710FFFFE780C09417132D
:1017B000FFFF6700E392B387340303290403850422
:1017C0003E994A8597000000E78060F123040900F4
:1017D00065B78347350093F7070299E30145828097
:1017E0008357E500E39CB7FEC167FD176316F6005B
:1017F00005458280054599A81713FFFFE702A38CD2
:1018000093170601C187B2842A8401496359F00203
:10181000835705009DCB01456367F60003458400AF
:101820003E953325A6001375F50F0DA01C48131720
:101830001900BA9783D70700E38E97FA05099790A6
:10184000FFFFE7806062E343A9FE01451713FFFF36
:101850006700A3891713FFFFE7024385AE89AA84B7
:101860009790FFFFE78000562A8497D0FFFFE7801C
:10187000A02EAA86014713068401970500009385D0
:1018800085E41745FF1F1305E54C9790FFFFE780A0
:10189000801C2A8925C98C441304C50022859E0515
:1018A00093F5050897A0FFFFE780403CCC40838775
:1018B0007400E18163DD070493E50508228597A0A4
:1018C000FFFFE780A03A0D4693854400228597A04C
:1018D000FFFFE780C03683D50400228597A0FFFF75
:1018E000E780E03D83D52400228597A0FFFFE780B5
:1018F000003D03D6490083A50900228597A0FFFF7C
:10190000E780E0334A851703FFFF6700637D93F5A7
:10191000F5076DB71703FFFFE702E37A01112A8489
:10192000328532C697A0FFFFE780E0279780FFFF50
:10193000E7806034835704001747FF1F1307C75A17
:101940003246231BF100930700F8A30DF1001C475A
:101950001843231AA1008983858BB307F740B2850A
:1019600048083ECE231C0100230D01009700000013
:10197000E78080EE05611703FFFF67000377170319
:10198000FFFFE702A372004101453DC49304C40078
:1019900026853289AE8997A0FFFFE780C024954550
:1019A0002A8A2685035B040197A0FFFFE780202198
:1019B000268597A0FFFFE780603E8D45AA8A268591
:1019C00097A0FFFFE780A01F268597A0FFFFE78075
:1019D000E03C5C48420A135A0A01D2975CC42318BF
:1019E0006401814763983A0146054D8133062541DC
:1019F0009337160013F5F70F1703FFFF6700436EC9
:101A00001703FFFFE702A36989692A8BAE8B328A2D
:101A1000B68A81440144314CFD199790FFFFE7805D
:101A2000A04363CDA4009790FFFFE780E045018DC0
:101A300033B5AA001703FFFF6700E3693389840306
:101A400083270B003E9963170A00834789008504AA
:101A50003E94E1B703560A00DE854A8533F6C90095
:101A600097000000E780E0F16DD10545E1B717036D
:101A7000FFFFE702436501112A847C000355E5005E
:101A80003ECAB70707003ECC7C003ECE9720000040
:101A9000E78020082A898545480897A0FFFFE7804E
:101AA00020399945480897A0FFFFE780E015AA84F0
:101AB0004A8597200000E780A0082380A40097476C
:101AC000FF1F938767429C434166130606F0939677
:101AD000870113D78701558F93D68700F18E558FD5
:101AE000A207B706FF00F58FD98F11462C0013858A
:101AF00014003EC497D00000E78020CF5008A38296
:101B000004008945228597000000E780E0E019C9BC
:101B1000AA851305840397A0FFFFE780E0313C40CE
:101B200085073CC005611703FFFF6700035C1703CF
:101B3000FFFFE70243599790FFFFE780E0342A84D4
:101B400005049790FFFFE78020333305A402F14797
:101B500091453305F50297200000E78020BA11E592
:101B600065551703FFFF670043589747FF1F23A9D9
:101B7000A71E9790FFFFE78020312A8405049790E5
:101B8000FFFFE780602F3305A402894506059720F3
:101B90000000E780A0B669D59747FF1F23AAA71AC0
:101BA0009790FFFFE780402E2A8405049790FFFF5F
:101BB000E780802C3304A4029747FF1F239C8718DB
:101BC0009790FFFFE780402C2A849790FFFFE780E3
:101BD000A02A930714003385A7029747FF1F239C71
:101BE000A716970701009387E7CA1747FF1F232708
:101BF000F7160145BDB71703FFFFE702234BAA8481
:101C00002E8901449749FF1F9389092E130A8006E4
:101C10009790FFFFE78040266347A4000145170324
:101C2000FFFF6700E34B3305440383A709024A869D
:101C3000A6853E9597000000E780E0B919E105040C
:101C4000C1BF0545E9BF1703FFFFE7024345AA8A65
:101C50002E8BB28B368C3A8A814401448149974C51
:101C6000FF1F938C6C28130D80069790FFFFE78071
:101C7000A02063C9A40011E085494E851703FFFF2A
:101C8000670063453389A40383A70C025E86D6856B
:101C90003E994A8597000000E780E0B31DC1979008
:101CA000FFFFE780601E0544636D4501D2866286B2
:101CB000DA851305090397000000E780A0D411C15D
:101CC000854985045DB71703FFFFE702233EC16422
:101CD00041112A8901449749FF1F9389E920130A7A
:101CE0008006FD1436C632C42EC29790FFFFE780EF
:101CF000A01892452246B2466348A400014541011E
:101D00001703FFFF6700C33D3305440383A70902A0
:101D10003E9509C683473500C18B9DC791C6834751
:101D2000350093F707028DC3630699008357E500DA
:101D3000639C27010357050001CB63E7E500834758
:101D40008500BA97E3CDF5FA050469BF1703FFFFD5
:101D5000E702C335C1642A8901449749FF1F93896B
:101D6000A918130A8006FD149790FFFFE780C010A2
:101D70006346A4001703FFFF67008336330544035F
:101D800083A709023E958357E500638A97006304A1
:101D900099006396270197000000E780E09705040B
:101DA000E1B71703FFFFE702032F89692A8AAE8A8A
:101DB000328BB68B8144174CFF1F130CEC12930C23
:101DC0008006314DFD199790FFFFE780E00A63C65A
:101DD000A4001703FFFF6700C32F338994038327F1
:101DE0000C028355CA015A863E994A859700000025
:101DF000E780609E31C1814D15A03384AD038327F8
:101E0000090303D60B00D68533F6C9003E9422851C
:101E100097000000E780E0B609E9850D9790FFFF85
:101E2000E7808003E3CBADFC01A82285970000008A
:101E3000E780E08A23040400850471B71703FFFFDD
:101E4000E702E3254169AA8A014A174BFF1F130BDA
:101E5000AB097D19C14B054C9790FFFFE780C0018E
:101E60006346AA001703FFFF6700E3269309800675
:101E7000B3073A0383290B02BE9983D7E900638E27
:101E8000270163842A01639A570103A4890301E8A7
:101E90004E8597000000E780C0BD050A75BF8357D7
:101EA0000401639977099304C400268597A0FFFF76
:101EB000E78060D385452A8D2685835C040197A041
:101EC000FFFFE780C0CF268597A0FFFFE780A0E750
:101ED00062056185635905048D45268597A0FFFF3E
:101EE000E780E0CD8945268597A0FFFFE78020CDDC
:101EF0008945268597A0FFFFE78060CC854526852C
:101F000097A0FFFFE780E0CC83470500094793F7E0
:101F1000F707639AE7009945268597A0FFFFE780BA
:101F200040CBA30285014848337D2D01231894013D
:101F30006A9548C40040A1BF1703FFFFE702A3183A
:101F400037E404008327041D82979747FF1F83C748
:101F5000A7E61715FF1F1305A55BA300F500832750
:101F6000441C82978327841C81461306F00F814509
:101F7000014582971703FFFF670023171747FF1FCD
:101F8000130787D318439745FF1F83C5E5E297479B
:101F9000FF1F9387E7E08346870303469703639712
:101FA000D5009747FF1F2389C7E0828083C587013B
:101FB0000347A7036317B6009747FF1F238EE7DE8B
:101FC000828003C687016317C7009747FF1F2385D9
:101FD000D7DE828083C68701130750026319D700BA
:101FE000930760021747FF1F2308F7DC828083C630
:101FF0008701130660026315D60093077002DDB7F0
:1020000083C7870155BF9747FF1F938767D9D44B75
:102010000947638DE6081703FFFFE702C30A174964
:10202000FF1F130929D53E8483470900918B9DCF5B
:10203000B7E4040083A7041D829783A7441C1745B7
:10204000FF1F1305A5D3829783A7841C81461746DB
:10205000FF1F0346A6D481450145829721C58347CA
:102060000900ED9B1747FF1F2306F7D083470400A5
:1020700093F7F70F85CB91471747FF1F232CF7D214
:1020800097000000E78080EB97000000E78040EFBA
:10209000B7E70400BC4F414691451745FF1F034574
:1020A000A5D082971703FFFF6700230482801703E0
:1020B000FFFFE70243018D4741116306F504C54761
:1020C0006308F50285476310F5029747FF1F2387D2
:1020D000A7CEB7E70400BC4B930500101745FF1FC0
:1020E000034585CC829741011703FFFF6700E3FF9B
:1020F00085471747FF1F2303F7CCB7E70400BC4B06
:1021000093050020E1BF9747FF1F938767C9D44B12
:102110001147638DE600B7E7040083A7071D829788
:10212000B7E70400BC4B930500044DBF05491747B2
:10213000FF1F232127C983C7070032C62E8493F7C8
:10214000F70FD5D3B7E4040083A7041D7D141374DF
:10215000F40F8297E37689FCB245994703C61500D0
:10216000E3F0C7FCFC4409061745FF1F130545C5EE
:102170008297BC48930500081745FF1F0345C5C259
:10218000829779BF1703FFFFE702E3F31747FF1FAB
:10219000130707C14047184B1C409746FF1F23A752
:1021A000F6C06316E4001747FF1F2323F7C013058B
:1021B00084FE9790FFFFE78000AA035564FF978095
:1021C000FFFFE780807297A0FFFFE78060D01703D2
:1021D000FFFF670083F11703FFFFE702C3EE974796
:1021E000FF1F9387E7BBD84BDC4789C797000000E8
:1021F000E78080F985471747FF1F232DF7BA9747D8
:10220000FF1F938767AB9C43930500021745FF1F91
:10221000034585B983C787031747FF1F230EF7B808
:10222000B7E70400BC4B82971703FFFF6700E3EB9F
:102230009747FF1F23A8A7B682801703FFFFE70277
:10224000E3E637E404007C4CA1451745FF1F034536
:10225000A5B582977C48A1451745FF1F0345C5B426
:102260009744FF1F9384C4B38297DC4489EB9700A3
:102270000000E78080D91703FFFF670063E603D5FE
:1022800067FF9780FFFFE7804066AA896DD1D84835
:1022900091476310F7027C4C91451745FF1F03459A
:1022A000A5B082977C4891451745FF1F0345C5AFF0
:1022B000829703A9490103D409018947B7E90400BA
:1022C0001747FF1F2328F7AE83A7091D21044204E7
:1022D000829783C784011715FF1F130565236119B2
:1022E0001717FF1FA306F72283A7491C4180829777
:1022F0009747FF1F238407AC83A7C91C8146094663
:102300009375F40F4A85829711E99747FF1F83C79A
:1023100027BB89C79710FF1FE780208CB7E7040011
:10232000BC4F2146A1451745FF1F0345E5A78297EE
:1023300099B71703FFFFE70203D993F705200111AF
:102340002E8481CF97000000E78020E91345042008
:1023500005611703FFFF670043D993F70510A9CF65
:102360009744FF1F9384C4A3DC4897000000E780D4
:1023700020C11747FF1F13072794184383C7840101
:10238000034787036318F700DC4489C79700000000
:10239000E78080DF85471747FF1F232DF7A0B7E7AA
:1023A0000400BC4B930500021745FF1F0345C59F62
:1023B00082971345041069BF93F70508BDC7974777
:1023C000FF1F83C7F79FE91719469745FF1F93859E
:1023D000459F1305D10093F4F70F1749FF1F0349D9
:1023E000299E97C00000E780404093970401C18375
:1023F0001747FF1F1307479D231DF100231CF10002
:102400009747FF1F9387C7993ACE3ACAD843230606
:10241000010009CBDC439315890154080D46E18581
:10242000680082971345040825B793F72500A5C3D4
:102430009747FF1F9387C796D84B89476306F702D4
:102440009747FF1F83C7079313F7270011EF918B5F
:1024500099CFB7E70400BC4F1306000A894517451A
:10246000FF1F03456594829713452400D5B5974710
:10247000FF1F938767849C4383C787031747FF1F0A
:10248000230CF79297000000E78060DBF1BF93F721
:10249000050281CB97000000E78060DA1345040253
:1024A00045BD93F7850081CB97000000E780E0D21F
:1024B0001345840071BD93F7150081CB9700000090
:1024C000E780A0B41345140061B593F7450081CBB4
:1024D00097000000E78060B31345440095BD93F773
:1024E000050495C39747FF1F83C7878B91CB970040
:1024F0000000E780A0A491471747FF1F232CF78A0D
:1025000013450404B1B593F705010145E38207E4DF
:102510009747FF1F9387C788D84B91476310F704ED
:102520009747FF1F938707859C4313D72700858311
:10253000D98F858B91E7B7E7040083A7071D8297A2
:10254000B7E70400FC4F91451745FF1F0345C585BC
:10255000829785471747FF1F232EF78413450401F1
:10256000C5BB9747FF1F238DA79482801703FFFFEA
:10257000E70263B59747FF1F23AA07829747FF1F0C
:1025800023A8078285471734FF1F1304E4721747F7
:10259000FF1F2321F7821C4083C787031747FF1FB4
:1025A000230CF7809790FFFFE780409329C597178A
:1025B000FF1F23A3A7F61C40170500001305A5D78E
:1025C00083C787031737FF1F2308F77E1717FF1FDF
:1025D000A300F7F49737FF1FA384077CB7E7040035
:1025E00083A7070882979737FF1F238FA77A1703C0
:1025F000FFFF670083AFB7C7898E938767ED171713
:10260000FF1F232BF7F045BF1737FF1F03474779FD
:10261000795555E79737FF1F9387877803C71700CA
:1026200005079736FF1FA38DE67603C717008D4673
:102630003377D7029736FF1FA384E67683C6170049
:102640001737FF1F13074767184393F6F60FA9EED6
:10265000834787031737FF1F2300F7768547173710
:10266000FF1F230FF7729737FF1F9387A7709C43B5
:102670000145998BA9E71703FFFFE702C3A437E4DD
:1026800004007C48C1451735FF1F0345E57182975B
:102690003C4885451735FF1F034505718297014565
:1026A0001703FFFF670063A483C717008546639580
:1026B000F6008347970379BF8347A70361BF8280F2
:1026C0009737FF1F83C7C76DA1CF1703FFFFE7022F
:1026D000839F37E404009737FF1F2383076C7C48F0
:1026E00085451735FF1F0345256C82977C4C914526
:1026F0001735FF1F0345456B82977C489145173579
:10270000FF1F0345656A82973C48C1451735FF1F87
:1027100003458569829701451703FFFF6700E39C26
:10272000795582801703FFFFE702E3992A84035556
:1027300065FF9780FFFFE780401B9737FF1F938758
:102740002766D847BE841DEF9790FFFFE78080770C
:102750009C48232004009DEB9737FF1F23AA876422
:102760009737FF1F23A48764B7E70400BC4B894554
:102770001735FF1F03454563829701451703FFFF88
:102780006700A396630A8700184375BF80C3973715
:10279000FF1F23AF8760C9BF7955CDB71703FFFF70
:1027A000E70263929737FF1F9387C77188432326F9
:1027B000050023240500510597A00000E780C033E1
:1027C0001703FFFF670063921703FFFFE702A38F62
:1027D0001734FF1F1304046F1C40411199CF9C470D
:1027E0002302B5002AC61CC197000000E78040FB09
:1027F0001C409C4B99C33245829741011703FFFF50
:102800006700A38E1703FFFFE702E38B4111444DDE
:10281000328532842EC69790FFFFE780C0522AC4CB
:1028200022859790FFFFE780205403A84400630CA3
:102830000800B245835744001840224683D545001E
:10284000AA862685029841011703FFFF6700E389E6
:102850001703FFFFE7022387404D1DC808C09705F7
:102860000000938565031305440197A00000E780ED
:1028700040169737FF1F9387E7649C43014589E71C
:102880009737FF1F23A087641703FFFF6700E385C7
:102890007D55DDBF1703FFFFE702E38201116800EA
:1028A0009305F00F02C602C802CA02CC02CE9700FE
:1028B0000000E780A0F105611703FFFF6700E382D6
:1028C0009737FF1F938707609C43D847A1679D07F1
:1028D0006319F70217F3FEFFE702E37E0111328569
:1028E0009790FFFFE7802046230AA10081456800FA
:1028F00097000000E78080ED056117F3FEFF670099
:10290000C37E82809737FF1F9387C75B9C43D8475E
:10291000A167938777036319F70217F3FEFFE702B6
:10292000837A011132859790FFFFE780C041230A27
:10293000A1008145680097000000E78020E905615B
:1029400017F3FEFF6700637A82809737FF1F938734
:1029500067579C43D84795476316F70417F3FEFF64
:10296000E70263760111328532849790FFFFE7809A
:10297000803D230AA10022859790FFFFE780C03E9B
:1029800083574400231BA10081453ECC1C406800B6
:102990003ECE97000000E78060E3056117F3FEFF7D
:1029A0006700A3748280930785FF8DC38327C5FFCB
:1029B00091CFDC4B81CF17F3FEFFE702C3700325F5
:1029C00085FF829717F3FEFF67002372828017F35B
:1029D000FEFFE702436F2A8432859790FFFFE7806E
:1029E0008036BD4763EBA70018449377F500034595
:1029F000B70041995D8DA305A70017F3FEFF67009F
:102A0000C36E17F3FEFFE702036C01117C003ECAA0
:102A1000B70707003ECC7C003ECE5C4DA9C72A8498
:102A200013858700AE8497A00000E780E0FCA165D5
:102A30002A899D0548089770FFFFE780603E93054F
:102A4000803EB345B902480893F5F50F9790FFFF14
:102A5000E780C021014781465008A68522859770EE
:102A6000FFFFE7804061056117F3FEFF6700E36742
:102A700017F3FEFFE702236597000000E780A0F848
:102A800017F3FEFF6700636617F3FEFFE702A36319
:102A900001117C00AE843ECAA165B70707002A84F5
:102AA0003ECC48087C00938575033ECE9770FFFFAF
:102AB000E78000371C44480883C5B700BD8997905C
:102AC000FFFFE780A01A500801478146A6852285AE
:102AD0009770FFFFE780205A056117F3FEFF67003C
:102AE000C36017F3FEFFE702035E2A84AE849700FB
:102AF0000000E78000EEA685228597000000E780B1
:102B0000E0F817F3FEFF6700435E17F3FEFFE702EE
:102B1000835B97000000E78060F717F3FEFF670014
:102B2000C35C17F3FEFFE702035A0329C5014111F5
:102B3000630809022A843285B2849790FFFFE780F8
:102B400080202AC626859790FFFFE780E021832713
:102B500049002A8691C7DC4781C7B2452285829702
:102B6000410117F3FEFF6700435817F3FEFFE7022A
:102B70008355444D91CC2A8432859790FFFFE7809E
:102B8000A01EDC40AA8589C79C4799C322858297ED
:102B900017F3FEFF6700635517F3FEFFE7020351CB
:102BA000032AC5014111630D0A062E89AA849545A1
:102BB000328532849770FFFFE78080268545228525
:102BC0009790FFFFE7804004AA89CA8522859790E5
:102BD000FFFFE780A00B83274A008DCBDC439DC716
:102BE00022859790FFFFE780A00083274A001040CE
:102BF00083564400DC437115A307A100B296130766
